:020000040800F2
:1000000000000110D96B030879710208A95F01088B
:10001000DD6C0308DD6C0308DD6C030800000000E4
:10002000000000000000000000000000C57702088A
:10003000C177020800000000BD77020889060108A8
:10004000DD6C0308DD6C0308DD6C0308DD6C030860
:10005000DD6C0308DD6C0308A18D0008918E00089B
:10006000DD6C0308558E0008198E0008FDAA0008F3
:10007000EDAA0008DDAA0008CDAA0008BDAA000864
:10008000A9AA000895AA0008DD6C0308DD6C030826
:10009000DD6C0308DD6C0308DD6C0308DD8D0008F2
:1000A000DD6C0308DD6C0308DD6C0308DD6C030800
:1000B00031FB000821FB0008DD6C0308DD6C030840
:1000C000DD6C0308DD6C0308DD6C0308DD6C0308E0
:1000D000DD6C03084D080108DD6C0308B107010859
:1000E000678D0008DD6C0308C9770208E1FA000893
:1000F000F1FA0008DD6C030801FB000881AA000882
:10010000DD6C0308DD6C030811FB0008DD6C0308DF
:10011000DD6C0308DD6C0308DD6C0308DD6C03088F
:100120006DAA000859AA000845AA000831AA0008CB
:100130001DAA0008DD6C0308DD6C0308DD6C0308F4
:10014000DD6C0308DD6C0308DD6C03087D710208BB
:1001500009AA0008F5A90008E1A900081507010887
:10016000DD6C0308DD6C0308DD6C0308DD6C03083F
:10017000DD6C0308DD6C0308DD6C0308DD6C03082F
:08018000DD6C0308DD6C0308CF
:1001880002020300B81D0020B41D0020000000007A
:100198000000000014000200342300208C230020FB
:1001A80000000000AC0500080B100C00701F0020B8
:1001B8009023002000000000AE050008270004007E
:1001C800C8240020C825002000000000BA05000847
:1001D80016000800CC250020D425002000000000CF
:1001E800BE050008010104002C2C0020883A0020DC
:1001F800000000000000000008020900FC3900208F
:100208008C3A00200000000001800008FA0101007B
:10021800263A0020983A002000000000C605000891
:1002280002000C00083A00209C3A00200000000060
:100238000000000003123200BE3C00208C3C00206D
:10024800000000000000000025005A00D83B0020F4
:10025800323C00200000000000000000F601080009
:10026800D03B0020C83B0020000000000000000038
:10027800150070009C3F0020844000200000000012
:100288000000000003000100983F0020F440002017
:1002980000000000000000002A006000A83E0020C6
:1002A800F84000200000000061000208000205007C
:1002B8005841002084440020000000000000000095
:1002C8001E000400604100208C4400200000000053
:1002D800C805000822000C000044002090440020BB
:1002E80000000000CC0500080C002400B0450020E8
:1002F8001C5300200000000059C001080E00DE0059
:10030800B444002040530020000000007109030895
:100318001300040040460020205400200000000084
:10032800D805000802010300A3440020245400203B
:100338000000000081C001081F000E00F4540020D6
:100348007C55002000000000DC05000805020100C3
:10035800485500208C55002000000000EA050008E0
:1003680005000500C2550020FC56002000000000D2
:10037800EC050008120016009955002004570020CB
:1003880000000000F20500080400C00038720020D8
:10039800D47300200000000000000000F9010400F0
:1003A800787A00207C7A00200000000081F00008A4
:1003B80018002C00447A0020807A002000000000F9
:1003C8001995020806001A0068750020AC7A00200A
:1003D8000000000091090308340010009474002004
:1003E800C87A002000000000890002082C001000D4
:1003F800647C0020547C00200000000071910208F9
:100408002B002400987C0020747C00200000000051
:1004180041910208FD012400E47E0020487F00206D
:100428000000000011F00008FE010800D07E002046
:100438006C7F002000000000C5EC000803010600E6
:10044800E47F0020F87F0020000000000806000874
:100458001B00F400088000209881002000000000A4
:100468001D17020829005000D4850020608600204E
:100478000000000000000000FB010100E4A50020CE
:1004880008A7002000000000BDEC0008FC010900DE
:10049800ACA400200CA700200000000089EC000894
:1004A800F7010600A4A4002018A7002000000000FF
:1004B8000E0600080A0012001099002020A700204C
:1004C80000000000140600080D003400DC9800202D
:1004D80034A70020000000000595010811000C0059
:1004E800708D002068A7002000000000294E030836
:1004F80001000A00D4AD0020E0AD0020000000009B
:10050800260600081A000800C0AD0020ECAD002047
:100518000000000030060008100003005CB0002056
:1005280060B00020000000003806000828000C0019
:1005380050B0002064B00020000000003C06000815
:100548002600080048B0002070B00020000000001D
:100558004806000823000E0038B0002078B00020BC
:100568000000000071DB02081900050030B000200F
:1005780088B000200000000050060008F8010100C3
:100588002CB0002090B000200000000056060008A3
:100598000001040028B0002094B0002000000000F2
:0405A80058060008E9
:1005AC0003002B21231E0002000001000A0120037E
:1005BC000000C409000019012828230000000100D4
:1005CC00C800141E010064002C0128000801000062
:1005DC000000000000000100000000050000000009
:1005EC0001010300010000000001000000000000F8
:1005FC0000000000000000000000000004010100E9
:10060C00000026010000000000300100005A00002C
:10061C00000090012C01C80064000A0AE8030000E5
:10062C00640001007E05EA05B405320000010500F6
:10063C00000000010000000000000000011558023D
:10064C00D903C5030000280100000400900100003C
:10065C005001000007000000020000000000000034
:10066C000000000001020304060708090101000054
:10067C0030C103080CD40308000000000000000087
:10068C0040C1030848C1030800000000012000001D
:10069C004CC1030854C103080000000001400000D5
:1006AC0058C1030838ED03080000000001200000C9
:1006BC0064C1030870C103080000000004000000BE
:1006CC0074C1030880C1030800000000040000008E
:1006DC0084C103087CE40308000000000100000052
:1006EC00020000000000803F0000803FFF0000007F
:1006FC001D250308D5240308252403080000000049
:10070C002122030859230308F9230308C1220308F3
:10071C000000000000000000D569020855690208BD
:10072C00516902084D690208416902083D690208D5
:10073C004969020845690208C9690208BD690208CD
:10074C0095690208A9690208816902086D690208A5
:10075C0059690208109E03080508040000000000F7
:10076C00B0AE03084CAE0308FC9D0308000000006B
:10077C003C9E030805080A0000000000B0AE030808
:10078C004CAE0308F0A5030800000000FFFFFFFFBC
:10079C000000803F20700020702D7200AA550300CD
:1007AC009FAA5505010000AA550701000001AA5592
:1007BC000B010000AA550902000000000100000016
:1007CC00000000000001000000000000000000001C
:1007DC00C4D803080E000000000000000000000058
:1007EC0000000000740E0020FFFFFFFFFA00000065
:1007FC0001000000010000005CD4030800000000B0
:10080C0000000000000000000000000051D40308AC
:10081C00040000007DBA0208000000000000000087
:10082C0064D4030801000000000000000000000078
:10083C0000000000000000000D000000000000009F
:10084C0000000000000000001E2300200100C4096D
:10085C00000000001C2300200100C409000000005F
:10086C001A2300200100C4090000000018230020F6
:10087C000100C40900000000142300200100C40979
:10088C0000000000162300200100C4090000000035
:10089C00122300200100C4090000000010230020D6
:1008AC000100C4090000000090D403080E000000F1
:1008BC00000000000000000000000000A801002063
:1008CC00E07F00209CFF2C01000000007411002030
:1008DC000A000000F0A50308847F0020E0150C1727
:1008EC000000000076110020080000004CAE030848
:1008FC007511002005000000B0AE0308867F0020B3
:10090C000200000008A60308C855002001200100C1
:10091C00C75500200200000014A603089A450020C9
:10092C000000F40101000000984500200000F401D3
:10093C0001000000964500200000F40101000000B9
:10094C00944500200000F4010100000092450020B5
:10095C0000FF0100AE450020E803D0070A000000AC
:10096C00AC450020006401000A000000AD450020E9
:10097C00006401000A000000A6450020006401008C
:10098C000A000000AB450020006401000A000000D2
:10099C00AA450020006401000A000000A9450020BF
:1009AC00006401000A000000A545002000FF0100C2
:1009BC000A000000A445002000FF01000A0000000E
:1009CC00B04400200000F40101000000AE440020FF
:1009DC000000F40101000000AC4400200000F40110
:1009EC0001000000AA4400200000F40101000000F6
:1009FC00A145002000C80100A045002000C801004E
:100A0C009F45002000C801009E45002000640100A5
:100A1C000A0000009D45002000FF01000A000000B4
:100A2C009855002000C801009755002000C801000F
:100A3C009655002000C801009555002000C8010003
:100A4C009455002000C801009355002000C80100F7
:100A5C009255002000C801009155002000C80100EB
:100A6C009055002000C8010098D403080000000035
:100A7C00000000000000000000000000A8D40308E3
:100A8C0009000000000000004C02002004000000DF
:100A9C00B0D4030809000000000000004002002050
:100AAC000400000074D703080900000000000000D7
:100ABC003402002004000000B8D403080900000030
:100ACC00000000002802002004000000BCD4030831
:100ADC0009000000000000001C02002004000000BF
:100AEC00C4D403080900000000000000100200201C
:100AFC0004000000CCD40308090000000000000032
:100B0C000402002004000000D4D4030809000000F3
:100B1C0000000000F80100200400000064D4030869
:100B2C0001000000000000000000000000000000B8
:100B3C00000000000D00000000000000000000009C
:100B4C0000000000DCD403080000000000000000DE
:100B5C000000000000000000ECD4030805000000B9
:100B6C0000000000A94400200000000064D4030829
:100B7C000100000000000000000000000000000068
:100B8C00000000000D00000000000000000000004C
:100B9C0000000000F4D40308000000000000000076
:100BAC0000000000000000000CD40308000000004E
:100BBC0000000000741300200400000000D503089E
:100BCC000C00000015BB0208AC0200200000000065
:100BDC0034DA03080C000000E1B80208A00200207F
:100BEC000000000004D503080C000000C5B8020882
:100BFC0094020020000000000CD50308080000003F
:100C0C0000000000880200200400000014D5030836
:100C1C000C00000031B802087C020020000000002B
:100C2C001CD5030809000000000000007002002021
:100C3C000400000024D5030803000000A159020899
:100C4C00580200200000000064D4030801000000DA
:100C5C000000000000000000000000000000000088
:100C6C000D0000000000000000000000000000006B
:100C7C0028D5030800000000000000000000000060
:100C8C000000000038D503080C0000000000000034
:100C9C00C00200200000000040D503080A0000003C
:100CAC000000000024560020000000004CD5030872
:100CBC000A000000000000002C560020000000007C
:100CCC0054D503080A000000000000003456002030
:100CDC00000000005CD503080700000000000000C5
:100CEC00B80200200000000068D5030804000000D2
:100CFC00DD5A0208000000000000000064D4030864
:100D0C0001000000000000000000000000000000D6
:100D1C00000000000D0000000000000000000000BA
:100D2C000000000074D50308000000000000000063
:100D3C00000000000000000088D503080700000038
:100D4C0000000000FC0200200000000094D5030805
:100D5C000800000000000000F0020020000000006D
:100D6C00A0D503080800000000000000E4020020E9
:100D7C0000000000ACD503080800000000000000D3
:100D8C00D802002000000000B8D5030808000000BD
:100D9C0000000000CC0200200000000064D4030816
:100DAC000100000000000000000000000000000036
:100DBC00000000000D00000000000000000000001A
:100DCC0000000000C4D50308000000000000000073
:100DDC004701002000000000D0D503080B000000E4
:100DEC00000000006403002000000000D8D50308B8
:100DFC000B00000000000000580300200000000061
:100E0C00E4D503080B000000000000004C03002098
:100E1C0000000000F0D503080B00000000000000EB
:100E2C004003002000000000FCD503080B0000006C
:100E3C0000000000340300200000000008D6030866
:100E4C000B00000000000000280300200000000040
:100E5C0010D603080B000000000000001C0300204B
:100E6C00000000001CD603080B000000000000006E
:100E7C00100300200000000028D603080800000022
:100E8C0000000000040300200000000064D40308EC
:100E9C000100000000000000000000000000000045
:100EAC00000000000D000000000000000000000029
:100EBC000000000034D60308000000000000000011
:100ECC00000000000000000048D6030808000000E5
:100EDC0000000000940300200000000054D603081A
:100EEC000800000000000000880300200000000043
:100EFC0060D6030808000000000000007C030020FE
:100F0C00000000006CD60308080000000000000080
:100F1C00700300200000000064D4030801000000EE
:100F2C0000000000000000000000000000000000B5
:100F3C000D00000000000000000000000000000098
:100F4C0074D60308000000000000000044010020DB
:100F5C000000000084D603080B0000000000000015
:100F6C00C40300200000000090D603080B00000012
:100F7C0000000000B8030020000000009CD603080D
:100F8C000700000000000000B0030020000000007B
:100F9C00A8D603080700000000000000A8030020EA
:100FAC0000000000B4D60308070000000000000099
:100FBC00A00300200000000064D40308010000001E
:100FCC000000000000000000000000000000000015
:100FDC000D000000000000000000000000000000F8
:100FEC00C0D60308000000000000000044010020EF
:100FFC0000000000CCD60308070000000000000031
:10100C001004002000000000D4D6030807000000E4
:10101C00000000000804002000000000DCD60308DB
:10102C000700000000000000000400200000000089
:10103C00E4D603080700000000000000F8030020BD
:10104C0000000000ECD603080700000000000000C0
:10105C00F003002000000000F4D603080700000095
:10106C0000000000E803002000000000FCD603088C
:10107C000700000000000000E0030020000000005A
:10108C0004D703080700000000000000D80300206C
:10109C00000000000CD7030807000000000000004F
:1010AC00D00300200000000064D4030801000000FD
:1010BC000000000000000000000000000000000024
:1010CC000D00000000000000000000000000000007
:1010DC0014D703080E000000000000003132020893
:1010EC000000000018040020A74400200A32010070
:1010FC00A644002001FA0100A244002000C801000F
:10110C00A0440020E803D00701000000534F554CC9
:10111C00463400001CD703080E00000047320208BA
:10112C00000000008F380208F404002024D70308C4
:10113C000E0000006DB80208000000000000000066
:10114C00440500202CD703080E000000BD5A0208ED
:10115C00B5580208C15702082006002034D70308EE
:10116C000E000000E1320208B1320208000000005B
:10117C00D40600203CD703080E00000059330208A7
:10118C00E95602080000000074070020A245002068
:10119C000103010048D703080E0000008D3202083D
:1011AC0069320208000000006408002050D70308D0
:1011BC000E00000011330208B938020800000000CC
:1011CC00F00800205CD703080E0000001557020839
:1011DC002358020800000000900900209C450020C4
:1011EC000103010064D703080000000000000000A8
:1011FC00000000000000000070D703080800000089
:10120C0000000000B00A00200000000078D703089E
:10121C000700000000000000A80A002000000000E9
:10122C0088D703080700000000000000A00A002077
:10123C000000000094D70308070000000000000025
:10124C00980A002000000000A0D70308030000004B
:10125C00A1590208800A00200000000064D4030891
:10126C000100000000000000000000000000000071
:10127C00000000000D000000000000000000000055
:10128C0000000000A8D703080000000000000000C8
:10129C000000000000000000B8D703080A0000009E
:1012AC000000000090C1030800000000C0D7030834
:1012BC000A00000000000000C8D70308000000006E
:1012CC00D0D703080A00000000000000AF55002032
:1012DC0000000000D8D703080A000000000000003E
:1012EC00BC0A00200000000064D4030801000000C8
:1012FC0000000000000000000000000000000000E2
:10130C000D000000000000000000000000000000C4
:10131C00E0D70308000000000000000000000000FF
:10132C0000000000B0C2030803000000A15902082D
:10133C00F40A002000000000F4D7030803000000AA
:10134C00A15902087811002000000000FCD7030806
:10135C0003000000A1590208DC0A00200000000074
:10136C0004D8030803000000A1590208C40A002095
:10137C000000000064D4030801000000000000001D
:10138C000000000000000000000000000D00000044
:10139C0000000000000000000000000010D803084E
:1013AC000000000000000000000000000000000031
:1013BC001CD8030807000000755802088C0B00208D
:1013CC0000000000C8F2030803000000A159020845
:1013DC00740B00200000000028D803080300000054
:1013EC00A15902085C0B00200000000030D8030853
:1013FC0003000000A1590208440B0020000000006B
:10140C0038D8030807000000555802083C0B002090
:10141C000000000050DA030803000000A159020884
:10142C00240B00200000000044D803080300000037
:10143C00A15902080C0B00200000000064D4030822
:10144C00010000000000000000000000000000008F
:10145C00000000000D000000000000000000000073
:10146C000000000050D803080E00000005320208EE
:10147C00D731020800000000940B002058D8030854
:10148C000E0000009557020800000000000000004C
:10149C00340C002064D803080E000000000000008B
:1014AC000000000000000000C00C002074D80308ED
:1014BC000E00000061570208955802080000000059
:1014CC004C0D00207CD80308000000000000000038
:1014DC00000000000000000088D803080300000092
:1014EC00A15902085C0E00200000000068D8030817
:1014FC0003000000A1590208440E00200000000067
:10150C0090D8030803000000A15902082C0E0020FB
:10151C00000000009CD8030803000000A159020839
:10152C00140E002000000000A4D8030802000000E4
:10153C00295B02080000000000000000ACD8030882
:10154C0002000000295B02080100000000000000FE
:10155C00B8D8030802000000295B02080200000052
:10156C0000000000000000000D0000000000000062
:10157C000000000000000000040309041201000236
:10158C0002020040830440570002010203010000E4
:10159C0009024300020100C03209040000010202EA
:1015AC00010005240010010524010001042402029D
:1015BC000524060001070582030800FF0904010049
:1015CC00020A000000070501024000000705810225
:1015DC00400000007527030875260308F12703084F
:1015EC007D220308B12503088D220308A9220308D4
:1015FC0055220308452203080000000000000000EB
:10160C000100000000600240106002400000000079
:10161C00000B000000002000000000000000000093
:10162C00006002402860024000000000060C000030
:10163C0000002000000000000000000000600240DC
:10164C004060024000000000100D0000000020006F
:10165C0000000000000000000060024058600240E2
:10166C0000000000160E000000002000000000002A
:10167C0000000000006002407060024000000000AA
:10168C00200F0000000020000000000000000000FF
:10169C00006002408860024000000000261000003C
:1016AC00000020000000000000000000006002406C
:1016BC00A06002400000000030110000000020007B
:1016CC00000000000000000000600240B860024012
:1016DC0000000000362F0000000020000000000079
:1016EC000000000000640240106402400000000092
:1016FC000038000000004000000000000000000066
:10170C00006402402864024000000000063900001A
:10171C0000004000000000000000000000640240D7
:10172C004064024000000000103A0000000040003D
:10173C0000000000000000000064024058640240F9
:10174C0000000000163B00000000400000000000FC
:10175C0000000000006402407064024000000000C1
:10176C00203C0000000040000000000000000000D1
:10177C00006402408864024000000000264400001F
:10178C000000400000000000000000000064024067
:10179C00A064024000000000304500000000400042
:1017AC00000000000000000000640240B864024029
:1017BC000000000036460000000040000000000061
:1017CC000000000001010100D4DA03080E00000043
:1017DC0065B902080000000000000000F8120020AB
:1017EC00A8DA030800000000000000000000000060
:1017FC00000000000CD403080000000000000000F2
:10180C00B01700200400000034DA03080C000000BC
:10181C00495102088C1700200000000004D5030871
:10182C000C0000002151020880170020000000006D
:10183C000CD50308080000000000000074170020FD
:10184C000400000014D503080C000000A74B02088C
:10185C00681700200000000024D5030803000000D6
:10186C00A15902085017002000000000B8DA030844
:10187C0003000000A15902083817002000000000E6
:10188C0064D4030801000000000000000000000008
:10189C0000000000000000000D000000000000002F
:1018AC000000000000000000A8DA0308000000009F
:1018BC000000000000000000000000000CD4030831
:1018CC000000000000000000B01700200400000021
:1018DC00E0D90308030000001BBA020820170020FF
:1018EC000800000014D503080C000000A74B0208E8
:1018FC00681700200000000024D503080300000036
:10190C00A15902085017002000000000B8DA0308A3
:10191C0003000000A1590208381700200000000045
:10192C0064D4030801000000000000000000000067
:10193C0000000000000000000D000000000000008E
:10194C000000000000000000C0DA030800000000E6
:10195C000000000000000000000000000CD4030890
:10196C000000000000000000B01700200400000080
:10197C00E8D9030803000000A159020898170020B9
:10198C000000000064D40308010000000000000007
:10199C000000000000000000000000000D0000002E
:1019AC0000000000000000000000000000FFFF002D
:1019BC000000000000000000010203040102030407
:1019CC00060708092D202D2D202D2D2D2D202D2DF8
:1019DC002D2D0000000000000000000000000000A1
:1019EC00000000009C7F002088130C1701000000F1
:1019FC009E7F002088130C170000000038D90308C4
:101A0C0000000000000000000000000000000000CA
:101A1C0048D903080800000000000000A0130020B3
:101A2C000400000054D90308080000000000000066
:101A3C00941300200000000024D5030804000000CB
:101A4C0055BB0208000000000000000064D403082D
:101A5C000100000000000000000000000000000079
:101A6C00000000000D00000000000000000000005D
:101A7C0000000000C01200009A7F002088130C1791
:101A8C0001000000987F002088130C170000000054
:101A9C0090D903080E000000B9B90208000000003C
:101AAC0000000000AC130020CB7F002001000000E0
:101ABC0070AE0308967F0020010000007CAE030886
:101ACC00C87F00200200000084AE0308CE73002003
:101ADC000000000000000000CC730020000000009B
:101AEC0000000000CA73002000000000000000008D
:101AFC00C87300200000000000000000C673002026
:101B0C000000000000000000C47300200000000072
:101B1C000000000024140020000000000000000061
:101B2C00957F00200200000090AE030898D90308AE
:101B3C000000000000000000000000000000000099
:101B4C0048D90308080000000000000034140020ED
:101B5C000400000054D90308080000000000000035
:101B6C00281400200000000024D503080400000005
:101B7C0099B90208000000000000000064D40308BA
:101B8C000100000000000000000000000000000048
:101B9C00000000000D00000000000000000000002C
:101BAC0000000000A8D9030800000000000000009D
:101BBC000000000000000000B8D903080C00000071
:101BCC00314A02087014002004000000C4D9030834
:101BDC000C00000089460208641400200400000078
:101BEC00D0D903080C000000FD490208581400204D
:101BFC0000000000DCD903080300000039BA020819
:101C0C004014002008000000E8D90308030000007D
:101C1C00A1590208981700200000000064D40308A2
:101C2C0001000000000000000000000000000000A7
:101C3C00000000000D00000000000000000000008B
:101C4C00000000005CD4030800000000000000004D
:101C5C000000000000000000F0D9030804000000A0
:101C6C0071BB0208000000000000000064D40308EF
:101C7C000100000000000000000000000000000057
:101C8C00000000000D00000000000000000000003B
:101C9C00000000003CDA0308000000000000000017
:101CAC00000000000000000068D103080C000000D8
:101CBC0000000000D0140020040000004CDA0308DF
:101CCC000800000000000000C41400200400000004
:101CDC0058DA03080800000000000000B8140020C7
:101CEC000400000060DA0308080000000000000097
:101CFC00AC1400200400000068DA0308080000009F
:101D0C0000000000A01400200400000070DA03089A
:101D1C0008000000000000009414002004000000E3
:101D2C0078DA030808000000000000008814002086
:101D3C000400000080DA0308080000000000000026
:101D4C007C1400200400000064D40308010000008F
:101D5C000000000000000000000000000000000077
:101D6C000D0000000000000000000000000000005A
:101D7C0088DA03080E000000A9B902080000000070
:101D8C0000000000DC14002090DA03080E000000B4
:101D9C0000000000000000000000000054150020AE
:101DAC0098DA03080E00000000000000000000009C
:101DBC0000000000F4150020CC7F0020040000007F
:101DCC009CAE0308F47F0020E0150C170000000007
:101DDC00C97F0020080000004CAE0308CA7F002019
:101DEC0005000000B0AE0308A0DA03080E000000E6
:101DFC00000000000000000000000000441600205D
:101E0C002D202D2D202D2D2D2D202D2D2D000000A4
:101E1C0000000000000000000000000000000000B6
:101E2C0000000101FFFF00001CCF030800000000B0
:101E3C000000000095C00108A0860100040000000D
:101E4C000000000000000000000000000000000086
:101E5C00000000000000000000000000C8F20308B1
:101E6C0080CE030800000000710B01087D0000000B
:101E7C000600000000000000000000000000000050
:101E8C000000000000000000000000000000000046
:101E9C00ECDA03080000000000000000055C0308F9
:101EAC00E803000003000000000000000000000038
:101EBC000000000000000000000000000000000016
:101ECC0000000000F4DA030800000000000000002D
:101EDC00990A03081027000003000000000000000E
:101EEC0000000000000000000000000000000000E6
:101EFC00000000000000000000DB030800000000F0
:101F0C00D1E5020871710108204E000005000000A7
:101F1C0000000000000000000000000000000000B5
:101F2C0000000000000000000000000074D0030856
:101F3C000000000000000000C1560308102700003C
:101F4C000100000000000000000000000000000084
:101F5C000000000000000000000000000000000075
:101F6C0004DB03080000000000000000155D010800
:101F7C00E803000005000000000000000000000065
:101F8C000000000000000000000000000000000045
:101F9C000000000010DB030800000000000000003F
:101FAC004DC30108204E000003000000000000009B
:101FBC000000000000000000000000000000000015
:101FCC00000000000000000020DB030800000000FF
:101FDC000000000055C10108204E00000300000065
:101FEC0000000000000000000000000000000000E5
:101FFC0000000000000000000000000030DB0308BF
:10200C00000000000000000021550308400D0300F3
:10201C0003000000000000000000000000000000B1
:10202C0000000000000000000000000000000000A4
:10203C0038C203080000000000000000C5A701081A
:10204C00102700000100000000000000000000004C
:10205C000000000000000000000000000000000074
:10206C00000000008CCE03080000000000000000FF
:10207C00492C02081027000003000000000000009B
:10208C000000000000000000000000000000000044
:10209C0000000000000000007CC2030800000000EB
:1020AC00000000005D950108A00F00000100000079
:1020BC000000000000000000000000000000000014
:1020CC0000000000000000000000000040DB0308DE
:1020DC000000000000000000E1CA02081027000008
:1020EC0001000000000000000000000000000000E3
:1020FC0000000000000000000000000000000000D4
:10210C00F8CF03080000000000000000594D030840
:10211C00A00F000001000000000000000000000003
:10212C0000000000000000000000000000000000A3
:10213C0000000000D4D003080000000000000000E4
:10214C002D440208102700000100000000000000D0
:10215C000000000000000000000000000000000073
:10216C00000000000000000074CE03080000000016
:10217C00000000006D5C02081A4100000100000024
:10218C000000000000000000000000000000000043
:10219C000000000000000000000000004CDB030801
:1021AC000000000000000000E1940108400D030055
:1021BC000000000000000000000000000000000013
:1021CC000000000000000000000000000000000003
:1021DC0054DB03080000000000000000754E0308EB
:1021EC00A0860100030000000000000000000000B9
:1021FC0000000000000000000000000000000000D3
:10220C000000000001010000E5E1020800000000F0
:10221C0000000000010000000001010101000000AD
:10222C000000803FFF0000000100000043000000A0
:10223C000000000000000000000000000000000092
:10224C00000000000000000000000000430000003F
:10225C000000000000000000000000000000000072
:10226C00000000000000000000000000430000001F
:10227C000000000000000000000000000000000052
:10228C0000000000000000000000000043000000FF
:10229C000000000000000000000000000000000032
:1022AC0000000000000000000000000043000000DF
:1022BC000000000000000000000000000000000012
:1022CC0000000000000000000000000043000000BF
:1022DC0000000000000000000000000000000000F2
:1022EC00000000000000000000000000430000009F
:1022FC0000000000000000000000000000000000D2
:10230C00000000000000000000000000C97103087C
:10231C0009700308000000005AF503084CD40308A8
:10232C00E5C50308E5C50308E5C50308E5C50308CD
:10233C00E5C50308E5C50308E5C50308E5C50308BD
:10234C00E5C50308FFFFFFFFFFFFFFFFFFFFFFFFD8
:10235C00FFFF000001004153434949000000000009
:10236C000000000000000000000000000000000061
:10237C0000000000000041534349490000000000E8
:10238C000000000000000000000000000000000041
:10239C0000000000000000004C1D002000000000A8
:1023AC000000000000000000000000000000000021
:1023BC000000000000000000000000000000000011
:1023CC000000000000000000000000000000000001
:1023DC0000000000000000000000000000000000F1
:1023EC0000000000000000000000000000000000E1
:1023FC0000000000000000000000000001000000D0
:10800000152303701623C370172383713A238370DB
:108010003B2343713C230372704740F2E93300E095
:10802000A3B10289013B12F0020F9BB2F8D089B2D2
:10803000818140F2E93300E043B10289013B12F053
:10804000010F9BB2F8D08089C0B27047094A9042B4
:1080500005D0094B984201D0FF2070470223074A00
:1080600002EB03135A89013292B25A815889C0B285
:10807000704700BF00300140003C0040BC7C002045
:10808000F0B5446814B12568A4886C8341F0800180
:10809000046840F2E93501E0002D54D02689013D05
:1080A00016F0020FADB2F7D089B2A18140F2E931EA
:1080B00001E0002958D02589013915F0010F89B256
:1080C000F7D0A189A1894FF0000C4FF47A714FF6D7
:1080D000FF764FF0FF0E624502D12DE0B1421BD07A
:1080E0002589013915F0020589B2F7D0A4F80CE012
:1080F0004FF47A7102E0B9B2B1420DD0258915F082
:10810000010501F1FF37F6D0A589ADB20BB11D70A5
:1081100001330CF1010CDEE71B4B9C4204D0A3F5AC
:1081200074439C4208D10225184B03EB05156B895B
:1081300001339BB26B816B89436813B11A689B88CA
:1081400013830120F0BD10498C4204D0A1F5744185
:108150008C42B7D102250D4901EB05156989013122
:1081600089B269816989ADE7074DAC4203D00849FE
:108170008C42A7D10221054D05EB01114D89013536
:10818000ADB24D8149899DE700300140BC7C0020A3
:10819000003C004030B4446814B12368A5885D8376
:1081A000036840F2E93001E0002832D01D8901382F
:1081B00015F0020F80B2F7D089B2998140F2E9310F
:1081C00001E0002947D01889013910F0010F89B268
:1081D000F7D0998940F2E93100E059B318890139A3
:1081E00010F0020F89B2F8D092B29A8140F2E932CF
:1081F00001E0002A3FD01989013A11F0010F92B233
:10820000F7D09B8914B12368A2881A83012030BC5F
:10821000704721498B4204D0A1F574418B42D9D1DA
:1082200002201E4901EB00104189013189B24181D0
:108230004189CFE7184A934204D0A2F57442934291
:10824000E0D10221154B03EB01114B8901339BB2A5
:108250004B814B89D6E71048834203D010498B42AB
:10826000B8D102210D4800EB01114889013080B2DC
:1082700048814989AEE708498B4203D0084A9342B6
:10828000C0D10222054B03EB0212538901339BB28A
:1082900053815389B6E700BF00300140BC7C002009
:1082A000003C0040002870B51EDB0928044620DD94
:1082B000012303EB83035B00B0FBF3F2092AF8D838
:1082C0007BB10E4EB4FBF3F00928CCBF572230220D
:1082D000A6FB03E5024403FB1044EB0801F8012B65
:1082E000F0D100230B7070BD2D230B704042013183
:1082F000DBE7303001F8010BF3E700BFCDCCCCCC8D
:10830000884230B44FF001042ED301FB04F4B0FBDB
:10831000F4F58D42F9D284B1AAB901E0B0FBF4F5CD
:10832000092DCCBF572230222A4404FB150003F844
:10833000012BB4FBF1F4002CF0D100221A7030BCF8
:108340007047B0FBF4F5092DCCBF372230222A4408
:1083500004FB150003F8012BB4FBF1F4002CF0D161
:1083600000221A7030BC70470546002AEBD1D7E7CF
:1083700003685A1C0260197070472DE9F047089C89
:108380002578002B804689460CBF4FF0200A4FF01D
:10839000300A661C35B3002A29DD334601E0024667
:1083A00098B113F8011B501E0029F8D1971E60B137
:1083B0003D46013D51464046C8476B1C002BF8DC4A
:1083C000257827EAE770013055B1041B294640465D
:1083D000C847301916F8015B002DF7D1BDE8F087CA
:1083E000BDE8F087002A04DC2846BDE8F0870020BD
:1083F000EBE7571EDCE70A44914251D030B441F21A
:10840000210411F8013B80EA0320430010F4004FDF
:1084100084EA03059BB2ADB208BF1D466B0015F49C
:10842000004F84EA03009BB280B208BF18464300A5
:1084300010F4004F84EA03059BB2ADB208BF1D469D
:108440006B0015F4004F84EA03009BB280B208BFB2
:108450001846430010F4004F84EA03059BB2ADB206
:1084600008BF1D466B0015F4004F84EA03009BB261
:1084700080B208BF1846430010F4004F84EA030599
:108480009BB2ADB208BF1D466B0084EA030015F431
:10849000004F85B298B218BF28468A42B1D130BC8D
:1084A000704783684268D0ED037A00EB83010133A3
:1084B000934281ED040A836004BF0023836000EBD4
:1084C000830393ED047A036870EE277A9A42C0ED35
:1084D000037A77EEC77AC0ED037A0CDA013307EE40
:1084E000103AF8EEC76AB7EE007A87EEA60A036084
:1084F00030EE070A704707EE102AB8EEC77A87EE0B
:10850000870A704790ED097A90ED004AD0ED0A6A2B
:10851000D0ED014AD0ED047A90ED035AD0ED025A25
:10852000A4EE007AB0EE406AB0EE470AB0EE667A8A
:10853000A6EE247A67EEC07AA0EE457AE6EE257ABA
:1085400080ED097AC0ED0A7A7047D0ED057A90ED9A
:10855000013AD0ED003AD0ED064A90ED024A90ED96
:10856000077A90ED035A90ED086AD0ED045AC0EDF9
:10857000067AF0EE406A27EE830AC0ED056AA3EEA4
:10858000A60A80ED087AA4EE240AA5EE470AA5EE15
:10859000C60A80ED070A7047D0ED007A90ED017AA7
:1085A00030EE670AE7EE007AB0EE670AC0ED007AB7
:1085B000704770474FF480530382704750F8043C73
:1085C000012280F83520143803B118477047BFF3F3
:1085D0004F8F0549054BCA6802F4E0621343CB6034
:1085E000BFF34F8F00BFFDE700ED00E00400FA0588
:1085F00070B4037B04681F2B08D9203B20216268DC
:1086000001FA03F31A421CD170BC70472021226882
:1086100001FA03F31A42F7D042691449582000FBCB
:10862000021251685689CD680868296821F0010155
:108630002960828992B222EA06028281A36070BC1C
:10864000704742690949582000FB02125168568957
:10865000CD680868296821F001012960828992B2F9
:1086600022EA06028281E36070BC704794750020A4
:1086700030B4094B1C786CB1084A002502EBC404E5
:10868000116893884D628889083203439BB2A242E5
:108690008B81F5D130BC7047B4790020B8790020C7
:1086A00010B4037B01681F2B09D9203B20224C68A2
:1086B00002FA03F31C4214D15DF8044B70472022E8
:1086C0000C6802FA03F31C42F6D00C4A40680024FE
:1086D000147002685DF8044B22F0010202608B60A6
:1086E0007047064A40680024147002685DF8044B25
:1086F00022F001020260CB60704700BF0B810020B6
:1087000090F8493013B1002280F84920184670478C
:1087100070B5044682B00830256A6B4606223B21BC
:10872000A847A8B19DF804009DF800609DF80110CD
:108730009DF802509DF803209DF8053041EA06217E
:1087400043EA002342EA05226182A282E3820120F9
:1087500002B070BDF8B50468C4F30D0405460E46BA
:1087600004B32F6823F000FC092840F08880454CB2
:10877000236923F440732361236943F40073236165
:10878000236943F0010323613E6023F0EDFB23697D
:10879000092823F00103236171D12B6804332B6076
:1087A0000020F8BD384B394A93422BD902F580425C
:1087B000934226D902F5804293422AD902F580429B
:1087C000934228D902F58032934226D902F500322D
:1087D000934224D902F50032934222D902F50032A5
:1087E000934220D902F5003293421ED902F580222D
:1087F00093421CD9B3F1016F1BD3052007F0B0FBE6
:10880000FBE7082423F0B0FB092814D04FF0FF3019
:10881000F8BD1024F6E71824F4E72024F2E7282412
:10882000F0E73024EEE73824ECE74024EAE7482478
:10883000E8E75824E6E7134F3B6923F440733B61B4
:108840003B6943F400733B613B6923F0F8033B61F0
:108850003B6943F002031C433C613B6943F48033B2
:108860003B6123F081FB3B6923F002033B613B69E1
:10887000092823F0F8033B613FF473AFC6E76FF0BC
:108880000100F8BD003C024000400008FF3F000826
:10889000F8B504460D468E180027B54201D120696F
:1088A000F8BDE368591CE160234415F8012B1A72E6
:1088B0000429F2D1206918B9A1682046FFF74AFFC0
:1088C0002061E760E9E7024B186808F071B800BF63
:1088D000E0B00020F8B5027B466903681F2A2DD955
:1088E000A2F120055F682024AC402742114617D032
:1088F0001022AA40DC60DA605A68EA40D40749D402
:10890000716B756A0A68B46A22F00102A5420A60B6
:1089100037D1012286F84C20027B11461F2A20D92C
:108920002039082258688A40024200D0DA600422C6
:10893000586802FA01F1014221D1F8BD20241D68D6
:108940009440254211460CD0102191409C609960C2
:108950001968D140C907D3D5012101FA02F29A6002
:10896000CEE7082218688A40024200D09A600422AA
:10897000186802FA01F101420BD09960F8BDD96084
:10898000F8BD0446304607F0AFFF227B236811464E
:10899000C4E7F8BD012202FA05F5DD60B0E770B565
:1089A00082B004466946183022F008F9A8B19DF853
:1089B00005009DF801609DF802109DF803509DF898
:1089C00004209DF8063041EA062143EA002342EAEA
:1089D0000522A184E2842385012002B070BD002815
:1089E00055D0026802F13F4303F57E032DE9F04FB5
:1089F0009B0A544DEB5C03F01F055B090124032B1C
:108A000004FA05F444D0042B00F09780022B44D0E4
:108A100001F00306731E012BC1F3810CC1F3001892
:108A20008588C1F341113DD90024234601274FF029
:108A3000030E03E0102B04F1020426D007FA03F022
:108A4000A84303F10103F5D1D2F800C00EFA04F0F7
:108A5000C04300EA0C0CC2F800C0D2F8008006FA4D
:108A600004FC4CEA080CC2F800C0D2F80CC000EAC2
:108A70000C00D060D2F80CC001FA04F040EA0C00FF
:108A8000102BD06004F10204D8D1BDE8F08F7047FC
:108A90002D4B1D6C2C431C64BAE72B4B5D6C2C4397
:108AA0005C64B5E7002003464FF0010E4FF0030968
:108AB00004E00133102B00F102003CD00EFA03F762
:108AC00037EA0504F5D1D2F800A009FA00F4E4432E
:108AD0000AEA040AC2F800A0D2F800B006FA00FAC6
:108AE0004AEA0B0AC2F800A0D2F808A004EA0A0A6F
:108AF000C2F808A0D2F808B00CFA00FA4AEA0B0A49
:108B0000C2F808A0D2F804A02AEA07075760D2F8F2
:108B100004A008FA03F747EA0A075760D7683C4001
:108B2000D460D76801FA00F401333C43102BD460C1
:108B300000F10200C2D1BDE8F08F034B1D6B2C4346
:108B40001C6365E754AC030800380240F0B50446E6
:108B500090F84D0083B0002840F0A480674E37782D
:108B6000002F40D004F11805A06921F063FF94F8AC
:108B700046201A212846FFF70DFB012007F08CFC48
:108B8000A06921F043FF284694F85C10256D6B46E0
:108B90000622A847D0B19DF802609DF803309DF8E9
:108BA00000509DF801109DF804009DF8052043EA4F
:108BB00006231BB2E3845BB241EA052142EA0022AC
:108BC0000133A184228506D003B0F0BDB4F926306C
:108BD0005BB20133F8D194F924300133F4D106208B
:108BE00007F0BEF9F0E7254655F8180F21F022FFEF
:108BF00080226B212846FFF7CDFA962007F0A6FCCD
:108C0000032268212846FFF7C5FA962007F09EFC4C
:108C100003226B212846FFF7BDFA0F2007F03CFC2A
:108C200010226A212846FFF7B5FA0F2007F034FC1E
:108C30003A466C212846FFF7ADFA0F2007F02CFCCE
:108C400094F8482019212846FFF7A4FA0F2007F0CE
:108C500023FC18221B212846FFF79CFA0F2007F05F
:108C60001BFC10221C212846FFF794FA0F2007F066
:108C700013FC102237212846FFF78CFA0F2007F04B
:108C80000BFC012238212846FFF784FA0F2007F059
:108C900003FCA06921F0BAFE012007F0FDFB0123CF
:108CA000337061E706F0F6FE0546D8B120230021B7
:108CB0008371C171FFF793FE2146114B41F8143FB8
:108CC000284621F00FFFAB88B3FA83F3C3F11F03EB
:108CD000012212FA03F33FF441AF0A490A68134331
:108CE0000B603BE70146FFF77AFE2146044B41F853
:108CF000143F284621F0F6FE30E700BFB01D0020EB
:108D0000BD850008003C014010B1036882885A8389
:108D1000704710B1036882881A83704710B5014606
:108D200000BF064C2068FFF7EFFF0548FFF775F915
:108D30002068FFF7EEFF00BF10BD00BF283A0020FB
:108D4000003C004018B10368828809B95A83704713
:108D50001A83704730B1036882881B691A4214BFB6
:108D60000120002070472DE9F0410B4E34687369F3
:108D70001C400FD0DFF824800127B4FA84F3C3F13C
:108D80001F0307FA03F558F8230003689847AC431C
:108D90007561F2D1BDE8F081003C0140747E002095
:108DA0002DE9F0410B4E346873691C400FD0DFF899
:108DB00028800127B4FA84F3C3F11F0307FA03F5EF
:108DC00058F8230003689847AC437561F2D1BDE8B9
:108DD000F08100BF003C0140747E00202DE9F0418D
:108DE0000B4E346873691C400FD0DFF828800127D0
:108DF000B4FA84F3C3F11F0307FA03F558F823000C
:108E000003689847AC437561F2D1BDE8F08100BFBB
:108E1000003C0140747E00202DE9F0410B4E346887
:108E200073691C400FD0DFF828800127B4FA84F35F
:108E3000C3F11F0307FA03F558F8230003689847A6
:108E4000AC437561F2D1BDE8F08100BF003C014048
:108E5000747E00202DE9F0410B4E346873691C408C
:108E60000FD0DFF828800127B4FA84F3C3F11F0381
:108E700007FA03F558F8230003689847AC43756177
:108E8000F2D1BDE8F08100BF003C0140747E0020BB
:108E90002DE9F0410B4E346873691C400FD0DFF8A8
:108EA00028800127B4FA84F3C3F11F0307FA03F5FE
:108EB00058F8230003689847AC437561F2D1BDE8C8
:108EC000F08100BF003C0140747E0020084A094840
:108ED00008B5536C43F4804353640021402230F0C2
:108EE00024FB054B4FF0FF321A60C3F8032008BD86
:108EF00000380240747E0020B47E002003685B6A64
:108F000018472DE9F041044618460D461646984686
:108F10002DF0A4F92768E6722844A07229467D69DD
:108F2000434632462046AC46BDE8F0416047036800
:108F300010B504461B689847236820469B689847ED
:108F4000A37B0133A37310BD10B5036804469B686F
:108F50009847FF2301226373227310BD08B506F002
:108F600099FD38B12C2282710022C2712021BDE806
:108F7000084034E508BD30B4456815B12B68AA88AF
:108F80005A83026841F0800140F2E93301E0002B8E
:108F900043D01089013B10F0020F9BB2F7D089B289
:108FA000918140F2E93301E0002B36D01189013B79
:108FB00011F0010F9BB2F7D09389938940F2E93306
:108FC00000E0D3B11189013B11F0020F9BB2F8D040
:108FD000FF23938140F2E93300E073B11189013B33
:108FE00011F0010F9BB2F8D09489E4B215B12B684F
:108FF000AA881A83204630BC704710498A4203D0A1
:109000000F4B9A42F2D102230E4A02EB03135A8904
:10901000013292B25A815B89E8E708498A4203D05B
:10902000074B9A42C9D10223064901EB0313598920
:10903000013189B259815B89BFE700BF003001402F
:10904000003C0040BC7C0020F8B5654C0601A71927
:109050000546387A21F002FD3B7A03F01F015B09D7
:109060000122032B02FA01F26DD0042B66D0022BF1
:109070005CD0A3190135187906F00CFDEDB2074656
:1090800010B11223C5718371A319587906F002FD3E
:1090900010B11323C5718371A319987906F0FAFCF6
:1090A00010B11423C5718371A5190A21EA793846D4
:1090B00006F024FC687906F0EDFCEA790A2106F056
:1090C0001DFCA87906F0E6FCEA790A2106F016FCF8
:1090D000A359444A934247D0434A934250D0434A0B
:1090E000934259D0424A934262D0424A93426BD053
:1090F000414A93422CD03444227BE2B9012002221F
:10910000198801F4415141F445710A4302431A8020
:109110009A8B22F400621204120C07219A8319829E
:109120001A8892B242F040021A80F8BD334B596A55
:109130000A435A629DE700200246E1E72F4B196976
:109140000A431A6195E72D4B196A0A431A6290E7A0
:1091500002F564424FF40010536A43F40013536263
:1091600022F062FFA359C6E702F584324FF4805023
:10917000536A43F48053536222F056FFA359BAE76F
:1091800002F500324FF48040136A43F480431362C7
:1091900022F052FFA359AEE702F5FE324FF4004031
:1091A000136A43F40043136222F046FFA359A2E777
:1091B00002F582324FF40050536A43F40053536275
:1091C00022F032FFA35996E702F568424FF480106F
:1091D000536A43F48013536222F026FFA3598AE7AF
:1091E000BC7C00200030014000380040003C0040C2
:1091F000003401400050014000540140003802405A
:10920000427A02B9704710B504460368406804F119
:109210000A0198470023637210BD437A5A1C034425
:10922000D2B242729972037A934200D802B970475F
:1092300010B504460368406804F10A01984700230A
:10924000637210BD302827D0312827D0322827D08C
:10925000332827D0342827D0352827D0202827D0D6
:10926000212827D0102827D0112827D0122827D02E
:10927000132827D0142827D0152827D0162805D042
:10928000172808BF0F2202D0002070470E22104B73
:1092900003EB4203587870470022F8E70122F6E713
:1092A0000222F4E70322F2E70422F0E70522EEE7C8
:1092B0000622ECE70722EAE70822E8E70922E6E7C8
:1092C0000A22E4E70B22E2E70C22E0E70D22DEE7C8
:1092D0009496030870B5448806460D46C4F30B0403
:1092E00022460021284630F020F93369094A93428A
:1092F00009D3094A934206D2224628461946BDE8B8
:1093000070402DF093BE23B121462846BDE8704041
:10931000184770BDAC0500085C060008064B0749FD
:109320008B4202D30023184670471A88C2F30B02FF
:109330009042F8D01433F3E788010008AC05000828
:10934000024A136823EA000010607047404600207C
:10935000F8B51A4D2B789F2B2ED16B78BE2B2BD1C5
:1093600005221749A81C30F02BF928BB07222946F3
:109370004FF6FF70FFF73FF8124FEC1D22884AB1FD
:10938000A618BE4218D2052A16D92146FFF733F88F
:109390003446F3E721460222FFF72DF80222A118F6
:1093A000FFF729F80634084B641B1C8041F60F5365
:1093B000C31A58425841F8BD0020F8BD00400008CB
:1093C000E4C0030800800008BC3A00202DE9F04FFB
:1093D000DFF85891504F8DB00326A7EB09071822EC
:1093E0000DEB0200002130F0A0F84C4BCDF81890A6
:1093F00007971A69002A04DA494A5A6002F188324A
:109400005A6001228DF82C20F322DA60454B464C3D
:1094100018689A8804909B79ADF8142004A9072253
:1094200006A88DF81630FFF733FA072204A94FF685
:10943000FF70FEF7E0FFDFF8F8B080464FF0000A5B
:109440005C4539D30CAC002524F82C5D0222214662
:1094500006A8FFF71DFA022221464046FEF7CBFF81
:1094600040BAC043ADF80800022202A906A8FFF7DF
:109470000FFA099878B108ABC0F1040229461844E4
:1094800030F053F80A9818B9089906A8FFF762F95E
:1094900000230A9009939DF82C300A9A23B11F49A2
:1094A0000B6943F000430B61013E2DD0002A96D199
:1094B000FFF74EFF50B32CE065888DF80DA0C5F383
:1094C0000B05AA1DADF808202288C2F30B01120B70
:1094D000ADF80A108DF80C2002A9062206A8FFF7A5
:1094E000D7F9062202A94046FEF785FF616880464B
:1094F0002A4606A8FFF7CCF9616840462A46FEF7DF
:109500007AFF143480469BE7002AD1D0052006F06C
:1095100027FD0DB0BDE8F08F00800008003C024040
:1095200023016745B496030888010008004000083D
:10953000AC0500080378202B024600F10100F9D0A9
:10954000092BF7D02D2B2CD02B2B03BF5378B7EE44
:10955000000A0246B7EE000AA3F13001C8B209289A
:109560009FED467A10D8F2EE046A07EE901AF8EEF4
:10957000E77A12F8013FE7EE267AA3F13001C8B28C
:109580000928B0EE677AF0D92E2B4CD003F0DF0318
:10959000452B0BD0F7EE007A67EE276A20EE260AFD
:1095A00070475378BFEE000A0246D5E710B45178F1
:1095B0002D2959D02B290ABF9178501C901C0024CA
:1095C000A1F13003092B53D8002303EB830301EBF4
:1095D000430310F8011FA1F13002092AA3F130035F
:1095E000F3D9B3F59A7F28BF4FF49A73072B42D96A
:1095F000DFED236A1A46F7EE007A083A072A67EE8B
:10960000A67AFAD803F007032BB1F2EE046A013B05
:1096100067EEA67AFBD124B3C7EE276A5DF8044B48
:1096200020EE260A70475378A3F13001C8B209280A
:1096300002F10102AAD8F2EE046AF0EE665A07EED1
:10964000901AF8EEE77A12F8013F87EEA66AA3F1C6
:109650003001C8B2092866EEA56A37EE067AEED95F
:1096600094E767EE276AD9E7901C91780124A7E771
:10967000F7EE007ACFE7F7EE007AC5E700000000CA
:1096800020BCBE4CB5EEC00ADFED317AF1EE10FA27
:10969000CCBF30EE270A30EE670ADFED2E7A20EEDF
:1096A000270A30B5FDEEC07A87B017EE904A05461E
:1096B00084EAE470002303A9A0EBE4700193009313
:1096C00002931FF0C1FB002CACBF20232D2303A865
:1096D0008DF800302CF0C2FD012803A924D0022807
:1096E0002DD0032805BF3023684668468DF8013029
:1096F0002FF041FF68462CF0B1FD0338C4B222467A
:10970000694628462FF095FF00232B5528462CF05C
:10971000A5FD2E22431C2A540DEB0401E8182FF05E
:1097200047FF284607B030BD302368468DF801302A
:109730008DF802308DF803302FF01DFFDAE730236B
:1097400068468DF801308DF802302FF014FFD1E714
:109750006F12033A00007A442DE9F041064615469F
:109760000846B6FBF2F43CB905FB1464124B1B5DD2
:1097700000F8013BBDE8F081B4FBF2F767B90E4B8E
:1097800005FB174705FB1464DA5D00F8012B1B5D30
:1097900000F8013BBDE8F081B7FBF2F8B8F1000F2B
:1097A00002D04046FFF7D8FF05FB1878024B13F8AC
:1097B000082000F8012BE3E7ECC0030830B402688E
:1097C0001146531C036011F8024B0160D31C517801
:1097D00003609378151D05601B0443EA0123D078CC
:1097E000234343EA006030BC70470368591C1A46A3
:1097F000016012F8021B0260587841EA00207047AD
:1098000038B50446006815462DF010FC22682A443D
:10981000226038BD036810B40A0E5C1C04601A7024
:1098200003680A0C5C1C04601A7003680A0A5C1C5A
:1098300004601A7003685A1C026019705DF8044BCA
:109840007047036810B40A0A5C1C04601A7003684D
:109850005A1C026019705DF8044B704703685A1C6B
:10986000026010B4197003680A0A5C1C04601A7064
:1098700003680A0C5C1C04601A700368090E5A1C09
:10988000026019705DF8044B704703685A1C02604F
:1098900019700368090A5A1C0260197070472DE993
:1098A000F047002488B080460F461E46A14605AD0D
:1098B000531C0393117839B3252933D1931CCDF868
:1098C00010900393507830284ED04FF0000AA0F14A
:1098D0003003DBB2092B42D96C2819D0642800F080
:1098E000938024D825281CD063D9582876D06328A3
:1098F0001BD131784046B847039A531C0393117823
:10990000043601340029D7D1204608B0BDE8F087DD
:10991000039B5A1C03921B78642B7CD02AD8252BDE
:1099200054D1252140460134B847039AC0E7732833
:1099300033D044D975284FD106F1040E30682B4638
:1099400000220A217646FEF7DBFC049A0095534676
:1099500039464046FEF711FD039A0444A8E704AADD
:1099600003A91FF04DFAB7E7D31C039390784FF08B
:10997000010AACE7732B10D05BD9752B3AD0782B4A
:1099800096D1A3F15802B2FA82F2306852092B46FE
:1099900010210436FEF7B4FCD7E73368049A00932D
:1099A000394600234046FEF7E8FC04360444039A97
:1099B0007EE70028B9D1204608B0BDE8F0876E28C0
:1099C000B3D1039A336804361C6071E72AD9582B47
:1099D000D7D0632B8DD06BE77828A6D1A0F15802A1
:1099E000B2FA82F2306852092B461021FEF788FC49
:1099F0000436AAE706F1040E30682B4600220A213D
:109A00007646FEF77DFCA0E7331D306829461E46EA
:109A1000FEF748FC99E7331D306829461E46FEF7DD
:109A200041FC92E7002B7FF443AF204608B0BDE82D
:109A3000F0876E2BC6D03BE70EB400B584B005AB03
:109A4000019053F8042B0649039301A8FFF727FF61
:109A5000019B00221A7004B05DF804EB03B070475C
:109A6000718300080FB430B583B006AB0A490B48C8
:109A700053F8042B096800680193FFF710FF084CA6
:109A80000546206806F080FF0028FAD0284603B07B
:109A9000BDE8304004B07047D8390020DC390020E0
:109AA000E0B00020DFED2B7AB4EEE70AF1EE10FA19
:109AB0004ADDDFED296A9FED297A01E0B0EE670A01
:109AC000B4EEC70AF1EE10FA70EE667AF6DC9FED9E
:109AD000247AF4EEC77AF1EE10FA38D5DFED1E6A7B
:109AE0009FED207A01E0F0EE407AF4EEC77AF1EED5
:109AF00010FA37EEA60AF6D4DFED1B7AB4EEE70AC9
:109B0000F1EE10FA14DDDFED137A37EEC00A60EEE5
:109B1000006A9FED166A9FED167ADFED167AA6EEC3
:109B2000867A20EE266AE6EE877AA6EE270A704746
:109B3000DFED117AB4EEE70AF1EE10FA44BFDFED83
:109B4000087A37EEC00AE2E7F0EE407ABFE7B0EEFF
:109B5000670AD1E7DB0F4940DB0FC940E4CB164170
:109B6000DB0F49C0E4CB16C1DB0FC93F92E741B917
:109B70009730083C15A82ABEDB0FC9BF41404A00F8
:109B800011F0800F82F0D503D2B2DBB208BF1346CA
:109B9000590013F0800F81F0D502C9B2D2B208BFCC
:109BA0000A46510012F0800F81F0D503C9B2DBB232
:109BB00008BF0B46590013F0800F81F0D502C9B2DF
:109BC000D2B208BF0A46510012F0800F81F0D503CF
:109BD000C9B2DBB208BF0B46590013F0800F81F009
:109BE000D502C9B2D2B208BF0A46510012F0800FA6
:109BF00081F0D503C9B2DBB208BF0B465A0082F030
:109C0000D50013F0800FD2B2C0B208BF1046704723
:109C100009B909E0194690FBF1F301FB130308466B
:109C2000002BF7D1084670470146FBE7F0EEC07AFB
:109C3000B0EEE07AB4EEE77AF1EE10FAB4BFB0EE2F
:109C4000676AB0EE476AB5EE406AF1EE10FA46D0A8
:109C5000B4EEE77AF1EE10FA8CBFF0EE675AF0EE50
:109C6000475AC5EE866A9FED1F3A9FED1F6A9FED2A
:109C70001F4A9FED1F5ADFED1F3ADFED1F4ADFED50
:109C80001F5AA6EEC36AE6EEA34AA6EE864AB7EED0
:109C9000006AA6EE845AA6EEA46AE6EE855AC5EEE0
:109CA000866AB4EEE77AF1EE10FA48BFDFED147A77
:109CB000F5EEC00A48BF77EEE66AF1EE10FA48BF4B
:109CC000DFED107AB5EEC00A48BF77EEE66AF1EE36
:109CD00010FA48BFF1EE666AB0EE660A7047DFED33
:109CE000076ADEE739094E3DE3B59E3E88FA163E27
:109CF00045FE7F3F99FB243F69A2163EA7DFA834AB
:109D0000DB0FC93FDB0F4940DFED317A30EE277AB8
:109D1000FDEEC76A16EE903A2033402B02D99FED34
:109D20002D0A7047B4EEE70AF1EE10FA4DDD9FED13
:109D30002A6ADFED2A6A01E0B0EE677AB4EEE67ACD
:109D4000F1EE10FA77EE467AF6DC9FED257AF4EE26
:109D5000C77AF1EE10FA35D5DFED1F6A9FED217A53
:109D600001E0F0EE407AF4EEC77AF1EE10FA37EE49
:109D7000A60AF6D4DFED167AB4EEE70AF1EE10FA91
:109D80001BDCDFED197AB4EEE70AF1EE10FA44BFFE
:109D9000DFED137A37EEC00A60EE006A9FED136ABA
:109DA0009FED137ADFED137AA6EE867A20EE266A0F
:109DB000E6EE877AA6EE270A7047DFED0F7A37EED8
:109DC000C00AE9E7B0EE670AD4E7F0EE477ABCE7ED
:109DD000DB0FC93F00000000DB0FC940E4CB164198
:109DE000DB0F49C0E4CB16C1DB0FC9BF92E741B915
:109DF0009730083C15A82ABEDB0F4940FDEEC07A1B
:109E000017EE903A2033402B51D8DFED2D7AB4EE87
:109E1000E70AF1EE10FA50DDDFED2A6A9FED2A7AAB
:109E200001E0B0EE670AB4EEC70AF1EE10FA70EE88
:109E3000667AF6DC9FED257AF4EEC77AF1EE10FA39
:109E400038D5DFED206A9FED227A01E0F0EE407A0E
:109E5000F4EEC77AF1EE10FA37EEA60AF6D4DFED8B
:109E60001D7AB4EEE70AF1EE10FA1BDCDFED1A7A88
:109E7000B4EEE70AF1EE10FA44BFDFED147A37EEE4
:109E8000C00A60EE006A9FED156A9FED157ADFED5E
:109E9000157AA6EE867A20EE266AE6EE877AA6EE98
:109EA000270A7047DFED067A37EEC00AE9E79FED33
:109EB0000E0A7047B0EE670AD1E7F0EE407AB9E7D4
:109EC000DB0F4940DB0FC940E4CB1641DB0F49C033
:109ED000E4CB16C1DB0FC93FDB0FC9BF92E741B925
:109EE0009730083C15A82ABE0000000010B507EE08
:109EF000901A2DED028BB8EE678ADFED227A28EEFC
:109F0000008A044628EE278AB0EE480A2DF04EFA61
:109F1000F0EE408AB0EE480A2DF0AAF9F7EE007A8A
:109F20009FED197AF0EE675AE8EE875A0023A36195
:109F3000B0EE676AC7EEA56A63612362E361A3625C
:109F40006362A8EEC76ABDEC028B77EEC07AB6EE0C
:109F5000007AF8EE005A27EE877A20EE250A27EEDF
:109F6000267A26EE266A67EEA67A20EE260A84ED89
:109F7000046AC4ED017A84ED007A84ED027A84EDFE
:109F8000030A10BD27D4D236F304353F10B44C0970
:109F9000012250F8243001F01F0102FA01F10B43B5
:109FA00040F824305DF8044B70474B0901F01F0165
:109FB00050F82320012303FA01F1114214BF18467F
:109FC00000207047074A084B10781B78074A8342E5
:109FD00096BFC31AC3F180030020126818441044CE
:109FE000704700BFF856002075560020D08500202D
:109FF000064A074B10781B7883428ABFC3F180035F
:10A00000C01AC018C0F17F00704700BFF85600208A
:10A010007556002010B582B000249F2332208DF8A1
:10A0200004308DF805408DF806408DF8074006F0A5
:10A030008DFA8DF8014000BF334C2068FEF764FEB6
:10A0400001A90422684620F0A5FC2068FEF761FE05
:10A0500000BF9DF802309DF801009DF803102B4AC7
:10A060001B0243EA00430B43934246D01ADD284AC1
:10A0700093423AD02FDD274A93422FD001329342A8
:10A0800022D1254B4FF480721A805A809A88198801
:10A09000224C120202FB01F101209A60D96060702B
:10A0A00002B010BD1E4A934218D001329342E8D04C
:10A0B000A2F51A42033A934206D1174B20214FF4DE
:10A0C000807219805A80E1E7134B00201880588075
:10A0D0009860D860E4E7023A9342F5D10E4B8021B4
:10A0E0004FF4807219805A80D0E70B4B4FF4007107
:10A0F0004FF4807219805A80C8E7074B40214FF413
:10A10000807219805A80C1E7283A00201620C200C8
:10A110001920C2001740EF0070010020B01D002080
:10A1200017BA200030B5124C637883B01BB90120F8
:10A13000637003B030BD052200238DF800208DF838
:10A14000013000BF0B4D2868FEF7DEFD6946022294
:10A1500001A820F01FFC2868FEF7DBFD00BF9DF87A
:10A16000053003F0010383F00100637003B030BDDC
:10A17000B01D0020283A002070B5064C0646256820
:10A1800003E023685B1BB34203D8FFF7CBFF002833
:10A19000F7D070BD407F00202DE9F04F89B0B2F1BB
:10A1A000000801900391029340F39F800B46002228
:10A1B00001EB880153F8040B8B420244FAD1029B55
:10A1C0000592002B00F08980059B002B5ED04B4B45
:10A1D000DDF814B01B685FFA83FA0AEB0B02B2F5E4
:10A1E000807F474AD2688CBFCAF5807ADA469A42A5
:10A1F0005ED9190C1A0A4FF0020406208DF81F30A0
:10A200008DF81E208DF81D108DF81C40FFF7B4FF4F
:10A210000620FEF783FD3B4A0123537000BF3A4BF3
:10A220001868FEF771FD07A90422002020F0B2FB98
:10A230000024039D019E5746A1462968A3000020E3
:10A240000A46013459B1B94224D2316820F0A2FB48
:10A250002A68336813443360BF1AC5F80090A045DC
:10A2600005F1040506F10406E7D1274B1868FEF74F
:10A2700050FD00BF214B214A1B6853441360029AD2
:10A28000ABEB0A0B0AB3BBF1000FA4D1059809B0E0
:10A29000BDE8F08F019C04933A46E15820F07AFB28
:10A2A000049B2A68E1583944D71BE1502F60DCE752
:10A2B00005981649164AA0EB0B0005900598002357
:10A2C0000B70137009B0BDE8F08F059BA3EB0B0377
:10A2D0000593059809B0BDE8F08FFFF723FF00282C
:10A2E0007FF472AF029B0593D0E7029C1CB9FFF785
:10A2F00019FF0594CAE700230593C7E7D08500201E
:10A3000070010020B01D0020283A0020F8560020DF
:10A310007556002070B5104D104E2B7831788B4259
:10A3200084B016D00E4A03921A4402928CBF0C4697
:10A33000CA1A04A98CBFC3F180020024012341F88A
:10A34000102D02A802220194FFF726FF002333708C
:10A350002B7004B070BD00BF75560020F856002069
:10A360007856002070B5194C194D237829789942F8
:10A3700084B027D0174A03921A44029234BF0E4683
:10A38000CA1A04A934BFC3F180020026002341F891
:10A39000102D02A802220196FFF7FEFE2378184432
:10A3A000C0B203062B7848BF80F080008342207043
:10A3B00002D0002004B070BD002301202B70237058
:10A3C00004B070BD012004B070BD00BF7556002000
:10A3D000F85600207856002008B545F20820FFF70F
:10A3E000CBFE0620FEF79AFC064B0122C7205A70CE
:10A3F000FEF794FC04480549054A002303700B70DE
:10A40000136008BDB01D0020F856002075560020CE
:10A41000D08500202DE9F04182B00346060C050AE4
:10A42000032406208DF80730884617468DF805600E
:10A430008DF806508DF80440FFF79EFE98B100BFDE
:10A440000A4C2068FEF760FC01A90422002020F0DD
:10A45000A1FA3A460021404620F09CFA2068FEF717
:10A4600058FC00BF384602B0BDE8F081283A002011
:10A47000F0B5124BDD6885B00DB905B0F0BDED0A41
:10A4800014D0002704AE7C196410E0021022694643
:10A49000FFF7C0FF0F2809DD6B4653F8042B01328C
:10A4A0000AD1B342F9D12546AF42ECDBFFF732FFC8
:10A4B000034BED021D60E0E7671CF5E7700100202B
:10A4C000D08500200C4B984213D0A3F580639842AE
:10A4D0000FD003F5804398420BD003F58063984278
:10A4E00007D003F58063984203D0044B18684008F6
:10A4F0007047024B186870470004014064750020E3
:10A50000F0B5774B774A87B01968914200AF00F0F9
:10A51000DB800023744A3B607B60136843F4803324
:10A52000136003E03B68B3F5A04F09D0136803F450
:10A5300000337B603B6801333B607B68002BF1D0CC
:10A54000694B1B6813F4003318BF01237B607B68E1
:10A55000012B7BD0654D644B654AEA606549586FB5
:10A56000654A0860AA605E6B644C654A654826F0DF
:10A5700080065E635E6F46F080765E67196B0C4303
:10A580001C63596B5963996B9963196C41F05B516A
:10A5900041F47B1141F41F6141F00F011964596CC2
:10A5A00007F118040A4348F2FF715A6444F8101D79
:10A5B000002621460123FB733E737E73BE7321F098
:10A5C000E7FC21464FF6FF734F48BB6021F0E0FCEB
:10A5D0004FF6FF7321464D48BB6021F0D9FC214660
:10A5E0004B4821F0D5FC21464A4821F0D1FC2146B8
:10A5F000494821F0CDFC2146484821F0C9FC2146BC
:10A60000474821F0C5FC2146464821F0C1FC2046C0
:10A6100021F0C8FD444B454C1B68BA684448454985
:10A62000A4FB03439B09A0FB0202013B920CB3F184
:10A63000807F0A6007D2404AF0200721536085F8E6
:10A640002300966011601C37BD46F0BD264B3B4D84
:10A650001A6C3B4842F080521A642C684268816848
:10A6600044F440442C609C689C609C6844F4004422
:10A670009C609C6844F4A0549C600068120642EA06
:10A68000801242F48002490842F00802013942EA8D
:10A6900001425A601A6842F080721A601A68920188
:10A6A000FCD52849104A40F205700860996821F0ED
:10A6B00003019960996841F002019960936803F081
:10A6C0000C03082BFAD145E700221A6062B61E4B34
:10A6D0001B6883F308881D4B1B689847FEE700BF83
:10A6E000FCFF0120EFBEADDE0038024000ED00E0CF
:10A6F0000005FA05707A002000000008FF9167004D
:10A70000335F0700000002400004024000080240DE
:10A71000000C0240001002400014024000180240E9
:10A72000001C02400020024064750020D34D6210DE
:10A7300083DE1B43447F002010E000E000700040F7
:10A7400000000020003C02400000FF1F0400FF1F2B
:10A7500008B5054B1B6803B19847044B044A1A60BF
:10A7600072B6FDF734FF00BF58A10020FCFF0120A6
:10A77000EFBEADDE08B5034B1B6803B1984772B658
:10A78000FDF725FF58A10020084B10B507281B68CE
:10A79000C8BF143818440C46007E05F07BF920B180
:10A7A0002146BDE81040FEF7CDBA10BDE07E002086
:10A7B00038B50D4B07281B68CCBFA0F11404044624
:10A7C00023440546187E05F065F958B10134272267
:10A7D000C47182710121FEF702F928460021BDE80B
:10A7E0003840D1E738BD00BFE07E002070B50F4C87
:10A7F0000F4DC0EBC00004EB8004286B266930438A
:10A80000286382B09209667BA1600025012101A81E
:10A8100063618DF804608DF805208DF806508DF881
:10A82000071020F03DF902B070BD00BFB40F00204A
:10A8300000380240074BC0EBC00030B403EB80008F
:10A84000054C0569236B2B4323630176427630BCAC
:10A85000704700BFB40F0020003802402DE9F04FD0
:10A860005B4C54F8204083B0002C00F0AC80E66DC7
:10A87000002E00F0AA809046564A3569226099461B
:10A8800004F2622204F162036361A2614FF4007377
:10A890007268A1600746E3602361A265A246B5B174
:10A8A0004D4B00205A68954203F11C0376D00130CD
:10A8B0001028F7D100207A1CD2B20C21FFF7BAFF82
:10A8C000A36DB168326922630433A1636365F068E4
:10A8D000E8B1414B00215A68904203F11C035BD060
:10A8E00001311029F7D100257A1CD2B20B2128465C
:10A8F000FFF7A0FF2346F27F38492846FFF776FF8F
:10A90000A36DB168F26862630433E163236594F870
:10A91000610005F0BFF8054694F8600005F0BAF84C
:10A920008346307F00284BD119F0080F38D118F03A
:10A93000020F09D045B10B227B1CAA71EB7128468E
:10A94000727F222104F0DAFF18F0010F15D1A36BFA
:10A950007BB996F82020B17F8DF8063001A89309C5
:10A9600001228DF805308DF804108DF8072020F0B5
:10A9700097F8504603B0BDE8F08FBBF1000FE6D06A
:10A9800001370C238BF807708BF806305846727F1E
:10A99000222104F0B3FFDAE7CDB2A5E7C0B28AE71F
:10A9A0000137FFB215B10B23EF71AB7119F0100F26
:10A9B000284614BF02211221727F04F09FFFC6E7D0
:10A9C00020F04CF8B0E7A246D3E7B246D1E700BF8B
:10A9D000E4390020BC960308B40F0020D588000895
:10A9E0000348D0F8AC3113B100F5D2701847704766
:10A9F000B40F00200348D0F8903113B100F5C470B3
:10AA000018477047B40F00200348D0F8743113B1D1
:10AA100000F5B67018477047B40F00200348D0F80F
:10AA2000583113B100F5A87018477047B40F0020D3
:10AA30000348D0F83C3113B100F59A7018477047BD
:10AA4000B40F00200348D0F8203113B100F58C700A
:10AA500018477047B40F00200348D0F804310BB1F9
:10AA6000FC301847704700BFB40F00200348D0F8EF
:10AA7000E8300BB1E0301847704700BFB40F00203A
:10AA80000348D0F8CC300BB1C4301847704700BF32
:10AA9000B40F00200348D0F8B0300BB1A8301847ED
:10AAA000704700BFB40F00200348D0F894300BB1BA
:10AAB0008C301847704700BFB40F00200248836FE6
:10AAC0000BB1703018477047B40F00200248C36DB7
:10AAD0000BB1543018477047B40F00200248036C84
:10AAE0000BB1383018477047B40F00200248436A52
:10AAF0000BB11C3018477047B40F00200248836820
:10AB000003B11847704700BFB40F00201549164B1A
:10AB100016480A6810B48C681549B2FBF4F203FBBE
:10AB200002F30360D1F88820124B134C42F47002F8
:10AB3000C1F888201A68002042F001021A6098606B
:10AB40001A6822F0847222F480321A605C601A68FB
:10AB50004FF0006422F480221A60D8608C605DF8A7
:10AB6000044B70470000002040420F006475002035
:10AB700000ED00E00038024010300024044B4FF498
:10AB8000F0700A21022283E80700FFF7BFBF00BF71
:10AB9000000000202DE9F04FA34CDFF8C09294F89C
:10ABA0005C312DED028B83468FB0002B40F05A8133
:10ABB00094F8DD31002B39D0D4F8E0319B4AABEB6F
:10ABC0000303934200F2348494F84862002E00F0AC
:10ABD000B780D4F850324BB3D4F8583240F6B7327D
:10ABE000ABEB0303934221D994F85432002B00F0CD
:10ABF00061858F4F013BDBB284F85432002B00F0AB
:10AC00006985D4F8505294F85C2215F8011B94F829
:10AC10005D323868C4F850520A44013384F85C222B
:10AC200084F85D3205F0C4FEC4F858B294F85E3280
:10AC3000D9F8005043B17F4E306828B194F85F32A4
:10AC4000013B012B40F2F38494F8A03353B17A4EC8
:10AC500033683BB1D9F80070D4F8A433FB1A632BE6
:10AC600000F22A8294F8DC33022B00F0D482734D78
:10AC700095F87430032B00F0488794F8F8336BB1E3
:10AC8000D4F8FC3353B105F0BBFBD4F8003444F6E0
:10AC90001F62C31A9342074600F2E88294F87A359D
:10ACA000002B40F08B8194F88B3533B1D4F88C3580
:10ACB00003F5C333A0339B4578D294F8C235BBB1BA
:10ACC0005F4D2E46D4F8C40505F06EFE80B1D4F871
:10ACD000C40505F061FE94F8C83507465A1E63B1F5
:10ACE000D4F8C40584F8C82505F05EFE0028EED12E
:10ACF0000FB0BDEC028BBDE8F08F0322514928460E
:10AD00002EF0F9FB94F8CC3594F8CD2584F8CF7566
:10AD100083F47F4383F0FF039B1ABFB29BB2B7EB70
:10AD2000132FCFD194F8CE25DBB29A42CAD1304648
:10AD30001AF0D0FA94F8C835184484F8C805C1E769
:10AD40003B4F386805F030FEC0B201280FD9022809
:10AD50003A4D40F0CE842B78002B41F0A087D4F8F8
:10AD60004C32ABEB0303B3F57A6F81F09A85D4F8DC
:10AD70005032002B3FF45AAF94F84832002B7FF446
:10AD80002BAF314B1B689B7801211E3B00228B426D
:10AD900084F8481284F85C2241F2D2873868022194
:10ADA00004301AF0C0FB94F8543223E794F890353D
:10ADB000264AC4F88CB502EB8302526C42B3244F8E
:10ADC000244E0EADFB1C45F8203D07F11503002174
:10ADD0000793A523318084F894358021152384F8C6
:10ADE0009635284684F89515904728463188FEF711
:10ADF0004CFD069DED1B152DA8BF15252A4639468D
:10AE000007F118002CF012F994F8903584F8C15528
:10AE1000114A013382FB0312A2EBE37202EB4202FE
:10AE20009B1A84F8903548E7BC1D00203F0D0300B5
:10AE30007055002010550020685500201C0000208F
:10AE4000882300208923002074550020E4960308FD
:10AE50005023002058B1002056555555407F002002
:10AE600000007A44D4F86031D9F80020D31A7C2B42
:10AE70007FF69EAE94F864311FED078AC4F8602116
:10AE8000013384F8643104F5CE77242528461AF07E
:10AE9000C1FBB4F87831F7EC016A07EE103AF8EE2E
:10AEA000E66AB8EEC77A0135C6EE877AEDB267EE8C
:10AEB000887AFDEEE77ACDED007ABDF90060F0B258
:10AEC0001AF07EFBC6F307201AF07AFB272DDDD19E
:10AED00030201AF09FFBD94E00201AF071FB0020A1
:10AEE0001AF06EFB30685E2105F062FD94F8643163
:10AEF00013F0030528D1D4F8602141F288339A4237
:10AF000001F2C98714201AF085FBCD4AB4F9B0319B
:10AF1000DD1782FB0323C5EBA3052DB2E8B21AF0BF
:10AF20004FFBC5F307201AF04BFB1C201AF072FBF5
:10AF300000201AF045FB00201AF042FB5E21306829
:10AF400005F036FD94F8643113F0070501F02E8505
:10AF5000282B7FF42DAE00251720D9F8008084F827
:10AF600064511AF057FB28461AF02AFBB54BB64F2E
:10AF7000A3FB08239B0BA7FB03125209C2EB02128F
:10AF8000A3EB8203D8B21AF01BFB18201AF042FB85
:10AF9000AE4BA3FB08239B09A7FB03125209C2EB8C
:10AFA0000212A3EB8203D8B21AF00AFB28461AF069
:10AFB00007FB30685E2105F0FBFCF9E5A44D2A781B
:10AFC00032B1A449D4F87C0505F0BAFC00232B70FB
:10AFD000D4F8803503F5C333A0339B45FFF463AE4B
:10AFE00094F88935C4F880B5234493F88455E8076C
:10AFF00001F10B86A90701F1CD856A0701F1918561
:10B000002A074DD5944B07930EAA1046A3F12102AF
:10B0100040F8202DA3F1240206460090002003F8FA
:10B02000240C1125022355709370D4F8C8113046B2
:10B03000FEF7F0FB3046D4F8CC11FEF7EBFBB4F88A
:10B04000D6317F4903EBC3039B00053381FB03210A
:10B05000DB17C3EBA10189B23046FEF7F2FBB4F86F
:10B06000D83103EB8303590089B23046FEF7E9FB80
:10B0700094F8C231009D9B0743BFB4F8D01101F58D
:10B080007A7189B24FF47A712846FEF7DAFB069B93
:10B0900094F8C421591C069128461A702BF058F8D0
:10B0A00094F8893594F88A15013393FBF1F201FB8A
:10B0B000123384F88935F6E541201AF0E5F9604D40
:10B0C000B4F9AE31DFF8A08185FB0320DB17C3EBB9
:10B0D000A00080B21AF0BCF9B4F9AC3185FB0320B2
:10B0E000DB17C3EBA00080B21AF0B2F9B4F9B031AB
:10B0F00085FB0320DB17C3EBA00080B21AF0A8F990
:10B1000098F80010306805F053FC94F8A85315F037
:10B11000010200F0B585514B1B689A0668D594F87A
:10B12000C2319B0701F1B583012547201AF0ACF924
:10B13000D4F8C8011AF058F9D4F8CC011AF054F92F
:10B14000474AB4F8D6313068A2FB0323C3F3471A49
:10B15000514605F02DFCB4F8D02198F80030642059
:10B1600000FB02F08AEA030388F800301AF03CF989
:10B1700094F8C431306845EA8305EDB2294605F0FC
:10B1800017FC98F8003030685D40294688F8005078
:10B1900005F00EFC94F8A85355BB4F201AF074F933
:10B1A000D4F8D4031AF020F9D4F8D8031AF01CF913
:10B1B00028461AF019F90121306805F0F9FB94F8D6
:10B1C000C25198F80030306805F00105294683F037
:10B1D000010388F8003005F0EBFB98F80030306888
:10B1E0005D40294688F8005005F0E2FB94F8A8532A
:10B1F0001C4AC4F8A4736B1CDBB2A2FB0312D20876
:10B2000002EB8202A3EB420384F8A83394F8DC3308
:10B21000022B7FF42CAD05F0F3F8D4F8E06340F690
:10B22000B833861B9E4201F24E8294F8EC333A2BDF
:10B2300001F03A85002384F8DC331EE578550020C0
:10B240006766666673B2E74589888888D34D621061
:10B25000A4B1002080B1002080B100205CA10020BA
:10B260001F85EB51CDCCCCCC6C55002094F8063426
:10B27000002B40F0CB846A4B1B6848F6034113F067
:10B28000080F49F607464FF0190208BF0E46580747
:10B2900084F8062403D546F4005646F008069906BD
:10B2A00048BF46F4804694F8B85148BF46F020069F
:10B2B000C6F30908002D41F01B8394F8B931002B27
:10B2C00041F024861D4664204FF0FF3A4FF0000CF9
:10B2D00006960796ADF82650CDF82080ADF828A048
:10B2E0008DF83600ADF824C0ADF82AC0ADF82CC0FA
:10B2F000ADF82EC0ADF830C0ADF832C0ADF834C0F6
:10B300000DF1180EBEE80F00464E35460FC59EE8FB
:10B310000F0007C525F8023B180C0121FE221F2350
:10B32000287084F8531084F84E2084F84F3094F835
:10B33000162484F851C05118C82084F8161484F8D3
:10B340005020311F84F852004FF6FF7501E011F8CC
:10B35000013B6B4083EA0313DBB21A0982EA152230
:10B3600042EA03228E4282EAC305F0D12D49A4F8B5
:10B370004C5001F11F0011F8013B6B4083EA0313AD
:10B38000DBB21A0982EA152282EA032282EAC303A7
:10B390001BB29DB28142A4F84C50ECD183F07C03E7
:10B3A00083EA0313DBB21A0982EA152282EA032236
:10B3B00082EAC3031BB29AB24FEA122C5FFA83FEF1
:10B3C000194EA4F84C2084F874C084F873E004F19A
:10B3D0004E0804F16E0AD8F80000D8F80410D8F826
:10B3E0000820D8F80C3035460FC508F11008D045B4
:10B3F0002E46F0D1D8F8000028600C4D98F80430A3
:10B40000337105F1270684F865E484F866C415F8FD
:10B41000011FD4F8FC0305F0CBFAAE42F7D1F8E3F4
:10B420005CA10020101E0020FC210020FB21002038
:10B43000D94ADA4BD07AD9F80010D4F810221B88F8
:10B44000891A4FF47A7202FB00F2DDB200201B0A67
:10B45000914284F8025284F8F85184F8033284F857
:10B46000F93184F8E60184F8E80181F0F480CC4BEE
:10B47000CC491A689B6894F8C20181FB026581FB84
:10B480000361D217DB17C2EBA502C3EBA1031512B0
:10B490001912F42684F80022012284F8015284F85B
:10B4A0000432302584F8051284F8FE617521782372
:10B4B00084F8FF21860794F8C42184F8065284F8A2
:10B4C000071284F8083284F8322241F1BF80D4F8A0
:10B4D000C851B549D4F8CCC1B448B54BDFF8E8A29F
:10B4E00081FB0567EE1781FB0CE1C6EBA7564FEA1F
:10B4F000EC77C7EBA15100FB065707EB47077F002E
:10B5000000FB01C083FB07E800EB400040004FEA6E
:10B51000A848052A4FEAD5754FEAE77201EB810189
:10B5200083FB00E301EB810106EB860684F82152E0
:10B53000A8EB02054FEAA34E00912A464FEAE071BC
:10B540006DB206EB860605EB8606B4F8D631AEEB97
:10B55000010529464FEADC7C0AFB127203EBC303A8
:10B56000944FDFF868E284F826C24FFA81FC009914
:10B570000AFB15054FEA8303B4F8D0010CEB8101F7
:10B580008EFB03CE87FB028C4FEAE27287FB0587B6
:10B59000C2EB6C12B6B289B24FEAE373B4F844C29C
:10B5A00084F8226200F5FA704FEAE5754FEA112A35
:10B5B000C3EBAE1EC5EB67154FEA162380B24FEA08
:10B5C000222884F828A284F823324FEA252784F819
:10B5D0002712CEF307264FEA102184F8242234BF25
:10B5E0004FF0320A4FF0330A4FEA1C22B4F84632C9
:10B5F00084F8258284F8295284F82A7284F81FE29C
:10B6000084F8206284F82D0284F82E1284F833A284
:10B6100084F82BC284F82C2284F8343294F84862DF
:10B62000C4F8E0B1002E7FF4D4AAFFF789BB624FC3
:10B630004FF0010A4FF0000808E01B2B00F07B825E
:10B640000D2B00F0878187F801A0306805F0ACF978
:10B6500000285BD0306805F09FF983B27E2BD9F8C3
:10B6600000204CD07A78002AEFD194F8601200299B
:10B67000E3D07D2B00F0468294F864E2BEF1000F27
:10B6800004D080F02003DBB284F864224A1CD2B2DA
:10B69000092A635484F8602200F02A82082AD4D848
:10B6A000B4F86222134403EB132303F0FF03A4F85E
:10B6B0006232CAE7C4F8503284F8483219F066FFA3
:10B6C00094F854323D4F013BDBB284F85432002BE6
:10B6D0007FF497AA94F85C1294F85D3238684A1C9B
:10B6E000013384F85C2284F85D3205F061F9FFF7DC
:10B6F0009BBA19F03BFF01232B70FFF738BB84F88E
:10B70000608284F8618287F801809EE794F8653250
:10B710002BB1637884F86502302B01F0398394F8FB
:10B720006122274B274FDFF8A8E0DFF86CC0012625
:10B73000002A3FF489AAD9F80000401B012825D827
:10B7400094F87883B8F1000F40F0068294F890A343
:10B7500003EB4A00008900283CD184F890633868E4
:10B760008106E5D594F8C2018007E1D5B4F8D62169
:10B7700010494FF4F36303FB02F381FB0321DB1752
:10B78000C3EB61114FF4036019F0B3FE002384F89A
:10B790006132FFF759BA00BFF4540020145500205D
:10B7A00018550020676666666BCA5F6B806967FF25
:10B7B00083DE1B431F85EB511C00002070550020C9
:10B7C000E49603085CA1002040420F00D34D6210B4
:10B7D000747A00200AF1010A5FFA8AFAB0F5E06F84
:10B7E00084F890A300F099801AD8B0F5047F00F097
:10B7F000318136D8B0F5887F00F00981B0F5007F3F
:10B8000000F0EF80B0F5807F92D1396849078FD57D
:10B81000002119F06EFE002384F86132FFF714BA9C
:10B82000B0F5026F00F001816CD8B0F5E46F00F064
:10B830008380B0F5006F00F09380B0F5E26F7FF485
:10B8400077AFD4F8A021B4F87811642303FB02F396
:10B8500093FBF1F119F04DFE002384F86132FFF7FC
:10B86000F3B9B0F5826F00F02481B0F5C06F00F03D
:10B870001081B0F5806F7FF45BAF94F891330133A2
:10B88000DBB2032B00F2628142F2107184F8913333
:10B8900001FB03F1B4F89233002B40F055810131E4
:10B8A000D24B1B78DF07B4F8943348BF0431DD076F
:10B8B00048BF0A31980748BF14311A0648BF2831DB
:10B8C000DF0548BF28315D0748BF6431180748BF0E
:10B8D000C8319A0548BF01F5C8719F0648BF01F5F8
:10B8E0007A71DD0648BF01F5FA61580648BF01F5D7
:10B8F0007A614FF4806019F0FCFD002384F8613216
:10B90000FFF7A2B9B0F5046F19D0B0F5116F4DD0A3
:10B91000B0F5036F7FF40CAF21E7D4F89C21B4F8A5
:10B920007811642303FB02F393FBF1F119F0E1FDBD
:10B9300084F86182FFF788B9D4F8A421EFE7B4F95D
:10B94000B01101EB8101490019F0D3FD84F8618247
:10B95000FFF77AB984F860A22370A4F8621274E643
:10B96000386881067FF5E4AE94F8C20180077FF560
:10B97000DFAE1AF0010F40F07887D4F8C8219C4957
:10B9800082EAE273A3EBE27303EB5303A1FB0331FF
:10B99000C908002AB8BF41F080414FF4006019F097
:10B9A000A8FD002384F86132FFF74EB994F8B8017E
:10B9B00000283FF4BDAE8F49087800283FF4B8AEA8
:10B9C0008D4B1B8803EB8303590080464FF41160B5
:10B9D00091FBF8F119F08DFD002384F86132FFF737
:10B9E00033B994F8B90100283FF4A2AE834B8449DF
:10B9F0001B6881FB0321DB17C3EBA1014FF400702F
:10BA000019F077FD002384F86132FFF71DB938681B
:10BA100041077FF58DAE00214FF4887019F069FD64
:10BA2000002384F86132FFF70FB9396889067FF582
:10BA30007FAE94F8C2A11AF0020F3FF479AEB4F8C9
:10BA4000D031642101FB03F119F053FD84F86182C8
:10BA5000FFF7FAB894F8B80100283FF469AE6549D9
:10BA6000087800283FF464AE664B5B7B002B01F046
:10BA70004982614B198891FBF0F101EB810149008A
:10BA80004FF4047019F035FD002384F86132FFF79C
:10BA9000DBB894F8B90100283FF44AAE574B4FF495
:10BAA000C060996819F025FD002384F86132FFF722
:10BAB000CBB83868810640F1F18594F8C22194F83A
:10BAC000C41112F0020F0CBF00234FF47A7312F06E
:10BAD000010F0CBF00224FF4FA62134419444FF4D3
:10BAE000826019F006FD002384F86132FFF7ACB8DC
:10BAF000B4F86222C2F1FF0293427FF4A4AD84F84D
:10BB000065A2A0E584F864A29FE5D4F8F403036875
:10BB10005B69984700283FF4B0A8D4F8F4030368A1
:10BB200001219B6998470222002385F8742084F83C
:10BB3000DC33FFF7A2B8306804F036FF00287FF44A
:10BB400082AD84F861A280E50231A9E6012384F880
:10BB5000913342F210719DE6D4F868322A4E94F87F
:10BB60008E23B34201F0B081511C94F88F03D4F8B6
:10BB70006C7284F88E1302F00F028DF818200DF10C
:10BB80001902F91A002941F3008306A900910DF169
:10BB90001E0502E0002E40F3A0850133C4F8683290
:10BBA00013F8011C02F8011BAA42A7EB030680EA66
:10BBB0000100EFD384F88F0301F0E182531CAB4204
:10BBC000107038BF002203D203F8012BAB42FBD127
:10BBD0000099322019F072FC4FF00008002384F81D
:10BBE000788384F86132FFF72FB800BFCD7F002043
:10BBF0001F85EB5157550020145500201855002083
:10BC000067666666F454002034200020013B84F807
:10BC1000063494F80734002B40F0958094F84815CA
:10BC2000D9F800E00A2284F80724002900F0598599
:10BC30000129B4F854A541F221830229B4F85685AC
:10BC400001F06A810329B4F858C501F04283B4F8C1
:10BC50005A250092042901F037830529B4F85C5570
:10BC600001F02E830629B4F85E0501F0268307292A
:10BC7000B4F8602500F03D85B4F8623500F039BDB8
:10BC8000B4F89433D80513D4D90601F1EF809D069A
:10BC900001F14981580601F16F82190701F17B8298
:10BCA000DD0701F1D78213F0020F0CBF04220C2232
:10BCB000B24994F8AF3391F800A00AF0010A0BB131
:10BCC0004AF0020A5320009219F0DEFBAC4B1B88AD
:10BCD00003EB830303EB8303980080B219F0B8FBF6
:10BCE000002019F0B5FBB4F8D033A6493068C3EB97
:10BCF000C3135B0081FB03211944DD17C5EB6125EC
:10BD0000EDB2294604F054FE98F80030009A3068ED
:10BD100042EA0A0A5D40002188F8005004F048FE1B
:10BD20005146306804F044FE98F8003030688AEAE2
:10BD30000303DBB2194688F8003004F039FE94F8AA
:10BD4000A853FFF729BA013B84F8073494F80A3462
:10BD5000002B40F06E848C4B1B68192284F80A2457
:10BD60009A0640F11A8294F8C2319B0700F1B88517
:10BD7000012604F045FBB4F8D811B4F8D051D4F83A
:10BD8000C831069001EB8101019349004FF47A70AC
:10BD9000ADF83210D4F8CC21B4F8D68194F8C4C1EF
:10BDA00001998DF8346000FB05F04FF0000E06ABF2
:10BDB0004FF6FF75ADF830808DF835C0CDF81CE03A
:10BDC0000A9008910992ADF82C50ADF82E50984683
:10BDD0000093B8E80F006D4EB446ACE80F0098E849
:10BDE0000F00ACE8070094F81624ACF8003084F893
:10BDF00051E0A6F1040A02F1010E1820FE211E23D3
:10BE00004FF0C80CD04684F8502084F816E484F82B
:10BE1000530084F84E1084F84F3084F852C001E08B
:10BE200018F8013B6B4083EA0313DBB21A0982EA7C
:10BE3000152242EA0322464582EAC305F0D1534A5D
:10BE4000A4F84C5002F11E0112F8013B6B4083EA4A
:10BE50000313DBB2180980EA152080EA032080EA88
:10BE6000C3031BB29DB28A42A4F84C50ECD183F0BC
:10BE7000180383EA0313DBB21A0982EA152585EA5F
:10BE8000032282EAC3031BB29AB2DBB24FEA122E3C
:10BE9000019384F87230DFF800C1A4F84C2004F15B
:10BEA0006E0384F873E004F14E060293F368306881
:10BEB0007168B26865460FC5029B10369E42AC465B
:10BEC000F4D13068CCF80000314D9DF8043084F88E
:10BED000643484F865E42E4616F8011FD4F8FC0398
:10BEE00004F066FD2B4BB342F6D104F089FAB4F9A5
:10BEF000B011DFF8A8E0B4F8D06106908EFB010E17
:10BF0000C9174FF47A7000FB06F0D4F8C821D4F8B2
:10BF1000CC31009E0990C1EBAE014FF0000EADF8A0
:10BF20002CE0ADF82EE0ADF830E0ADF832100A901C
:10BF3000079208930FCE04F1540CACE80F0096E87A
:10BF4000070021231C268CE8070084F85330C82200
:10BF50006FF0010384F851E084F84E3084F84F60AC
:10BF600084F8522094F8163484F850305A1C84F81F
:10BF7000162433464FF6FF7E564613E0CD7F002051
:10BF800014550020030820805CA10020101E002012
:10BF9000FB21002021220020FC210020676666662C
:10BFA00016F8013B83EA0E0383EA0313DBB21A0996
:10BFB00082EA1E2242EA0322B04582EAC30EEFD192
:10BFC000D248A4F84CE000F11C0110F8013B83EAD0
:10BFD0000E0383EA0313DBB21A0982EA1E2282EA05
:10BFE000032282EAC3031BB21FFA83FE8842A4F82D
:10BFF0004CE0EAD183F0680383EA0313DBB21A0949
:10C0000082EA1E2282EA032282EAC3031BB29AB2A8
:10C01000DBB2110A019384F87030DFF800C302919B
:10C0200004F16E03A4F84C2084F8711004F14E085A
:10C030000393D8F80C30D8F80000D8F80410D8F8DA
:10C040000820E646AEE80F00039B08F1100898456B
:10C05000F446EED1B8F80030AEF800309DF8043068
:10C0600084F862349DF8083084F86334A84618F8E0
:10C07000011FD4F8FC0304F09BFCA54B4345F6D10B
:10C08000D4F8D433D4F8D82306934FF0000E009B95
:10C09000CDF820E0079293E8070004F1540383E809
:10C0A000070094F8162484F851E0312002F1010EC3
:10C0B000FE210C2384F85020C82284F816E484F86A
:10C0C000530084F84E1084F84F3084F852204FF615
:10C0D000FF7E01E01AF8013B83EA0E0383EA0313B3
:10C0E000DBB21A0982EA1E2242EA0322564582EA9C
:10C0F000C30EEFD18549A4F84CE001F10C0011F812
:10C10000013B83EA0E0383EA0313DBB21A0982EAD6
:10C110001E2282EA032282EAC3031BB21FFA83FEB5
:10C120008142A4F84CE0EAD183F0270383EA0313A9
:10C13000DBB21A0982EA1E2E8EEA032E8EEAC30EA5
:10C14000A2460FFA8EFE1FFA8EF65AF84E0FDFF84F
:10C15000CCC1A4F84C604FEA16285FFA8EFE84F832
:10C1600060E084F86180DAF80410DAF80820DAF880
:10C170000C30BAF810A0ACE80F0004F25346ACF84B
:10C1800000A084F8538484F852E415F8011FD4F811
:10C19000FC0304F00DFCAE42F7D194F80E64002EBF
:10C1A00040F0BE80B4F9AC21B4F9AE319FED596ACC
:10C1B000D9F80010069106EE902AB4F9B021534D3B
:10C1C00084F851605B4207EE102A07EE903AF8EED1
:10C1D000E66AF8EEE77AB8EEC77A67EE867A66EE38
:10C1E000866A27EE067A0022CDED087ACDED076A41
:10C1F0008DED097A0A920B920C920DF1180EBEE8A1
:10C200000F002E460FC69EE8070094F816C486E875
:10C2100007004FF00508FE20C8214FF01E0E1C231A
:10C220000CF1010284F84E0084F8521084F80E8458
:10C2300084F853E084F84F30291F84F850C04FF63B
:10C24000FF7084F8162401E011F8013B434083EAB3
:10C250000313DBB21A0982EA102242EA03228D425A
:10C2600082EAC300F0D1294DA4F84C0005F11C016D
:10C2700015F8013B434083EA0313DBB21A0982EA53
:10C28000102282EA032282EAC3031BB298B28D42D3
:10C29000A4F84C00ECD183F0270383EA0313DBB24C
:10C2A0001A0982EA102282EA032282EAC3031BB23D
:10C2B0009AB24FEA122C5FFA83FEDFF86080A4F88E
:10C2C0004C2084F871C084F870E004F14E0604F14B
:10C2D0006E0930687168B268F36845460FC510365C
:10C2E0004E45A846F5D10C4D3388A8F8003005F12D
:10C2F000240684F862E484F863C415F8011FD4F8B6
:10C30000FC0304F055FBAE42F7D10CE0101E0020F8
:10C310001F22002088C3E43AFB210020FC210020DA
:10C32000731E84F80E3494F80F340193002B40F000
:10C330008481D24B1B6805229D0684F80F2400F1EE
:10C340008382DFEDCF7AB0EE677AB4F95A35B4F96B
:10C35000B011CC4DCC48CDED077AB3F5FA6FA8BF3C
:10C360004FF4FA63B3F57A7FB8BF4FF47A73A3F54D
:10C370007A72642303FB02F385FB032580FB012013
:10C38000DB17CA170026C3EBA51306A9C2EBA00250
:10C390008DED087AADF82A30ADF82820069609967A
:10C3A0000D4600910FCDDFF8E4E22E6894F816C434
:10C3B00084F850C075460FC54A212E60AEF10408BE
:10C3C00000250CF10100FE22142384F85310C8212B
:10C3D00084F85150464684F8160484F84E2084F8B8
:10C3E0004F3084F852104FF6FF7501E016F8013B0C
:10C3F0006B4083EA0313DBB21A0982EA152242EA90
:10C400000322B64582EAC305F0D1A049A4F84C50F6
:10C4100001F1140011F8013B6B4083EA0313DBB216
:10C420001A0982EA152282EA032282EAC3031BB2B6
:10C430009DB28142A4F84C50ECD183F0140383EAFE
:10C440000313DBB21A0982EA152282EA032282EA86
:10C45000C30325461BB21FFA83FC55F84E0FDFF8C5
:10C4600038E2A4F84CC0DBB24FEA1C2A84F869A079
:10C4700084F8683069680293AA68EB68AEE80F0038
:10C48000286969692B8BAEE8030004F23F45AEF8DA
:10C4900000309DF8083084F85BA4A94684F85A342B
:10C4A00004F25B4A19F8011FD4F8FC0304F080FA87
:10C4B000CA45F7D1764A94F878351278013BDBB259
:10C4C00012F0010214BFC0214021172B9BBF7148FD
:10C4D0001B184FF0000E93F82CE0B4F89433980733
:10C4E00006BF0120019041F0100113F4027F019872
:10C4F00018BF022013F0100F18BF062013F0200FF2
:10C500000CBF034610230193002A40F0B28403229B
:10C51000019B069303234FF0000C8DF82030009B05
:10C520008DF81CE08DF81E108DF81F208DF81DC0B1
:10C5300093E80700DFF854E184F853C0AEE8030045
:10C5400094F816148EF8002001F1010A4FF0FE094C
:10C550000923C82084F851C084F8501084F816A428
:10C5600084F84E9084F84F3084F852004FF6FF7EE6
:10C5700001E018F8013B83EA0E0383EA0313DBB200
:10C580001A0982EA1E2242EA0322464582EAC30EC3
:10C59000EFD13E49A4F84CE001F1090011F8013B4C
:10C5A00083EA0E0383EA0313DBB21A0982EA1E222E
:10C5B00082EA032282EAC3031BB21FFA83FE81428E
:10C5C000A4F84CE0EAD183F0320383EA0313DBB230
:10C5D0001A0982EA1E2282EA032282EAC303A646DD
:10C5E0001BB21FFA83FC5EF84E0F2B4EA4F84CC012
:10C5F000DBB24FEA1C2884F85D3084F85E80DEF8F8
:10C600000410DEF8082007C6BEF80C109EF80E20B5
:10C610003180B27004F58A6684F8508484F84F340F
:10C6200015F8011FD4F8FC0304F0C2F9AE42F7D1AB
:10C6300008E0013B84F80A34AFE5019B03F1FF39C0
:10C6400084F80F94C4F80074FEF728BB2D2384F8F7
:10C650003332FEF7E3BF94F81432D9F80020C4F85F
:10C660001022013B012B3EF602AF1022022384F878
:10C67000E62184F8E831FEF7FABE00BF5CA1002095
:10C6800000000000D34D621067666666101E002031
:10C69000CD7F0020E4960308FC210020DEF8000096
:10C6A000000600F1CC839CF80C0000283FF440A861
:10C6B00094F89613032900F2B485DFE811F05F01C6
:10C6C000550146012F01B4F8E43300220133A4F8E8
:10C6D000E43384F8DC23FEF7D0BA84F88F03FFF745
:10C6E0006DBA0A4608460D4600918C4688468A4631
:10C6F0000B46B4F8D013A64ECDF818E0C1EB0121DB
:10C7000086FB016E8E44C917C1EB6E21BDF8006037
:10C71000ADF81E804FF0000EADF820C0ADF82260DD
:10C72000ADF824508DF82CE0ADF81CA0ADF8260033
:10C73000ADF82820ADF82A308DF82D1006AD0FCDBC
:10C74000944E84F851E0B646AEE80F0095E8030039
:10C7500094F816C44EF8040B23250CF10108FE20B2
:10C760001623C822AEF8001084F8535084F850C045
:10C7700084F8168484F84E0084F84F30311F84F812
:10C7800052204FF6FF7501E011F8013B6B4083EA40
:10C790000313DBB21A0982EA152242EA03228E420F
:10C7A00082EAC305F0D17B49A4F84C5001F1160090
:10C7B00011F8013B6B4083EA0313DBB21A0982EAEA
:10C7C000152282EA032282EAC3031BB29DB2814290
:10C7D000A4F84C50ECD183F0F40383EA0313DBB2EA
:10C7E0004FEA131E8EEA152E8EEA032E8EEAC30E32
:10C7F00025460FFA8EFE1FFA8EF855F84E0F664E3C
:10C80000A4F84C805FFA8EFE4FEA182C84F86AE098
:10C8100084F86BC06968AA68EB680FC62869696903
:10C82000AA6904F23F4507C604F25D4684F85DC478
:10C8300084F85CE415F8011FD4F8FC0304F0B8F8A0
:10C84000AE42F7D1FFF782BAB4F8D631DFED536AC2
:10C8500007EE903AB4F8D031F8EEE77A07EE103AE6
:10C8600067EEA67AB8EE477A6FE5D4F8CC214C494A
:10C8700082EAE273A3EBE27303EB5303A1FB033100
:10C88000C908002AACBF41F0004141F04041FFF728
:10C8900084B894F8C431042B8CBF03250225FEF71D
:10C8A00044BC012338682B7004F076F805463868DC
:10C8B00004F072F86D067EF45AAA8A2800F09F846C
:10C8C0008E287EF454AA94F84832002B7EF481A975
:10C8D000344BC4F850322D2384F85432FEF751BA49
:10C8E00094F8C431042B8CBF03260226FFF741BA0B
:10C8F0002D4B94F8B9211B8803EB830303EB8303CF
:10C900009D00ADB2002A40F0B1844FF0FF330FFA22
:10C9100083FA10F081FB40B2FEF7D8BCD4F89C2318
:10C9200053799079D17903F1407303EB002303EB42
:10C930000141002384F896334FF4826018F0D9FD4A
:10C94000002384F86132FEF77FB9D4F89823137A74
:10C95000507992781B0403EB002313444A1C84F89B
:10C96000962303EB0161E7E7D4F89823D379107994
:10C9700052781B0403EB00231344EFE7D4F8982309
:10C980009379D07812781B0403EB00231344E5E776
:10C9900003082080101E0020FC2100200AD7233C21
:10C9A0001F85EB51A01F002014550020022018F015
:10C9B00031FEFF2018F016FC0378FF2B00F0D58322
:10C9C00090F90100C517EDB2C0B218F0F9FD284684
:10C9D00018F0F6FD032018F01DFEFF2018F002FCF1
:10C9E0000378FF2B00F05783B0F90850E8B2C5F385
:10C9F000072518F0E5FD284618F0E2FD94F8B83157
:10CA0000002B40F09382D24B1B68980640F139828C
:10CA100094F8C231990700F16D8300252F4601205B
:10CA200018F0F8FD384618F0CBFD284618F0C8FD80
:10CA3000092018F0EFFD002018F0C2FD002018F0CA
:10CA4000BFFDB4F8DA2194F8C451B2F5967F0AD943
:10CA500094F8643103F00F03072B04D842F20F75EA
:10CA6000954228BF1546BB4F052018F0D3FD3B7AF1
:10CA7000002B00F0BD83A5F1200307EE903A9FED57
:10CA8000B67AF8EEE77AF6EE006A67EE877ABEEEDF
:10CA9000007AF5EEC07AF1EE10FA58BFB0EE667A81
:10CAA00077EE877AFDEEE77ACDED007ABDF900509A
:10CAB000E8B218F085FDC5F3072018F081FD94F861
:10CAC000C221002304930593930700F1BD8294F8DB
:10CAD000DC31012B00F0B882B7F90030DFED9F6A3E
:10CAE00007EE103AB7F9023007EE903AB8EEC77A7F
:10CAF000F8EEE77A27EE267A67EEA67ABDEEC77AD9
:10CB0000FDEEE77A06A88DED067ACDED077A18F0EE
:10CB100093FD5E21306803F04BFF94F86431FEF71B
:10CB200017BA8F4B0793A3F1240600222121A3F10A
:10CB3000210703F8242CB1707270069727F022FEAB
:10CB4000884B8949B4F89423002814BF9946894634
:10CB5000530500F1B481D00700F19882910740F1AC
:10CB60000683DFF828924FF00308424649467F4883
:10CB70002AF05CFA07EB08030EA87D4A013340F85F
:10CB8000203D9B1A002207F80820737029F0E0FA74
:10CB9000FEF736BA724B774907930EAEA3F1210028
:10CBA00046F8200D0A2003F8230C0027082003F87C
:10CBB000220C03F8247C30460988FCF742FE6E4BB9
:10CBC0006E491B6881FB0321DB17C3EBA1013046D3
:10CBD00089B2FCF736FE10F01FFA069BB4F8BA21B2
:10CBE000591C06911F70069B110A5F1C069719704D
:10CBF000069B591C06911A70069B5A1C06921870C7
:10CC0000304629F0A5FAFEF7F8B9B4F9AE319FED38
:10CC10005C8A534A079207EE903AF8EEE77A0EAE36
:10CC200067EE887AA2F12101FDEEE77A46F8201D31
:10CC3000A2F124030020CDED007A02F8240C1E227C
:10CC400008209A70BDF8001058703046FCF7F9FDC6
:10CC5000B4F9AC3107EE903AF8EEE77A304667EE79
:10CC6000887AFDEEE77ACDED007ABDF80010FCF78A
:10CC7000E8FDB4F9B03107EE903AF8EEE77A3046C5
:10CC800067EE887AFDEEE77ACDED007ABDF8001008
:10CC9000FCF7D7FD304629F05BFAFEF7ABB9C4F8D4
:10CCA0004CB22E70FEF763B894F8EA03C0B10138B5
:10CCB000C0B2344D01302844002215F8013B5340E6
:10CCC00083EA0313DBB2120AD90042EA0322A84224
:10CCD00081EA131382EA0302EFD1002A7EF4AAAAA2
:10CCE000244B294D244AD4F8F4031B881168EB61C6
:10CCF0009268036BE962EA640021B4F8E423EE660B
:10CD0000E963EA65002B00F09D825B68816C8B42D1
:10CD10003BBFC2685B1A5B1A9B18002B7DF4A8AF5F
:10CD2000036802219B699847042394F8EB0385F874
:10CD300074301DF005FA032384F8DC33FDF798BF47
:10CD40000221386803F01CFE94F85432FDF752BFFC
:10CD50005CA10020F4540020E4380E3F0050C3478B
:10CD600080B100201CC1030814C103085FB100207A
:10CD70005DB10020145500201855002067666666D6
:10CD800058A08B41A42100201C0000202CC10308C6
:10CD9000A3785E09012E40F0648103F00F0E13F0BA
:10CDA000100300F07B81C64AE3782779A4F8860354
:10CDB000D11887EA0300C4F87C23134684F866621E
:10CDC000C4F88013073A84F88C03A4F8847394F8A9
:10CDD0008C03BC4F0CE012F8011BC4F87C63BA4210
:10CDE00080EA0100197007D2D4F88013D4F87C339C
:10CDF000994203F10106EED1BA4284F88C0300F0A7
:10CE00003982127894F88C339A4200F0C781AE4B85
:10CE1000C4F8683201330122B4F88413C4F86C32C8
:10CE200000204FF6F67384F86602A4F8701284F8B6
:10CE3000782284F87823A4F87232FEF770BC1023AD
:10CE400000250422184606A98DF818308DF81920FF
:10CE50008DF81A508DF81B508DF81C508DF81D5010
:10CE600018F02CFB84F86152FDF7EEBE3422FEF779
:10CE70001FBF94F8AF33002B0CBF04220522FFF72D
:10CE800047BB924B93E8030006AB83E803001846C8
:10CE900018F0D2FB3DE6102018F0BCFB284618F035
:10CEA0008FFB284618F08CFB212018F0B3FB284696
:10CEB00018F086FB284618F083FBFEF723B84FF0E6
:10CEC0000308DFF8289250E6B4F97212D4F86C72B5
:10CED000501C02F00F0242F010020029B8BF42F0CD
:10CEE000200284F88E0394F870028DF81820BA1B83
:10CEF0005040C0B28DF8192084F88F030DF11A024A
:10CF0000FEF73FBE724B1988FEF7B7BD714B642028
:10CF1000B3F900A0FEF7DAB91A4618461D46009389
:10CF20009C46FFF7E6BB2422FEF7C2BE6A4F97F885
:10CF30000080B8F1000F3FF466ADDFF894A1B4F8BB
:10CF4000C051BAF800302D016422ADB202FB038358
:10CF50004FEA4802B3FBF2F345EA0325ADB2C3F34F
:10CF600003231D43062018F055FBE8B218F028FBF8
:10CF7000280A18F025FBB4F8C0315849BAF8005017
:10CF800001339BB293FBF8F208FB12334A7AA4F800
:10CF9000C031012A00F087816E23514A497B03FB8F
:10CFA00005F382FB0302DB17C3EBA203002940F069
:10CFB00075814C4D9FB2A5FB07356D093A201FFACC
:10CFC00085F818F027FB5FFA88F018F0F9FA4FEAB5
:10CFD000182018F0F5FA3B2018F01CFB642303FB23
:10CFE00015739BB24048053380FB0320DB17C3EB6E
:10CFF000A000C0B218F0E4FA002018F0E1FA354FB2
:10D00000394D282018F006FB3B6885FB0325DB170C
:10D01000C3EBA505E8B218F0D3FAC5F3072018F062
:10D02000CFFA042018F0F6FAB4F8BA31002B40F029
:10D030001481BD6885F31005E8B218F0C1FAC5F394
:10D04000072018F0BDFADEE40121D4F8C821D4F895
:10D05000CC3184F8DC1104A80492059318F0ECFAA2
:10D0600057E5194B84F866025E1C4FF6F6710122F3
:10D07000A4F8700284F87802C4F86832C4F86C62CC
:10D08000A4F8721284F87823FEF749BB4FF0040825
:10D09000DFF85C9069E500252846AAE494F866224A
:10D0A000002A3EF43CAB94F88D23013202F00F02CB
:10D0B000724500F0C18084F86632FEF730BB00BFD5
:10D0C000C81D0020C41D002034200020E496030861
:10D0D000145500201855002057550020F454002006
:10D0E000310CC3301F85EB516766666620C10308AB
:10D0F00024C10308112018F08DFAB4F8D621784D18
:10D100004FF4F36707FB02F285FB0235D217C2EB3F
:10D110006535E8B218F054FAC5F3072018F050FA54
:10D12000192018F077FAB4F8D6316E4A07FB03F3EA
:10D1300082FB0301DB17C3EB611382FB0321DA17C8
:10D14000C2EB6112642101FB1233D8B218F038FA35
:10D15000002018F035FA94F8C231B4F8D0519A078B
:10D160007FF55BACEFB22D0A59E428462DE4484622
:10D1700029F074F88046F8E41022FEF799BD009972
:10D18000322018F09BF9FEF729BD06AB00930DF194
:10D190001E05FEF713BD2022FEF78ABD524BD4F8C0
:10D1A0007C23C4F88023002703F55B7203F51B760C
:10D1B000C4F86C2203F5177103F55C703A46C4F8A5
:10D1C0006862C4F87C3384F86672A4F87072A4F8BC
:10D1D000727200F093F8013058D0D4F86832C4F875
:10D1E0006C320123C4F8686284F87833FEF797BA8A
:10D1F000E8B218F0E5F9280A18F0E2F95FE43B4BD1
:10D200001B6898067DF5B3AD94F84832002B7DF489
:10D21000E0AC374BC4F850322D2384F85432FDF77C
:10D22000B0BD4B1CDBB2042B84F896334FEA01618E
:10D230003FF47FABFFF780BBD4F88013D4F87C3386
:10D240002C4AC4E5C269036A9A423CBFC1685218BD
:10D25000D31A62E50822FEF72BBD0FF0DDFE18F0B1
:10D26000AFF9002018F0ACF9FFF7CDBB224B1B68DB
:10D27000FFF74DBB84F88DE3FEF751BA1A46184606
:10D280001D4600939C469846FFF733BAD4F868329F
:10D290000222591CC4F868121A709EE79BB23A78B1
:10D2A00093FBF2F385E6392018F0B4F9E8B218F0F0
:10D2B00087F9280A18F084F9A1E61A46FFF719BA87
:10D2C0001A461846FFF715BA1A4618461D46FFF7C4
:10D2D00010BA1A4618461D460093FFF70ABA00BF57
:10D2E00089B5F8141F85EB51C81D00205CA10020F2
:10D2F000D41F0020BF1D0020185500202DE9F04F3D
:10D30000B0F908502DED048B0D81EDB2382D87B0AA
:10D310000C4600F0CF82804691462ED9802D00F039
:10D32000928079D8522D00F0018140F27082542D04
:10D3300000F032836E2D40F031818A4B0A681B88E1
:10D34000894DFF2BA8BFFF23511C21601370A968D2
:10D3500081F3100189B22046FCF797FA834B2046EF
:10D360001988FCF792FA296801F30F0189B2204667
:10D370000125FCF78AFA2B4647E0042D00F00083D4
:10D3800040F21182202D00F0B58040F24B82242D16
:10D3900000F0D582282D40F001810B68DFF8F08184
:10D3A000734E591C022221601A70236806275A1CEA
:10D3B00022601F7023680A22591C21601A7023689A
:10D3C00001255A1922601D70B8F800102046FCF79C
:10D3D0005CFAB8F802102046FCF757FA23685A198D
:10D3E00022601F7023685022591921601A70236827
:10D3F0000022591921601A7031882046FCF745FA3D
:10D4000071882046FCF741FA2B462846638107B015
:10D41000BDEC048BBDE8F08F822D3ED0C0F0D482ED
:10D42000A02D00F0C582FE2D40F0B880514D05F1D1
:10D43000080635F8021B2046FCF727FAAE42F8D161
:10D4400001252B46E1E7DFF84C814B4F4B4EDFF8CF
:10D4500048A108F10D090A2516E0322D00F0BB8124
:10D46000A5F13C00C0B2132840F2BB810023226822
:10D47000511C216015702268C14502F10101216033
:10D480001370DDD018F8015B0A2DE6D1BAF8003030
:10D49000FF2BA8BFFF23DBB2E9E70B68384A324D08
:10D4A0001178384A581C20601970D1882046FCF742
:10D4B000ECF92C4B22681B88FF2B02F10101A8BF5D
:10D4C000FF2321601370A96881F3100189B22046FF
:10D4D000FCF7DBF9296801F30F0189B22046FCF75C
:10D4E000D4F9294B22681978531C012523602B4657
:10D4F00011708AE70B68234D591C6A7821601A70F5
:10D5000023682A78591C21601A702368AA78591C4C
:10D5100021601A70E9882046FCF7B7F923682A7958
:10D52000591C21601A7022686979DDE70A68174E74
:10D53000531C0321236006F10C07334611700625A6
:10D5400001202268511C216010702268BB4202F148
:10D5500001012160157000F0D3819879DD790633DF
:10D56000EFE700BF14550020185500208C21002043
:10D570002C2C00206054002067666666442C002036
:10D5800057550020701F0020D01F002094C00308B2
:10D5900028B0002079970308742C0020A5F10A0315
:10D5A000E72B00F2EA80DFE813F0CD05E800E800A1
:10D5B000E800E800E800E800E800E800E800E8002B
:10D5C000E800E800E800E800E800E800E800E8001B
:10D5D000E800E800E800E800E8009C05E800E80052
:10D5E000E8008B05E800E800E8008605E80045054E
:10D5F000E8001205E8000605E8000105E8008E04D1
:10D60000E8007B04E800E800E800AF02B602E800AA
:10D61000F704E800E800EE04E800E800E800E800AD
:10D62000E800D004E800E800E800E800B404E800FE
:10D630001E08E8009E020608E800E800E800E8008E
:10D64000E800E800E800C207E8009707E80068077C
:10D65000E8001E07E8000D07E800E800E800E80021
:10D66000AA0677066E06460634060E06F805DF059E
:10D670002304E800E903AA03E800E800E800E80062
:10D680009E03E800E8004004E800E800E8002F04FA
:10D6900062048E035003E800E800E8003F032C0317
:10D6A000E800E800E800E800E800E800E800E8003A
:10D6B000E800E800E800E800E800E800E800E8002A
:10D6C000E800AA06E800E800E800E800E800E80052
:10D6D000E800E800E800E800E800E800E800F402FC
:10D6E000E800E800E800E800E800E800E800E800FA
:10D6F000E800E800E800E800E800E800E800E800EA
:10D70000E800E800E800E800E800E800E800E800D9
:10D71000E800E800E800E800E800E800E800E800C9
:10D72000E800E800E800E800E800E800E800E800B9
:10D73000E800E800E800E800E800E800E800E800A9
:10D74000E800E800E800E800E800E800E800E80099
:10D75000E800E800E800E800E800E800E800E80089
:10D76000E800E800E800E800E800E800E800E80079
:10D77000E800E800E800E802BE02742D00F0A08195
:10D78000772D64D1D8F80030D8F804209A421EBF13
:10D790005A1CC8F800201978B74A08BF0021204653
:10D7A00008F094FB4CE6022D00F0E28000F2CF80FE
:10D7B000012D7FF4F3AE0B680022591C21601A7012
:10D7C00023685A1C22601D7022682421531C236088
:10D7D0002B46117019E63388FF2BA8BFFF23DBB25D
:10D7E00045E617F0FFFC00283FF440AE03780A2B13
:10D7F00000F27781B0F9023087FB0312DB17C3EB2D
:10D80000A2039BB2FF2BA8BFFF23DBB22FE6442D60
:10D810007FF4C4AE002A3FF413AE984B1360012589
:10D820002B46F2E5052D7FF4B9AE0B229449204634
:10D83000FBF7E6FF082293492046FBF7E1FF0125AD
:10D84000072291492046FBF7DBFF2B46DDE5F52D4E
:10D8500001F08E80762D00F0E886472D00F06D8770
:10D86000292DD8F8003001F0668040F23F87392D2D
:10D8700001F04880532D41F03D80591CD8F8042018
:10D88000C8F800101878D21A531E0328DBB20DD83E
:10D89000421ED2B27D4D7E4902EB420205EB4202AE
:10D8A0000870527810B1934201F0AB814FF0FF3510
:10D8B0002B46AAE50A68774B0125511C216015709B
:10D8C0002268052150192060117022680A21501920
:10D8D00020601170226800215019206011702268A8
:10D8E00019785019206011702268597850192060F9
:10D8F000117022689978531923602B46117084E5C2
:10D90000634B21681A78481C20600A70002A3FF493
:10D9100097AD013AD2B202EB420206EB42025278D4
:10D92000002A3FF48DAD0132D5180133226813F877
:10D93000011F501C9D4220601170F7D180E5564BAD
:10D94000196820460125FBF789FF2B465DE50B682A
:10D950000222591C21601A70236801255A1922607D
:10D960001D7022680021531923602B4611704CE56D
:10D9700004224A4920460125FBF742FF2B4644E595
:10D98000474920462A46FBF73BFF00212046FBF78C
:10D990007CFF22680021A7E50B6800215A1C226049
:10D9A000197022680125531923602B4611702CE54C
:10D9B0003C4B08461968FBF751FF3B4B2046196862
:10D9C000FBF74CFF394BBBE7DFF8F090384F09F11C
:10D9D0000E064FF00A081DE0B8F1500F32D0B8F132
:10D9E000320F31D0A8F13C00C0B213282FD9002546
:10D9F000294623685A1C2260204683F80080FBF7E2
:10DA000044FF29462046FBF740FFB1453FF418ADDF
:10DA100019F8018BB8F10A0FDED1264B9D68196801
:10DA200005EB85054FF6FF736D009D42A8BF1D46AF
:10DA30009942A8BF194625EAE57521EAE171ADB220
:10DA400089B2D6E71C4BE9E797E82200E8E717F030
:10DA5000C9FB0028CBD003780A2BC8D8B0F9043012
:10DA6000B0F9061003EB830383F3500521EAE1715B
:10DA7000ADB289B2BDE700BF095D0108715D010863
:10DA8000A0C10308ACC10308B8C1030894C00308CF
:10DA9000708D0020A34400204046002090C1030860
:10DAA00098C10308107AFF1F147AFF1F187AFF1F0E
:10DAB0003C2C0020F02B0020302C0020699703081C
:10DAC000D8F80030D8F804209A421EBF5A1CC8F873
:10DAD00000201978984A08BF0021204608F0F6F97E
:10DAE000AEE4002391E6236800255A1C22601D70D5
:10DAF00023685A1C22601D7023685A1C2260294624
:10DB00001D702046FBF7AAFE002120460125FBF7E9
:10DB1000A5FE2B4679E422680121531823600D46A7
:10DB20000B46117071E4854B03F17005226819787A
:10DB3000501C2060117022685978501C20601170B0
:10DB400022689978501C206011702268D978501C86
:10DB50002060117022681979501C206011702268B1
:10DB60005979501C20601170226899790733501C34
:10DB7000AB4220601170D9D162E4714D2046A98971
:10DB8000FBF783FE698920460125FBF77EFE2B46C5
:10DB90003BE42368DFF8DCC1591C9CF800202160BD
:10DBA0001A709CF80030002B3FF44AAC654E664D6D
:10DBB000664867490023226816F8017F02F1010ECA
:10DBC000C4F800E01770226815F8017F02F1010E19
:10DBD000C4F800E01770226810F8017F02F1010E0E
:10DBE000C4F800E01770226811F8017F02F1010EFD
:10DBF000C4F800E017709CF8002001339342DADB90
:10DC00001EE42268534B501C197820601170226862
:10DC10005978501C2060117022689978501C20603F
:10DC200011702268D9785FE44B4D2046A98AFBF732
:10DC30002CFEE98A2046FBF728FE298B2046012589
:10DC4000FBF723FE2B46FFF7E0BBDFF82CE10027B4
:10DC5000FEB2714600232268501C206016702268B4
:10DC6000501C20601370226811F8010F0133551CFD
:10DC7000062B25601070EED10137062F0EF1060E2F
:10DC8000E6D1364900232268501C206017702268B4
:10DC9000501C20601370226811F8010F0133551CCD
:10DCA0000B2B25601070EED123682D49581C0722DC
:10DCB00020601A7023680022581C20601A702268A5
:10DCC00091F8F01010E42368264A274910781C4A7E
:10DCD0005D1C2560187023689278581C20601A70AB
:10DCE0002268897800E4214952232268501C206070
:10DCF000137011F8013F002BF7D1FFF7A1BB1C48AF
:10DD000000232268056803EB4301561C6D5C266006
:10DD10001570026825680A446E1C527826602A70C5
:10DD2000026825680A4401339278691C0A2B216035
:10DD30002A70E6D1FFF784BB495D01089C3F0020B3
:10DD400038B000207B4100208B410020AB410020F7
:10DD50009B4100206041002068750020EB8000207E
:10DD6000088000201099002050B000203897030848
:10DD70005421002079410020C7800020A04D236855
:10DD80002A68591C127821601A702B6822689978C9
:10DD9000531C2360002311702A6821681A44013340
:10DDA0005279481C032B20600A70F5D123682A6839
:10DDB000591C127A21601A7023682A68591CD2787B
:10DDC00021601A7023682A68591C127921601A7020
:10DDD0002B6820465989FBF758FD23682A68591C8F
:10DDE000527A21601A702B6822685978FFF77CBB41
:10DDF00000212046FBF732FD012500212046FBF7DC
:10DE000044FD2B46FFF701BB7E4D20462988FBF7DA
:10DE10003CFD69882046FBF738FDA988204601258E
:10DE2000FBF733FD2B46FFF7F0BA774D05F160069F
:10DE3000A9882046FBF729FDE9882046FBF725FD48
:10DE400029892046FBF721FD2368AA7A591C216005
:10DE50001A702368EA7A591C21601A7055F80C1B55
:10DE60002046FBF7FBFCB542E2D1FFF7E9BA226896
:10DE7000664B64491878551C2560107022685878E4
:10DE8000551C2560107022689B78501C2060137010
:10DE9000C98820460125FBF7F8FC2B46FFF7B5BAE9
:10DEA0005B4D5C4E05F1300795F902100023F256E8
:10DEB0008A4200F0FD830C33482BF8D10835AF427D
:10DEC000F2D1FFF7BDBA544B03F15A0522685979D4
:10DED000501C2060117022681978501C206011704D
:10DEE00022685978501C2060117022689978501C63
:10DEF000206011702268D978501C2060117022684F
:10DF000019790633501C9D4220601170DED1FFF755
:10DF100097BA2368414D591C2A7821601A702368EA
:10DF20006A78591C21601A7069882046FBF7ADFC9D
:10DF300023682A79591C21601A70E9882046FBF76A
:10DF4000A4FC2268297AFFF7CFBAFCF7EBF8236824
:10DF5000334D002803F101010CBF0222032221608E
:10DF60001A7029882046FBF779FCE9682046FBF700
:10DF700075FCFCF727F8012501462046FBF76EFCEF
:10DF80002B46FFF742BA0822264920460125FBF717
:10DF900037FC2B46FFF739BA2268234B501C99787F
:10DFA0002060117022685978FFF79EBA1D4B2268D5
:10DFB000597DFFF799BA1D4D05F1800655F8041FEC
:10DFC0002046FBF74BFCAE42F8D1FFF739BA184DAB
:10DFD00005F14006B5F880102046FBF756FC236893
:10DFE00095F88220591C21601A70236895F88320C7
:10DFF0000435591CAE4221601A70EBD1FFF720BAEC
:10E0000058210020C0AD0020A83E002030B00020E4
:10E01000DC980020FC790020D83B0020D4AD002003
:10E0200070010020447A00205CB0002004800020B1
:10E0300008800020B94D23682A7A591C21601A7083
:10E04000A98B2046FBF721FC298B2046FBF71DFC02
:10E05000698B2046FBF719FC2368EA7C591C216078
:10E060001A70E98C2046FBF710FC298D2046FBF73F
:10E070000CFC2368AA7F591C21601A70236895F84C
:10E080002020591C21601A70A98C2046FBF7FDFB4B
:10E090002368EA7A591C21601A70E9682046FBF768
:10E0A000DDFB23682A7C591C21601A70226895F8D0
:10E0B0002110FFF719BA9A4B22681978FFF714BAA2
:10E0C000984D20462988FBF7E0FBA9882046FBF7FE
:10E0D000DCFB298920460125FBF7D7FB2B46FFF700
:10E0E00094B9914D914F05F1500600212878904A3E
:10E0F0000B4607E00133242B02F10C0200F0BF8233
:10E1000012F80C1C8842F5D103EB4303226807EB9D
:10E110008303511C93F864302160137023686A787C
:10E12000591C21601A702368AA78591C21601A7042
:10E130002368EA780435591CAE4221601A70D4D1A4
:10E14000FFF77EB97B4828F089F800287FF778A987
:10E15000784B1D18226813F8011B501C9D4220604B
:10E160001170F7D1FFF76CB9734D20462988FBF782
:10E170008CFB69882046FBF788FBB5F904306F49B2
:10E18000DA1781FB0313C2EBA30399B220460125E2
:10E19000FBF77BFB2B46FFF738B9694B2046198804
:10E1A000FBF773FB674B20461988FBF76EFB664B4A
:10E1B00021681A7801254B1C02F0010223602B46CE
:10E1C0000A70FFF722B9614B22681B78604D511C21
:10E1D00003F002032160137023682A78591C216020
:10E1E0001A7069682046FBF739FBA9682046FBF7DF
:10E1F00035FBA9892046FBF748FB698A2046FBF7D7
:10E2000044FBA98A20460125FBF73FFB2B46FFF77D
:10E21000FCB8504E3378002B3FF412A94E4F002526
:10E2200037F8021F2046FBF730FB337801359D425B
:10E23000F6DBFFF705B9494D494EDFF84881DFF8B5
:10E240004891DFED488ADFED489A9FED489A05F145
:10E25000200708E020460435FBF717FBAF4206F124
:10E2600018063FF4EDA8717C0029F3D095ED008AE3
:10E27000B0EE480A29F04EF898F80030002B40F034
:10E28000FF8381B2E6E71022394920460125FBF7DA
:10E29000B7FA2B46FFF7B9B8364E338AB3F5007F8D
:10E2A00006F1340594BF01270427403655F8041BB6
:10E2B00091FBF7F1204689B2FBF7E7FAAE42F5D1C0
:10E2C0002D4D2E4F05F10C06B5EC010AD7ED087A5D
:10E2D00080EE270A29F01EF881B22046FBF7D5FA16
:10E2E000AE42F1D1264D05F10C0655F8041B20462F
:10E2F00089B2FBF7CAFAAE42F7D1FFF7A1B8002303
:10E30000DFF88890DFF888B00393029304930593B5
:10E31000984601214FF6FF7A44E000BF447A00207E
:10E3200034230020083A0020D485002038970308C1
:10E33000A09703089E550020681F00206766666648
:10E3400000200020022000206E4300207E1F0020BD
:10E35000801F0020042300200E2300209885002029
:10E36000E8A50020000040420040744400E08244E0
:10E3700088850020241F00204CA100202499002023
:10E38000F4AD002090750020747A0020889703086F
:10E390005021002008F10108B8F10B0F00F01582A0
:10E3A00019F9011F4E1CF5D04AFA08F3D807F1D528
:10E3B000BBF8003043FA08F3DA07EBD504A8FBF703
:10E3C000E5FDE7E72368AF4AAF49D078AF4A5D1C67
:10E3D0002560187023681278581C20601A70226813
:10E3E000C978FFF781B800212046FBF74EFA0021DB
:10E3F0002046FBF74AFA00212046FBF746FA22683E
:10E40000A34D0023511C2160137022682968501C01
:10E4100091F82F102060117022682968501C91F823
:10E420003A102060117022682968501C91F83B1046
:10E43000206011702268511C216013702268511CE9
:10E44000216013702268511C216013702B682046D4
:10E45000D98FFBF71AFA2B682046998FFBF715FA2C
:10E4600023682A68591C92F8312021601A702B68A1
:10E47000226893F83210FFF737B8864D23686A791F
:10E48000834E591C21601A7033682046198CFBF7A3
:10E49000FCF933682046598CFBF7F7F96989204667
:10E4A000FBF7F3F9A9892046FBF7EFF9336820461B
:10E4B000998CFBF7EAF933682046D98CFBF7E5F92C
:10E4C000E9892046FBF7E1F9298A20460125FBF777
:10E4D000DCF92B46FEF799BF6E4EF378002B00F067
:10E4E000C38223680822591C21601A702368012204
:10E4F000991821601A702368674D591C2A79216088
:10E500001A702368AA78591C21601A70298820463D
:10E51000FBF7BBF9698A2046FBF7B7F92368F27964
:10E52000591C21601A702268E978FEF7DDBF15F0EA
:10E53000FBF9FF28064600F0F08206A9002501F845
:10E54000125D0DF105008DF8055014F0D7FD06A8F9
:10E5500000F8115D14F0C6FD06A800F8105D14F077
:10E56000B5FD06A820F8085D14F0A4FD23685A1C28
:10E5700022601E7023689DF80520591C21601A70C6
:10E5800023689DF80620591C21601A7023689DF8A5
:10E590000720591C21601A7023689DF80820591C17
:10E5A00021601A70BDF8101020460125FBF76DF9A7
:10E5B0002B46FEF72ABF2268384B0125511C2160EB
:10E5C00015702268997850192060117022681978A6
:10E5D00050192060117022685978531923602B4616
:10E5E0001170FEF712BF2E4E3378002B3EF428AF89
:10E5F0002C4F0025B846236817F81520591C2160B8
:10E600001A7098F8011001EB810101EB810101F210
:10E61000EE2189B22046FBF738F9337801359D4267
:10E6200008F10208E7DBFEF70BBFD8F800305A1CF0
:10E63000C8F800201B78002B00F0AA82102B07BF1F
:10E64000194A92E82200002529462268501C2060C1
:10E6500013702046FBF702F929462046FBF7FEF827
:10E66000124B2046D968FBF7F9F820460021FBF74A
:10E670000CF900212046FBF708F9FFF78AB90023BF
:10E680001B7AFFDE38B0002050B0002048B00020D8
:10E69000542100201099002068750020C2550020E8
:10E6A00004230020987C0020C4260020A023002002
:10E6B00023685A1C2260197029882046FBF7E5F868
:10E6C0002368EA78591C21601A7023682A79591C3A
:10E6D00021601A702368AA79591C21601A70236876
:10E6E0006A79591C21601A70FFF7E8BB212D40F0B0
:10E6F00001811A46591CC8F80010CC4D12F8021BB3
:10E700006970C8F800205A782A70DA1CC8F800200E
:10E710009B78AB704046FBF768F8D8F80030E8808B
:10E72000591C1A46C8F8001012F8021B2971C8F8C3
:10E7300000205B786B71FFF7B9B8D8F80430D8F8CF
:10E74000005040465D1BFBF739F8052D064600F2E8
:10E75000DC8180252F464FF0010894E80C009B1ABD
:10E76000103BDFF8FC92AB42B8BF9FB2D9F80C3037
:10E770009B1B9F423146204688BF9FB2FBF76EF835
:10E78000B8F1000F00F0D181D9F80C30D4F8008036
:10E79000F219934200D29F1BFBF7BCFD41463A465B
:10E7A0003046FBF737FE2368A84203442360B8BF16
:10E7B000002102DBFEF744BE236801305A1CA84248
:10E7C00022601970F8D1FEF73BBEDFF898A24FF037
:10E7D00000084FF0080908F10108B8F1240F1BD018
:10E7E000C8F1200209FA02F22AFA08F6A8F1200379
:10E7F000164329FA03F31E4306F0010200231343D4
:10E80000E9D05FFA88F025F0CBFF0028E3D041463D
:10E8100004A8FBF7BBFBDEE7854B1B78DB0700F1A9
:10E82000A7810026834FB04602E00136242E0FD088
:10E8300031463846FBF7B9FB0028F6D0314604A82C
:10E84000FBF7B3FB002840F08E8008F10108ECE7ED
:10E85000794B7A4EB3F850102046FBF716F800219A
:10E860002046FBF712F8764B1A68530103F020019B
:10E87000C2F340030B43C2F3800143EA4103C2F3F6
:10E88000C00143EA8103C2F3401143EAC10102F02F
:10E89000100211432046FAF7F8FF02A9042220468D
:10E8A000FAF7AEFF23683178664A581C2060197069
:10E8B00011886429A8BF64212046FAF7E6FF962D47
:10E8C00000F05B8100212046FAF7DFFF2168B8F1F4
:10E8D000190348BFA8F11203A3F3C4034A1C226022
:10E8E00020460B701A4603A90125FAF789FF2B462B
:10E8F000FEF78BBD2846414607F06AFD054603B288
:10E90000FEF783BD5A1CC8F800201A780A2A7EF444
:10E91000CDAF9A1CC8F800204B4A59781170D91C09
:10E92000C8F8001099785170191DC8F80010DB78EC
:10E930009370FEF7BBBF5A1CC8F800201B780A2B47
:10E9400000F01181502B7EF4B1AF4046FAF74DFF35
:10E950003E4E30804046FAF748FF4FF0FF3570805A
:10E960002B46FEF752BD414602A8FBF70FFB6CE7B2
:10E97000D8F80030D8F804209A4240F014812D4B8A
:10E98000FF221A724FF00008314D0DF04FFF414643
:10E990003022304885F800802AF0C7FD8DF81080BD
:10E9A0009DF810300B2B00F24D812B4F294E424623
:10E9B0009DF8103003EB430307EBC3035B7CE3B12B
:10E9C0009DF8103003EB430307EBC3035B69A3B16E
:10E9D0009DF8103003EB430307EBC3032021586974
:10E9E00046F82200F9F7FBFF2B7856F82300FAF7D8
:10E9F00090F92A780132D2B22A709DF81030013392
:10EA0000DBB28DF810309DF810300B2BD0D9236875
:10EA1000591C21601A70B9F1000F3EF411AD0F4B73
:10EA2000C9F8003001252B46FEF7EFBC701F00200F
:10EA3000CD7F0020A0230020D8170020995500206A
:10EA40005CA10020BE3A0020A34400202C2C002012
:10EA5000433D0020C47B0020E8A50020DD02020821
:10EA60007001002090E33FF42368B1787D4A581C80
:10EA70002060197023681278591C21601A703AE5D9
:10EA8000D9F8003013F48053B4EEE88A00F08480A3
:10EA9000F1EE10FAC0F2B280B4EEC98AF1EE10FACB
:10EAA0000DD8DFED717A9FED717A77EEC87AB4EE0A
:10EAB000C78AF1EE10FAB0EE678A00F29F80F7EE97
:10EAC000007A78EE677AB6EE007AF0EE696AE7EEE1
:10EAD000876A40F2E932FDEEE67A17EE901AB1F558
:10EAE000FA6FA8BF4FF4FA619142B8BF114689B2DC
:10EAF000002B3FF4AFABB5EE408AF1EE10FA40F2D6
:10EB0000DC5308BF1946FFF7A5BB4046FAF76DFE78
:10EB10004FF00008074605461FE6226801255319F5
:10EB200023602B461070FEF770BC39462046FAF77A
:10EB3000ACFE23685A1C226083F80080D9F80C5080
:10EB4000D4F80080F219AA427ED8FBF7E3FB3A46DC
:10EB500041463046FBF75EFC2368012503442360F1
:10EB60002B46FEF752BC4046FAF73FFE404EF0E619
:10EB7000049B43F00103049353E623680322591CCA
:10EB800021601A7023687278591C21601A709DE602
:10EB9000384A92E8220058E5F1EE10FA8FDA4FF485
:10EBA0007A71FFF757BB5A1C1946C8F80020324843
:10EBB00011F8022B0272C8F800105B784372042A25
:10EBC00003D9FF2A7EF4E5AEDCE62C4909789942A8
:10EBD00005D8022A7EF4DDAEFF2B7EF4DAAE236880
:10EBE00001255A1922601D70B9F1000F3EF428ACBE
:10EBF000234BC9F800302B46FEF707BC4FF47A715F
:10EC000079E70022C1F80620C1F802208A726BB1B0
:10EC10000133D8F800000B444A1C0130C8F800004A
:10EC200010F8011C02F8011F9342F6D1154B1B7816
:10EC3000002B3EF43BAE4FF0FF3521F083F82B461E
:10EC4000FEF7E3BB4246E2E6AD1BFBF763FB2A4659
:10EC500041463046FBF7DEFB236803442360FEF7A2
:10EC6000EFBB00BF2CB0002000C0884400C082442D
:10EC700028B0002090210020A02300204D54002027
:10EC80007D5D0108243A00200B4B002210B4027273
:10EC900003F58474032102E0072A09DC99798907C6
:10ECA00002D51979815401329C4203F11803F3D142
:10ECB0005DF8044B704700BFBCAC03082E23037003
:10ECC000704700BF0123322131224170427103702D
:10ECD000037170472DE9F0410B78047BDB43DEB212
:10ECE00000F1100200F1380342F8044F9342FBD1C7
:10ECF000DFF89CC000F16001002243F8042F8B4232
:10ED0000FBD14FF0140E0521002546FA01F303F064
:10ED10000103002B1D4414BF4FF019084FF00A08DF
:10ED200011F0010FEDB214BF2746002700220EEBB1
:10ED300002039BB200EB8303013242455F61F6D1CF
:10ED4000013A92B2013201390EEB02034A1C9BB226
:10ED500001D09E46D9E715F0010F14BF19250A25E9
:10ED600000215A1892B200EB82020131A94254618B
:10ED7000F7D10B449BB21A1D00EB82020133002134
:10ED80009BB25160ACF800300361BDE8F08100BF78
:10ED9000B0230020254B5B880B332DE9F04F8A46CA
:10EDA00001F1060B1FFA83F94FF00108002100273B
:10EDB0001AF801EB3E464C460122A4F10B039BB22C
:10EDC00007E001339BB2B0F80CC0C5F814C09C42F8
:10EDD0000AD000EB8305002AF3D100EB8305013351
:10EDE0009BB29C426A61F4D1231D00EB8303013680
:10EDF000092FF6B259600CD0092E14D008FA07F387
:10EE000013EA0E0F14BF012200220C34A4B2013702
:10EE1000D3E709F17809DA451FFA89F9C7D1034B1D
:10EE20005980BDE8F08F0022EFE700BFB02300203B
:10EE30002DE9F047DFF85C80B8F8043004338A46E7
:10EE40001FFA83FC01F109094FF0010E1AF8017B4A
:10EE500064460026231F0EFA06F29BB23A40BAB16E
:10EE6000818900EB830501339BB29C426961F6D135
:10EE700001360434082EA4B2ECD10CF1200CCA45A2
:10EE80001FFA8CFCE2D10023A8F80430BDE8F0871B
:10EE90001146E6E7B023002010B4037B01681F2B66
:10EEA00009D9203B20224C6802FA03F31C4214D1FA
:10EEB0005DF8044B704720220C6802FA03F31C42F1
:10EEC000F6D00C4A40680024147002685DF8044BC8
:10EED00022F0010202608B607047064A40680024FD
:10EEE000147002685DF8044B22F001020260CB60EE
:10EEF000704700BF6C8D0020436A8269F0B4D15422
:10EF0000436A0469426B0133A34228BF0023436272
:10EF1000FAB1116811F0010101D0F0BC7047856AA7
:10EF20001768866927F001072E449D421760D66056
:10EF30000BD3641B546081621368002143F001030A
:10EF400080F84C10F0BC136070475D1B5560836205
:10EF5000F2E7826DD36843F08003D360DDE700BF42
:10EF6000026B10B462B1836CC2684469D11A013B70
:10EF7000615C5DF8044B08BF13468364C8B27047F8
:10EF8000016A4369C4685B5C0131A14228BF114634
:10EF900001625DF8044BD8B2704700BF436B13B1F8
:10EFA00090F84C007047836A406A181AB0FA80F0F3
:10EFB00040097047416A836A99420AD3CB1A416B70
:10EFC000026961B14968501E0B4483420AD2C01ADB
:10EFD000704702691144CB1A416B0029F2D1501ECF
:10EFE000C01A704700207047036B43B1826C5B68A6
:10EFF00093422FBF981AC0689B1AC0187047C26905
:10F00000036A9A422FBFD01AC0688018C01A70478E
:10F010000A4B30B503F1140493F900205D78072AF8
:10F02000C8BF143A811804330D7313F8025C855479
:10F0300013F8012C0A76A342EED130BD449903089F
:10F0400003682DE9F041DF691FB13B46BDE8F0419F
:10F050001847002A164611DD04460D460E4400E00E
:10F0600023689B68204698470028F9D0236815F844
:10F07000011B1B6820469847AE42F1D1BDE8F081E4
:10F0800000232522027043708370C370704700BF55
:10F09000038A2DE9F0478589ADB21D4029D00F467E
:10F0A00006464FF000484FF00009B5FA85F328FAFC
:10F0B00003F2D24391B21B3B15403182042B16D888
:10F0C000DFE803F03129211903007B6A002B32D0DD
:10F0D00003F1FF3A1FFA8AFAC7F824903C6A34B168
:10F0E00023682046514698476468002CF8D1002DCB
:10F0F000DBD1BDE8F0873868716B036889B2984747
:10F10000002DD2D1F5E77868B16B036889B29847D2
:10F11000002DCAD1EDE7B868F16B036889B2984752
:10F12000002DC2D1E5E7F868316C036889B29847D1
:10F13000002DBAD1DDE7F36A1FFA83FACEE700BFEC
:10F1400030B50446806D61718389A26823F4005351
:10F150001B041B0C838185B0A379009213F0040279
:10F1600030D04FF4805213F00203ADF8042056D192
:10F17000ADF806304FF480630022ADF8083011F08E
:10F180000103ADF80C2028D1ADF80A3008238D0713
:10F19000694648BFADF80A301DF052F8A279A36D58
:10F1A000D10724D412F0080F9A8A1BD122F008024A
:10F1B0001204120C9A829A8992B242F400529A81F5
:10F1C00005B030BD13F00203ADF8042024D04FF495
:10F1D00000551346ADF80650CEE70423ADF80A30CB
:10F1E0000C23D4E792B242F008029A82E3E70D4979
:10F1F0008B420FD0A1F548418B4209D00A498B427E
:10F20000D0D105200121FBF7BFFAA279A36DC9E790
:10F210000220F7E70020F5E7ADF80630ACE74FF441
:10F220000053A5E7001001400014014010B504464A
:10F23000806DA160838923F400531B041B0C838120
:10F24000A37984B013F00402009135D04FF48052BA
:10F2500013F00203ADF8042056D1ADF806304FF498
:10F2600080636279ADF80830D1074FF00003ADF844
:10F270000A30ADF80C3045BF0423ADF80A3008233E
:10F280000C236946920748BFADF80A301CF0D8FF3E
:10F29000A279A36DD1071FD412F0080F9A8A16D154
:10F2A00022F008021204120C9A829A8992B242F455
:10F2B00000529A8104B010BD13F00203ADF804208F
:10F2C0001FD04FF400511346ADF80610C9E792B2B3
:10F2D00042F008029A82E8E70D498B420FD0A1F56F
:10F2E00048418B4209D00B498B42D5D105200121E1
:10F2F000FBF74AFAA279A36DCEE70220F7E70020D8
:10F30000F5E7ADF80630ACE74FF40053A5E700BFD2
:10F31000001001400014014038B5384B5A899989D2
:10F32000914224BF00225A81198ADA89914224BF6E
:10F330000022DA81DA788AB1072A0FD0304C3148BE
:10F34000A27801210025062A01709970DD714CD93F
:10F350002379DFED2D6A002B36D138BDDA799B7821
:10F36000284807EE103A002A44D0DFED276A0178DA
:10F37000234CB8EEC77A07EE901AA278F8EEE77A37
:10F3800027EE267A062A67EE877A2BD81F4B03EBE7
:10F390008203D3ED056AF4EEE76AF1EE10FA10DDB0
:10F3A000C6EE877AFDEEE77A17EE903A102BA8BFEB
:10F3B0001023012BB8BF0123DBB28B4228BF0B46C1
:10F3C00003702379002BC8D0013A032AC5D8B7EEC1
:10F3D000000A80EE260A27F09DFF2388984238BF56
:10F3E000208038BDDFED086AD5E7DFED097AB0EEA1
:10F3F000677ACBE7DFED076AB9E700BF1099002015
:10F40000687500202CB000206F120338449903085F
:10F410006F12833A6F12033938B50D4C0D4DAC4263
:10F4200006D2616820461434F9F754FFAC42F8D391
:10F43000094B0A4C0A4818600025257011F002FF9C
:10F44000084B094A65701A60BDE8384012F0DABE10
:10F4500088010008AC0500085421002099550020BF
:10F46000B444002058210020B0450020F0B50C29FC
:10F4700034D8DFE801F0893333335E333333343348
:10F4800033330700048C9689B2F802E01788734D75
:10F4900024F480542404240C0484038C8488818BF9
:10F4A00023F4005321F4E6411B0409041B0C46EA33
:10F4B0000E06090C43EA063341EA0721A8429BB233
:10F4C000A4B289B200F09E8005F58065A84200F0E4
:10F4D000998092688480818302640384F0BD048CE7
:10F4E0009589B2F802C0B2F800E05C4F24F4807451
:10F4F0002404240C0484038C8688818B23F40073F9
:10F500001B0421F073011B0C45EA0C04090443EAB7
:10F510000423090CB8429BB2B6B241EA0E015CD09A
:10F520004F4CA04259D0926886808183C263038485
:10F53000F0BD048C9589B2F802C0B2F800E0474EE5
:10F5400024F010042404240C0484038C8788018B89
:10F5500023F0200321F4E6411B0409041B0C45EAB7
:10F560000C04090C43EA041341EA0E21B0429BB299
:10F57000BFB289B25DD03A4CA0425AD0926887801F
:10F58000018382630384F0BD048C9789B2F802E0A2
:10F590001688324D24F001042404240C0484038CC6
:10F5A0008488018B23F002031B0421F073011B0CE0
:10F5B00047EA0E0709043B43090CA8429BB2A4B2D8
:10F5C00041EA060125D005F58065A84221D0926860
:10F5D0008480018342630384F0BDD589148A578AED
:10F5E00023F4006343EA05254FF6FF332B4095884B
:10F5F00026F440563C4343EA052346EA04169BB2F0
:10F60000B6B290E7158A24F4804444EA8514A4B283
:10F610005FE7D689158A578A23F00803334324F419
:10F62000407496883D4323F004032C433343A4B233
:10F63000CDE7D489158A568A23F0800343EA041360
:10F640004FF6BF741C40938827F44067354344EA63
:10F65000031347EA85079BB2BFB28FE70000014062
:10F66000000401402DE9F84FC82200219348944C32
:10F67000DFF87492934D944E944FDFF8708229F026
:10F6800054FF93489349DFF868E2DFF868C200222C
:10F690001359834200F0F980B3F1804F00F0F780F6
:10F6A000AB4200F0F680B34200F0F580BB4200F0C0
:10F6B000F480734500F0F380634500F0F280434529
:10F6C00000F0F180DFF830A2534500F0EE800AF53B
:10F6D000806A534500F0EB800AF5806A534500F0DC
:10F6E000E880AAF5983A534500F0E5800AF5806A6B
:10F6F000534500F09C800AF5806A534508BF0D23EE
:10F7000000F096801832B2F5907FC1D1DFF8B08159
:10F71000714E08F590774FF0030A4FF0020998F800
:10F7200004301C09013C032C03F00F0378D86B4A0A
:10F7300032F8140040FA03F2D20771D5012505FA18
:10F7400003F3013B184027F033FA654B1B5D184467
:10F7500016EBC00264D056F83030624C98F80810AE
:10F7600003F13F4000F57E00800A205C00F01F049A
:10F770004009032805FA04F500F08180042878D0B8
:10F78000022804D15348406C054352484564B2F8FE
:10F7900004E0BEFA8EF2C2F11F0292B2D00803EB6F
:10F7A000800002F00702046A92000F25954024EAC7
:10F7B00005040462046A01FA02F22243002502628F
:10F7C0004FF0010C2A4603E0102A05F1020527D06C
:10F7D0000CFA02F030EA0E0102F10102F4D11C68C9
:10F7E0000AFA05F1C9430C401C60D3F800B009FACD
:10F7F00005F444EA0B041C609C680C409C609C6807
:10F800009C605C6824EA0000586058685860D868BA
:10F810000140D960D968D960102A05F10205D7D115
:10F8200008F1180847457FF47AAFBDE8F88F0C233C
:10F8300009EBC3034FF0010A93F8343003F01F0BB8
:10F840005B09032B0AFA0BFA09D0042B0CD0022B0C
:10F850007FF458AF4B6C4AEA03034B6452E70B6CDE
:10F860004AEA03030B644DE70B6B4AEA03030B639D
:10F8700048E71848006B05431648056387E71548B5
:10F88000006C05431348056481E70023D0E701239A
:10F89000CEE70223CCE70323CAE70423C8E7052306
:10F8A000C6E70623C4E70723C2E70823C0E7092306
:10F8B000BEE70A23BCE70B23BAE700BFB0860020EF
:10F8C000BCAC03080004004000080040000C0040ED
:10F8D0000000014000380240EC7C0020E0AD03084D
:10F8E000DCAD030854AC030844990308000401404C
:10F8F00000100040001400400040014000286AD081
:10F9000003682DE9F04F03F13F4404F57E045F4E98
:10F91000A40A0125345D04F01F066409032C05FACE
:10F9200006F559D0042C00F0AC80022C59D0858803
:10F93000B5FA85F0C0F11F0080B2C40803EB84045F
:10F9400000F00700266A80000F27874026EA070696
:10F950002662276A01F003068240701E3A4301289E
:10F96000C1F3810CC1F300182262C1F341113DD9EA
:10F970000024224601274FF0030E03E0102A04F171
:10F98000020426D007FA02F0A84302F10102F5D1E1
:10F99000D3F800C00EFA04F0C04300EA0C0CC3F820
:10F9A00000C0D3F8008006FA04FC4CEA080CC3F847
:10F9B00000C0D3F80CC000EA0C00D860D3F80CC02B
:10F9C00001FA04F040EA0C00102AD86004F10204A5
:10F9D000D8D1BDE8F08F70472D4C266C3543256497
:10F9E000A5E72B4C666C35436564A0E70020024612
:10F9F0004FF0010E4FF0030904E00132102A00F12C
:10FA000002003CD00EFA02F737EA0504F5D1D3F82C
:10FA100000A009FA00F4E4430AEA040AC3F800A0CB
:10FA2000D3F800B006FA00FA4AEA0B0AC3F800A0BD
:10FA3000D3F808A004EA0A0AC3F808A0D3F808B06B
:10FA40000CFA00FA4AEA0B0AC3F808A0D3F804A09B
:10FA50002AEA07075F60D3F804A008FA02F747EA2A
:10FA60000A075F60DF683C40DC60DF6801FA00F491
:10FA700001323C43102ADC6000F10200C2D1BDE833
:10FA8000F08F034C266B3543256350E754AC0308D5
:10FA90000038024010B50409013C032C17D80D4B67
:10FAA00033F8142000F00F0042FA00F313F00103C2
:10FAB0000DD0012303FA00F00138104027F078F848
:10FAC000054A064B125D104403EBC00010BD002038
:10FAD00010BD00BFE0AD0308DCAD0308EC7C0020E6
:10FAE00001490248FFF7D4BA5087002000180040AF
:10FAF00001490248FFF7CCBA2887002000040140E2
:10FB000001490248FFF7C4BA2887002000040140D9
:10FB100001490248FFF7BCBA00870020000C0040F2
:10FB200001490248FFF7B4BAD8860020000400401B
:10FB300002494FF08040FFF7ABBA00BFB08600200B
:10FB4000F0B50468474DA30AAB426ED009D8B3F5AF
:10FB5000801F66D0023DAB4258D14FF0480E0126BF
:10FB600008E0414DAB4264D03B35AB424FD14FF042
:10FB7000980E03264779B0004FEA970C00295CD015
:10FB800063460227A5899F4083190CEB43032F434B
:10FB900003F1040C354DBFB245F8231045F82C2075
:10FBA000A781EFF31181502282F31288821905EBAD
:10FBB000C202136963B313620433821905EBC202F4
:10FBC000576917B11F6053690433821905EBC202EC
:10FBD000976917B11F6093690433821905EBC2025C
:10FBE000D76917B11F60D36904330027CAB21F60F9
:10FBF00082F31188304405EBC000036A5BB9A38926
:10FC000023F001031B041B0CA381F0BDF0BDF0BD6C
:10FC100005EB0E03D1E7A3899BB243F00103A38157
:10FC2000F0BD4FF0200E0026A4E74FF0700E022624
:10FC3000A0E74FF0C00E04269CE70223BF0803FA9A
:10FC400007F7A389094D9BB223EA070387190CEB39
:10FC5000470CA3810CF1040345F82C1045F8232030
:10FC60009FE700BF0300100006001000B0860020D0
:10FC700010B5036883480139834282B089B200F02D
:10FC8000CB80A0F58060834200F0C68000F5804004
:10FC9000834200F0B88000F58060834200F0B380BA
:10FCA00000F58060834200F0AE80774C18882468AD
:10FCB0006408B4FBF2F4013CA4B282B2B3F1804F09
:10FCC0000AD07248834207D000F58060834203D097
:10FCD00000F58060834202D122F0700292B26C483B
:10FCE000834200F0A28000F58060834200F0A7808C
:10FCF00022F4407200F56C4092B283421A80D962BD
:10FD00001C854FD05F4A93424CD001229A821A88B8
:10FD100092B242F001021A80B3F1804F00F0998054
:10FD20005A4A934200F0978002F58062934200F0B5
:10FD3000948002F58062934200F0918002F5806227
:10FD4000934200F08E8002F58062934200F08B8037
:10FD500002F57042934200F0888002F5705293429F
:10FD600000F0858002F58062934200F0828002F507
:10FD7000806293427FD0A2F5983293427DD002F503
:10FD8000806293427BD002F58062934208BF0D22CD
:10FD900015D002A84FF0012340F8043D1AF080FE70
:10FDA00002B010BD0122002119869A821A883948B2
:10FDB00092B242F0010283421A80ADD10A46364B1C
:10FDC00003EBC20301A893F835408DF804400123EA
:10FDD00000228DF805308DF807308DF806201AF0D6
:10FDE0005FFE1B2C08D02E2CDAD12C4B019301A8DE
:10FDF0001AF056FE02B010BD294B019301A81AF06B
:10FE00004FFE02B010BD204C18882468B4FBF2F4F9
:10FE1000013CA4B282B251E71B4C18882468B4FBA1
:10FE2000F2F4013CA4B282B256E701201A80D962F2
:10FE30001C8598821A8892B202431A8070E70120CA
:10FE40001A80D9621C8598821A8892B202431A805D
:10FE500062E70122B3E70222B1E70322AFE70422FF
:10FE6000ADE70522ABE70622A9E70722A7E70822AC
:10FE7000A5E70922A3E70A22A1E70B229FE70C22AC
:10FE80009DE700BF000401406475002000040040AD
:10FE90000010004000000140449903082C010001BB
:10FEA000190100012C4B98423DD0B0F1804F3CD05D
:10FEB000A3F57C4398423AD003F58063984238D04A
:10FEC00003F58063984236D003F58063984234D0BE
:10FED00003F58063984232D003F57043984230D0E6
:10FEE00003F5705398422ED003F5806398422CD0CE
:10FEF00003F5806398422AD0A3F59833984228D01E
:10FF000003F58063984207D003F58063984208BFE9
:10FF10000D2202D0002070470C22104B03EBC203CD
:10FF200093F8340070470022F7E70122F5E7022238
:10FF3000F3E70322F1E70422EFE70522EDE70622CB
:10FF4000EBE70722E9E70822E7E70922E5E70A22CB
:10FF5000E3E70B22E1E700BF0000014044990308FA
:10FF60002DE98048013085B0C3B203938A4D8B4F91
:10FF70008B4C8C4E0A230293DFF82C921BF046FA2E
:10FF80004FF4FA7A4FF0100C4FF47A70D9F804302D
:10FF9000C3F30803002B40F0C180EFF31183002B63
:10FFA00040F0BC802968A26800BF2B689942F9D153
:10FFB000D7F800E000FB0EF39B1AB3FBFEF300FB47
:10FFC00001314FF0010E0191D9F80430C3F3080359
:10FFD000002B40F08780EFF31183002B40F08280EC
:10FFE0002B68A16800BF2A689342F9D1D7F800B006
:10FFF00000FB0BF2521AB2FBFBF200FB0323019A47
:020000040801F1
:100000009B1AB3F57A7FDFD3BAF1010ABED1039B05
:10001000002B40F0BD804FF47A7ADFF88C91504687
:100020004FF0100CD9F80430C3F30803002B40F054
:100030009280EFF31183002B40F08D802968A26835
:1000400000BF2B689942F9D1D7F800E000FB0EF30E
:100050009B1AB3FBFEF300FB01314FF0010E01913F
:10006000D9F80430C3F3080303BBEFF31183EBB9F2
:100070002B68A16800BF2A689342F9D1D7F800B075
:1000800000FB0BF2521AB2FBFBF200FB0323019AB6
:100090009B1AB3F57A7FE3D3BAF1010AC2D1029B6E
:1000A000013B02937FF468AFFAF764FBEFF311882A
:1000B0008CF31288A1682368DB0344BFC6F800E014
:1000C000A1682B6832685FFA88F888F31188D7F83E
:1000D00000801A4400FB08F35B1AB3FBF8F300FB43
:1000E0000233D4E7EFF311888CF31288A1682368F8
:1000F000DB0344BFC6F800E0A1682B6832685FFAF2
:1001000088F888F31188D7F800801A4400FB08F3B8
:100110005B1AB3FBF8F300FB023370E7EFF31182D5
:100120008CF31288D4F808E02368D90303D501239F
:100130003360D4F808E02B683168D2B282F31188BA
:100140003A68194400FB02F3A3EB0E03B3FBF2F38E
:1001500000FB013135E7EFF311828CF31288D4F8FC
:1001600008E02368D90303D501233360D4F808E0FD
:100170002B683168D2B282F311883A68194400FBC7
:1001800002F3A3EB0E03B3FBF2F300FB013164E7D0
:1001900018461AF09DFF3EE7407F0020447F002074
:1001A00010E000E03C7F002000ED00E02DE9F04F82
:1001B000013085B0C3B203930B4602918B4C8C4E39
:1001C000002B00F099808B4D8B4FDFF830921BF0A5
:1001D0001DF94FF4FA7A4FF0100C4FF47A70D9F8F9
:1001E0000430C3F30803002B40F0DE80EFF31183EB
:1001F000002B40F0D9802968A26800BF2B68994283
:10020000F9D1D7F800E000FB0EF39B1AB3FBFEF325
:1002100000FB01314FF0010E0191D9F80430C3F316
:100220000803002B40F08780EFF31183002B40F090
:1002300082802B68A16800BF2A689342F9D1D7F861
:1002400000B000FB0BF2521AB2FBFBF200FB0323DF
:10025000019A9B1AB3F57A7FDFD3BAF1010ABED1B6
:10026000039B002B40F0BD804FF47A7ADFF88C912D
:1002700050464FF0100CD9F80430C3F30803002B9C
:1002800075D1EFF31183002B71D12968A26800BFEB
:100290002B689942F9D1D7F800E000FB0EF39B1AC6
:1002A000B3FBFEF300FB01314FF0010E0191D9F8D1
:1002B0000430C3F3080313BBEFF31183FBB92B68BE
:1002C000A16800BF2A689342F9D1D7F800B000FBBB
:1002D0000BF2521AB2FBFBF200FB0323019A9B1AAA
:1002E000B3F57A7FE3D3BAF1010AC4D1029B013B93
:1002F0000293002B7FF467AF05B0BDE8F08FEFF3FA
:1003000011888CF31288A1682368DB0344BFC6F808
:1003100000E0A1682B6832685FFA88F888F31188DA
:10032000D7F800801A4400FB08F35B1AB3FBF8F31C
:1003300000FB0233D2E7EFF311888CF31288A16837
:100340002368DB0344BFC6F800E0A1682B6832686D
:100350005FFA88F888F31188D7F800801A4400FB08
:1003600008F35B1AB3FBF8F300FB023370E7EFF31B
:1003700011828CF31288D4F808E02368D90303D5DE
:1003800001233360D4F808E02B683168D2B282F3DD
:1003900011883A68194400FB02F3A3EB0E03B3FB88
:1003A000F2F300FB01317FE7EFF311828CF3128847
:1003B000D4F808E02368D90303D501233360D4F8C7
:1003C00008E02B683168D2B282F311883A68194488
:1003D00000FB02F3A3EB0E03B3FBF2F300FB0131CE
:1003E00018E718461AF074FE3EE700BF10E000E080
:1003F0003C7F0020407F0020447F002000ED00E093
:10040000204B5B68C3F3080330B4BBB9EFF311832F
:10041000A3B91D4B1D4C1868A16800BF1A68904213
:10042000F9D11B4B1C684FF47A7202FB04F3591A82
:10043000B1FBF4F130BC02FB00107047EFF3118206
:10044000102383F3128811498C680B6813F4803FE2
:10045000104B02D0012018608C680B49D2B20D6895
:10046000186882F311880A4B19684FF47A7228448D
:1004700002FB01F31B1B30BCB3FBF1F302FB0030AA
:10048000704700BF00ED00E0407F002010E000E07A
:10049000447F00203C7F00202DE9F84F8046FFF785
:1004A000AFFF254E2549DFF8A0E0254A254D8446BB
:1004B00010274FF47A740120DEF80430C3F30803E8
:1004C000D3B9EFF31183BBB90B68D2F808A000BF12
:1004D000D1F800904B45F7D1D6F800B004FB0BF9EA
:1004E000A9EB0A09B9FBFBF904FB0393A3EB0C038B
:1004F0004345E1D3BDE8F88FEFF3118A87F3128803
:10050000D2F808B01368DB0344BF2860D2F808B003
:100510000B68D5F800905FFA8AFA8AF31188D6F84A
:1005200000A0994404FB0AF3A3EB0B03B3FBFAF31B
:1005300004FB0933DAE700BF447F0020407F00203E
:1005400010E000E03C7F002000ED00E02DE9F04FDE
:10055000DFF830C1474A4849484E494D8046102788
:1005600018F1FF38C0F08480DCF80430C3F30803CE
:10057000002B5CD1EFF31183002B58D10B689468EA
:1005800000BF08688342F9D1D6F800904FF47A7022
:1005900000FB09FEAEEB040EBEFBF9FE00FB03EE12
:1005A000DCF80430C3F308034FF47A740120FBB97C
:1005B000EFF31183E3B90B68D2F808A000BFD1F8BC
:1005C00000904B45F7D1D6F800B004FB0BF9A9EB2E
:1005D0000A09B9FBFBF904FB0393A3EB0E03B3F584
:1005E0007A7FBDD2DCF80430C3F30803002BDFD0E0
:1005F000EFF3118A87F31288D2F808B01368DB038F
:1006000044BF2860D2F808B00B68D5F800905FFAB4
:100610008AFA8AF31188D6F800A0994404FB0AF3F9
:10062000A3EB0B03B3FBFAF304FB0933D5E7EFF3BA
:10063000118487F31288D2F808901368D80303D581
:1006400001232B60D2F808900B682868E4B284F389
:100650001188D6F800A04FF47A7400EB030E04FB67
:100660000AF3A3EB0903B3FBFAF304FB0E3E97E78F
:10067000BDE8F08F10E000E0407F0020447F0020C4
:100680003C7F002000ED00E030B4EFF31183102236
:1006900082F312880649074C0A6807480132002590
:1006A0000A602560DBB2026883F3118830BC7047B2
:1006B000407F00203C7F002010E000E00F4B1B88B3
:1006C000014643B90E4B0F4A1B7810680BB981F0F5
:1006D0000101F8F737BB0C4B5A691AB118B91A68FF
:1006E000106058747047094A18681188084A92FBCC
:1006F000F1F2012102605974704700BF187F002099
:100700001A7F00201C7F0020207F0020387F0020DF
:1007100020A1070038B5254B5C69236B73B1A36D2D
:10072000626BCAB1998A1A88C90592B201D5D207FB
:1007300000D438BD4FF6F7721A8038BDA36D998981
:100740001A88890692B2EBD59206E9D5E26ACAB157
:10075000988880B29047E2E799891A880D0692B28C
:10076000E0D51006DED5A26A616A8A4219D0A16975
:100770002569885C98800132B2FBF5F105FB1122F6
:10078000A262CFE79B88E2696169DBB28B54E269C0
:10079000E068A36D0132B2FBF0F100FB1122E261CF
:1007A000BEE7DA6822F08002DA60BBE7E4390020B5
:1007B00038B5254B9C68236B73B1A36D626BCAB1CE
:1007C000998A1A88C90592B201D5D20700D438BDDA
:1007D0004FF6F7721A8038BDA36D99891A88890679
:1007E00092B2EBD59206E9D5E26ACAB1988880B296
:1007F0009047E2E799891A880D0692B2E0D5100673
:10080000DED5A26A616A8A4219D0A1692569885C2D
:1008100098800132B2FBF5F105FB1122A262CFE70D
:100820009B88E2696169DBB28B54E269E068A36D81
:100830000132B2FBF0F100FB1122E261BEE7DA689F
:1008400022F08002DA60BBE7E439002038B5254B9E
:100850001C68236B73B1A36D626BCAB1998A1A8845
:10086000C90592B201D5D20700D438BD4FF6F77250
:100870001A8038BDA36D99891A88890692B2EBD582
:100880009206E9D5E26ACAB1988880B29047E2E759
:1008900099891A880D0692B2E0D51006DED5A26AB3
:1008A000616A8A4219D0A1692569885C9880013201
:1008B000B2FBF5F105FB1122A262CFE79B88E2694A
:1008C0006169DBB28B54E269E068A36D0132B2FB6F
:1008D000F0F100FB1122E261BEE7DA6822F080024B
:1008E000DA60BBE7E4390020436B826A816930B487
:1008F0001C68456A24F001041144AA421C60D960B6
:100900000DD3016900248A1A5A6084621A68002192
:1009100042F0010280F84C1030BC1A607047AA1AED
:100920005A608562F2E700BF03685B6A03B118474B
:10093000704700BF03681B6A03B11847704700BFC8
:1009400003682DE9F041DF691FB13B46BDE8F04186
:100950001847002A164611DD04460D460E4400E0F5
:1009600023689B68204698470028F9D0236815F82B
:10097000011B1B6820469847AE42F1D1BDE8F081CB
:1009800003689B69184700BF03685B69184700BF8D
:1009900003681B69184700BF0368DB68184700BF7E
:1009A00003689B68184700BF03685B68184700BF6F
:1009B00003681B68184700BF38B50C46097849B171
:1009C000054601342B6828461B68984714F8011B1C
:1009D0000029F7D138BD00BF10B40B4B0B4A1C786F
:1009E00001238340234052F8200031B9B3FA83F148
:1009F00049095DF8044BF8F7A5B9191C18BF012186
:100A00005DF8044BF8F79EB9087F00200C7F0020AA
:100A1000064B53F820302BB11A689B8851690B4262
:100A200001D1138370475383704700BF0C7F0020B0
:100A30002DE9F04F4A484B494B4B4C4C4FF0010AC3
:100A40004FF002094FF004084FF0080C4FF0100E61
:100A500020274026802530F8022B12F0010F03D00A
:100A60001960A3F804A0083312F0020F03D0196034
:100A7000A3F80490083312F0040F03D01960A3F810
:100A80000480083312F0080F03D01960A3F804C0E3
:100A9000083312F0100F03D01960A3F804E00833F4
:100AA00012F0200F02D019609F80083312F0400F1F
:100AB00002D019609E80083312F0800F02D01960B6
:100AC0009D80083312F4807F05D04FF4807B19603D
:100AD000A3F804B0083312F4007F05D04FF4007B74
:100AE0001960A3F804B0083312F4806F05D04FF4F6
:100AF000806B1960A3F804B0083312F4006F05D0BE
:100B00004FF4006B1960A3F804B0083312F4805F4F
:100B100005D04FF4805B1960A3F804B0083312F4D9
:100B2000005F05D04FF4005B1960A3F804B00833F0
:100B300012F4804F05D04FF4804B1960A3F804B035
:100B40000833D20B04D04FF4004219609A80083366
:100B500001F58061A1427FF47EAFBDE8F08F00BF58
:100B6000E0AD030800000240EC7C002000100240D1
:100B70002DE9F04FDFF80CB12DED0C8B9BF8003018
:100B80009DB0012B099002F07583394C94F8002137
:100B9000002A41F06B83072B364D02F0EC820023D4
:100BA00006936B683348984700286DD0B5F8A87055
:100BB000002285F84920002F40F09B82B5F924607F
:100BC000E96AB5F926002A6BB5F92830711AA963CC
:100BD00029490591821A686BEA630E461B1A95F83B
:100BE0004A1026482B641EF035FB336813F000537F
:100BF00002F0E482D5ED0F5AD5ED0E7A204A94ED3D
:100C0000676AD4ED686A94ED697AD4F8A8311268FD
:100C1000B8EEE58AD5ED105AF8EEE77AF8EEE58AF7
:100C2000013377EE867A38EE268A78EE878A934209
:100C3000C4ED677A84ED688AC4ED698AC4F8A83186
:100C400001F066869BF80070142F03F07B82D4F8C5
:100C5000B0614FF0000A062E02F28683DFE816F03C
:100C60007818F4192313091A3C1906187F1700BFC6
:100C7000B823002024990020747A00205C99002079
:100C800060A100205D5400209BF80090B9F1070F8F
:100C900000F0E88294F8C031002B40F0F082D44B91
:100CA0005B79002B40F0208201239BF8002084F820
:100CB000C031072A02F0158400230D93CD4B94ED2B
:100CC00072AA93ED007ACC4ADFF8A8A31268CB4B46
:100CD000DFF8A4830692F7EE007A77EECA8AC84A54
:100CE0000A9368EE878A0792F4EEE78AC54A05936D
:100CF00000255346F1EE10FA94ED719ADFF87C93DB
:100D00009FEDC1BADFEDC19ADFEDC1BADFEDC1CA17
:100D1000DFEDC1AA9FEDC1CAC14F0892C24688BF8C
:100D2000F0EE678A2E469846BE4B2B44D3ED007AF0
:100D3000BD4BF5EE407A2B44F1EE10FA93ED008AAC
:100D400017D0BA4B2B4493ED007A78EE476AB0EE99
:100D5000E66AF4EEC67AF1EE10FA08D5F5EEC06A4E
:100D6000F1EE10FACCBF37EE878A37EE678A83ED53
:100D7000008A079BB3F800E01EF0030F00F08782A3
:100D8000022E04F088870699A94B91F8322006EECE
:100D9000902A33F916202B4407EE102A13ED096A26
:100DA00091F83130B8EEC77AF8EEE66A5A4207EEAB
:100DB000902AA6EE867A7100F8EEE77AB4EEE77A2A
:100DC000F1EE10FA0AD407EE903AF8EE677AF4EEF4
:100DD000C77AF1EE10FA88BFF0EE477A954B0B9385
:100DE000954A0B44515EB3F90A30C81A07EE100A4F
:100DF000B8EEC77A1EF0010FE7EE697A00F097822D
:100E0000DFF87CE29EED008A27EE888A94F8D8E12C
:100E1000BEF1000F1FD0DFF868E2D4F8DC01DEED90
:100E2000007ADFF860E25B1A07EE103A099BDEF801
:100E3000001067EEA97AB8EEC78A1B1A8B4228EE1B
:100E4000278A01F3E681F7EE007AB4EEE7AAF1EE25
:100E500010FA01F1A981794B2B44D3ED007A059B5F
:100E6000D3ED01DA69EE277A38EE6DDA67EE8D7A26
:100E7000C8ED007A089BD9ED007A93ED007A704BAB
:100E8000D7ED006A67EE277A2B4427EEA87AD3EDD8
:100E9000007A67EE277AB0EE667AADEE277AF0EE4A
:100EA000477A94ED726AB7EE007AB4EEC76AF1EE53
:100EB00010FAACBF0123002343B1F0EEE66AB0EEB6
:100EC000E77AB4EEE67AF1EE10FA01D5C7ED007AD2
:100ED000022E04F0BB865B4A5B4B52F826001B686F
:100EE000B0EE6D0A9847594A594B52F826001B68D4
:100EF0009847069B93F83A30632B04D8079B1B88CE
:100F0000002B01F09881B0EE6C8A524BD9ED007A3B
:100F100038EE400A2B4493ED008A83ED000A069BCD
:100F200030EE480A93F8482080EE278ADAB1F7EECF
:100F3000007AB4EEE7AAF1EE10FA14DB464BD3EDDB
:100F4000007AB0EEC87AB4EEE77AF1EE10FA0ADD74
:100F5000424BD3ED007AB0EECDDAB4EEE7DAF1EE43
:100F600010FA01F380823E4B94F8E8212B44D3ED34
:100F7000007A69EE277A27EE888A8AED008A2AB9F4
:100F8000C8ED00CAC7ED00CACAED00CA059B04350A
:100F900004330C2D06F101060AF1040A08F10408D5
:100FA00007F1040705937FF4BFAE9BF80030072BD1
:100FB00002F0F081012B02F0998200230593294A67
:100FC0000D4B11681B6893F82F0011F480530693A2
:100FD00000F05A82DFF8B0E0234D9EF80030234E37
:100FE000ED8896ED037A13F0010F214B1A8B4DE03B
:100FF00010990020644000205421002048A10020C6
:10100000502100209400002000009642CDCCCC3D21
:10101000AE47813F000000000000C842610BB63BB4
:101020007085002058400020BC240020842500202A
:101030004825002038B00020681F00201440002000
:1010400020400020E8A70020E4A700204CA80020B2
:1010500048A80020982500207840002074400020F7
:101060002C400020747A0020C0AD0020585500208C
:10107000447A0020648500207C85002010400020F8
:101080004040002068400020CD7F002008BFA4F829
:10109000F021561B07EE906AF8EEE77AB4EEE77A95
:1010A000F1EE10FA42F29681571906EE907AF8EEB8
:1010B000E66AB4EEE67AF1EE10FA81F2FD83B4F856
:1010C000F021964283F28386DB4ADC4DD2ED004A62
:1010D000D5ED003ADA4AC4ED7D3AC4ED7E4AD2ED50
:1010E000006ADFEDD87AE9E1D74B1B78013BDBB230
:1010F000DBE5D64BD6490A9391F801A01B68DFF8CF
:1011000074839BF80090B8F906004FF47A71B1FB34
:10111000F3F3C3EB431603EB8603DE00B6B2B7422C
:1011200003F09680E96FB5F924E02B6E4A1C07EEB8
:1011300090EA7344012AEA672B66F8EEE77A03F037
:101140009180D5ED1B5AD5ED1D6A07EE102A37EEBA
:10115000E56AB8EEC75A012F86EE057A37EE257A92
:1011600077EEC77A85ED1C7AE7EE866A85ED1B7A05
:10117000F0EE667AC5ED1E6AC5ED1D6A03F0858640
:10118000D5F89010B5F926E06B6E4A1C07EE90EA90
:101190007344012AC5F890206B66F8EEE77A03F0F5
:1011A0007980D5ED205AD5ED226A07EE102A37EE68
:1011B000E56AB8EEC75A012F86EE057A37EE257A32
:1011C00077EEC77A85ED217AE6EE276A85ED207AFB
:1011D000F0EE667AC5ED236AC5ED226A03F08B86D0
:1011E000D5F8A410B5F928E0AB6E4A1C07EE90EADA
:1011F0007344012AC5F8A420AB66F8EEE77A03F041
:101200006280D5ED255AD5ED276A07EE102A37EE14
:10121000E56AB8EEC75A012F86EE057A37EE257AD1
:1012200077EEC77A85ED267AE6EE276A85ED257A90
:10123000F0EE667AC5ED286AC5ED276A03F04E86A2
:10124000A8F80600B5F8A8309BF80090013BA5F877
:10125000A8300A990023B9F1070F4B608B60CB606F
:101260007FF418ADFFF7CCF8069BDFF80882C01AB0
:1012700094F8C031A8F80000002B3FF410AD013BFA
:1012800084F8C0311DB0BDEC0C8BBDE8F08F94F834
:10129000D83163B1022E04F001856E4B0B936E4A78
:1012A00003EB460332F91610B3F90A30B3E56B4B82
:1012B0002B4493ED000A059BD3ED01DA29EE000AD9
:1012C00038EE6DDA022E20EE0D0A88ED000A7FF46A
:1012D000D1AD634A634B10681B689847089BD9EDF2
:1012E000007A93ED007A604BD7ED006A1A785F4B75
:1012F00083ED020A5E4B67EE277A2B4467EEA87AED
:1013000093ED006A67EE867AB0EE667AADEE277AE4
:10131000012AF0EE477A02D0192A7FF4C2ADB4EE6A
:10132000CBDAF1EE10FACCBF01230023C4E5B2F909
:1013300000C0D4ED5E6A94ED5F7AB2F902000C90C1
:101340008CEAEC70B4EEE67AA0EBEC70F1EE10FAF9
:101350000E900C984BBFB7EE007AF7EE006A77EE6E
:10136000665A76EEC75A0028B8BF40420F900E98D2
:1013700086460F98864541F33480BCF1000FD6BFF6
:10138000CCF1000007EE10CA07EE100ADFF8E8E023
:10139000B8EEC77A9EF800E027EE297ABEF1000F7A
:1013A00001F03180DFF8D4E09EED005AB5EEC05A6E
:1013B000F1EE10FA41F37387DFF8C4E0DEED004A86
:1013C000F5EEC04AF1EE10FA41F3698734EEC77AC0
:1013D000B7EE006AC7EE246A75EEC65AF4EEC66A26
:1013E00065EEAA5AF1EE10FA85EE857A88BFF0EE26
:1013F000466AF5EEC06AF1EE10FA37EE067AB8BF2B
:10140000F0EE6C6A66EE876AF4EEC66AF1EE10FAE8
:1014100088BFF0EE466AF5EEC06AF1EE10FAB8BF8A
:10142000F0EE6C6ADFF85CE09EED007A67EE877A9A
:10143000A7EEA68AEAE400BFB8AD00201CB00020E9
:10144000D0AD0020000000002CB0002048A10020FA
:101450001099002038B00020681F002014400020A0
:10146000ACAC0020C0AC0020A43E0020648500206D
:1014700020400020605400204C40002048400020C4
:101480005040002044400020E14BE24A5D8B92ED49
:10149000037AE14ADFF8B4E3D2ED003ADF4AC4ED63
:1014A0007D3A07EE905ADE4DD2ED006AD5ED004A46
:1014B000F8EEE77AC4ED7E4A77EE677AC7EEA65A71
:1014C000D84DD94A95ED005AD84D9FEDD97A95ED72
:1014D000003AD84D9FEDD86A95ED004AD2ED006AEA
:1014E000F7EE007AF4EEE75A35EE035AF1EE10FA11
:1014F00088BFF0EE675A35EE045AF4EEC75AF1EEA3
:1015000010FA25EE065AB8BFF0EE475AB1EE667AE9
:1015100033EEE43AB4EEC75AF1EE10FAC4ED7F5A56
:1015200084ED813A00F17384B4EEE65AF1EE10FADC
:1015300088BFB0EE665ABB4A9FEDBF6AD2ED017A12
:10154000BA4AD2ED012ABB4A77EEA27A92ED014A5D
:1015500077EE847A67EE867AB4EEE77AF1EE10FAE7
:1015600008DCF4EEE76AF1EE10FA8CBFB0EE677AB1
:10157000B0EE667AAB4A9FEDB06AD2ED027AAB4A22
:1015800092ED024AAD4A77EE847AD2ED006A67EEB8
:10159000867AB1EE664AF4EEC47AF1EE10FA08D417
:1015A000F4EEE67AF1EE10FA8CBFB0EE664AB0EED9
:1015B000674A002841F03982B7EE002AA04AA14EBE
:1015C000527894F80802002AFFEE002AB7EE006A6B
:1015D000327814BFF0EE467AF0EE627A002814BF3B
:1015E000F0EE626AF0EE466A002A02F0FD86B4EE82
:1015F000C62AF1EE10FA24EE274A934841F35E82A0
:1016000090ED026A90ED011AD0ED037ADFED881AB1
:1016100027EE066A62EE262AA5EE016AA7EE846A24
:1016200026EE226AB4EEE16AF1EE10FAB4BFF0EEF3
:10163000617AF0EE467A8DED106A88BFB0EE616A8D
:10164000012A00F0BD81D0ED066AD0ED051A90EDBB
:10165000072A67EE266AE5EE216AE2EE046A66EE84
:10166000A26AF4EEC66AF1EE10FAF4EEE76A8CBFF5
:10167000B0EE462AB0EE662AF1EE10FA98BFB0EE50
:10168000426AA8BFF0EE667A022ACDED116A00F038
:101690009781D0ED0A6AD0ED091A90ED0B2A67EE1A
:1016A000266AE5EE216AE2EE046A66EEA26AF4EECC
:1016B000C66AF1EE10FAF4EEE76A8CBFB0EE462A85
:1016C000B0EE662AF1EE10FA98BFB0EE426AA8BFFB
:1016D000F0EE667A032ACDED126A00F07181D0ED4A
:1016E0000E6AD0ED0D1A90ED0F2A67EE266AE5EE30
:1016F000216AE2EE046A66EEA26AF4EEC66AF1EED0
:1017000010FAF4EEE76A8CBFB0EE462AB0EE662A15
:10171000F1EE10FA98BFB0EE426AA8BFF0EE667A1A
:10172000042ACDED136A00F04B81D0ED126AD0EDA2
:10173000111A90ED132A67EE266AE5EE216AE2EEB1
:10174000046A66EEA26AF4EEC66AF1EE10FAF4EEEE
:10175000E76A8CBFB0EE462AB0EE662AF1EE10FAC8
:1017600098BFB0EE426AA8BFF0EE667A052ACDEDCA
:10177000146A00F02581D0ED166AD0ED151A90EDAF
:10178000172A67EE266AE5EE216AE2EE046A66EE43
:10179000A26AF4EEC66AF1EE10FAF4EEE76A8CBFC4
:1017A000B0EE462AB0EE662AF1EE10FA98BFB0EE1F
:1017B000426AA8BFF0EE667A062ACDED156A00F0FF
:1017C000FF80D0ED1A6AD0ED191A90ED1B2A67EE52
:1017D000266AE5EE216AE2EE046A66EEA26AF4EE9B
:1017E000C66AF1EE10FAF4EEE76A8CBFB0EE462A54
:1017F000B0EE662AF1EE10FA98BFB0EE426AA8BFCA
:10180000F0EE667A072ACDED166A00F0D9801FE067
:10181000447A0020585500201CB00020C8AD00209C
:101820008CAE0020648500207C4000207085002064
:10183000000000007C8500206F12833A8040002069
:10184000342300204D540020F8AC0020CD7F002030
:10185000D0ED1E6AD0ED1D1A90ED1F2A67EE266AA4
:10186000E5EE216AE2EE046A66EEA26AF4EEC66A6A
:10187000F1EE10FAF4EEE76A8CBFB0EE462AB0EE55
:10188000662AF1EE10FA98BFB0EE426AA8BFF0EEF9
:10189000667A082ACDED176A00F09280D0ED226AB0
:1018A000D0ED211A90ED232A67EE266AE5EE216A33
:1018B000E2EE046A66EEA26AF4EEC66AF1EE10FA8F
:1018C000F4EEE76A8CBFB0EE462AB0EE662AF1EE7F
:1018D00010FA98BFB0EE426AA8BFF0EE667A092A05
:1018E000CDED186A6CD0D0ED266AD0ED251A90EDBA
:1018F000272A67EE266AE5EE216AE2EE046A66EEC2
:10190000A26AF4EEC66AF1EE10FAF4EEE76A8CBF52
:10191000B0EE462AB0EE662AF1EE10FA98BFB0EEAD
:10192000426AA8BFF0EE667A0A2ACDED196A47D05E
:10193000D0ED2A6AD0ED291A90ED2B2A67EE266A9F
:10194000E5EE216AE2EE046A66EEA26AF4EEC66A89
:10195000F1EE10FAF4EEE76A8CBFB0EE462AB0EE74
:10196000662AF1EE10FA98BFB0EE426AA8BFF0EE18
:10197000667A0B2ACDED1A6A22D0D0ED2E1A90EDA0
:101980002D2AD0ED2F6A27EE217AA2EE057AA6EE57
:10199000847A27EE227AB4EEC67AF1EE10FAB4EE2B
:1019A000E77A8CBFF0EE466AF0EE476AF1EE10FA85
:1019B0008DED1B7AD8BFB0EE666AA8BFF0EE477A0D
:1019C00077EEC67AF7EE006AF4EEE67AF1EE10FAF8
:1019D000C4ED727A43F3E48186EEA77A012ADDED45
:1019E000107A67EE877ACDED107A55D0DDED117A59
:1019F00067EE877A022ACDED117A4DD0DDED127AAD
:101A000067EE877A032ACDED127A45D0DDED137AA1
:101A100067EE877A042ACDED137A3DD0DDED147A96
:101A200067EE877A052ACDED147A35D0DDED157A8B
:101A300067EE877A062ACDED157A2DD0DDED167A80
:101A400067EE877A072ACDED167A25D0DDED177A75
:101A500067EE877A082ACDED177A1DD0DDED187A6A
:101A600067EE877A092ACDED187A15D0DDED197A5F
:101A700067EE877A0A2ACDED197A0DD0DDED1A7A54
:101A800067EE877A0B2ACDED1A7A05D0DDED1B7A49
:101A900027EE877A8DED1B7ADF48006810F08050C2
:101AA00000F09A84F6EE005AC4ED7F5A002A02F044
:101AB000B6849EF80050DFF87493DFF87483DFF883
:101AC00074A3DFF874E394F800C25B8B0793FDEE18
:101AD000E37AD9ED006A9AF803A0B8F906909EF867
:101AE00000E005F0010301F0100817EE905A01F430
:101AF0008001BCF1000F40F0A181B8F1000F00F0AF
:101B00006E85002B43F0FB80BAF1000F43F0868115
:101B1000C248DDED107A90ED007AC149E7EE257AF2
:101B2000BDEEE47A17EE103AB0EE647AA3EE277AAF
:101B3000FDEEC77A17EE90EA17EE907AAE45A8BF91
:101B40002F467345C8BF1F4607EE907AF8EEE77A36
:101B5000012AC1ED007A00F04D8190ED047ADDEDAF
:101B6000117AE7EE257AB0EE647AA3EE277AFDEEDD
:101B7000C77A17EE90EA17EE907AAE45A8BF2F46C7
:101B80009E45B8BF1F4607EE907AF8EEE77A022A24
:101B9000C1ED017A00F02E8190ED087ADDED127A28
:101BA000E7EE257AB0EE647AA3EE277AFDEEC77AE7
:101BB00017EE90EA17EE907AAE45A8BF2F469E45E5
:101BC000B8BF1F4607EE907AF8EEE77A032AC1ED18
:101BD000027A00F00F8190ED0C7ADDED137AE7EEDA
:101BE000257AB0EE647AA3EE277AFDEEC77A17EE77
:101BF00090EA17EE907AAE45A8BF2F469E45B8BF33
:101C00001F4607EE907AF8EEE77A042AC1ED037AD0
:101C100000F0F08090ED107ADDED147AE7EE257A91
:101C2000B0EE647AA3EE277AFDEEC77A17EE90EA5B
:101C300017EE907AAE45A8BF2F469E45B8BF1F4607
:101C400007EE907AF8EEE77A052AC1ED047A00F003
:101C5000D18090ED147ADDED157AE7EE257AB0EEBD
:101C6000647AA3EE277AFDEEC77A17EE90EA17EEB4
:101C7000907AAE45A8BF2F469E45B8BF1F4607EED7
:101C8000907AF8EEE77A062AC1ED057A00F0B28084
:101C900090ED187ADDED167AE7EE257AB0EE647AEB
:101CA000A3EE277AFDEEC77A17EE90EA17EE907A48
:101CB000AE45A8BF2F469E45B8BF1F4607EE907A97
:101CC000F8EEE77A072AC1ED067A00F0938090EDEE
:101CD0001C7ADDED177AE7EE257AB0EE647AA3EE92
:101CE000277AFDEEC77A17EE90EA17EE907AAE45A6
:101CF000A8BF2F469E45B8BF1F4607EE907AF8EE64
:101D0000E77A082AC1ED077A74D090ED207ADDEDEC
:101D1000187AE7EE257AB0EE647AA3EE277AFDEE24
:101D2000C77A17EE90EA17EE907AAE45A8BF2F4615
:101D30009E45B8BF1F4607EE907AF8EEE77A092A6B
:101D4000C1ED087A56D090ED247ADDED197AE7EEF0
:101D5000257AB0EE647AA3EE277AFDEEC77A17EE05
:101D600090EA17EE907AAE45A8BF2F469E45B8BFC1
:101D70001F4607EE907AF8EEE77A0A2AC1ED097A53
:101D800038D090ED287ADDED1A7AE7EE257AB0EEBC
:101D9000647AA3EE277AFDEEC77A17EE90EA17EE83
:101DA000907AAE45A8BF2F469E45B8BF1F4607EEA6
:101DB000907AF8EEE77A0B2AC1ED0A7A1AD090ED04
:101DC0002C7ADDED1B7AE7EE257AE3EE274AFDEE6D
:101DD000E47A17EE900A8542A8BF05468342D8BF31
:101DE0002B4607EE903AF8EEE77AC1ED0B7A002A1F
:101DF00000F0A68192000B49094825F017F90A4B1B
:101E00001B68002B00F0A1810EF0A8FD9DE1B0EE53
:101E1000475AFFF790BB00BFFCAF0020F8AC002092
:101E200098850020C8AC00200C400020C4AC0020E5
:101E3000102300206821002090750020B8F1000FC9
:101E400040F07283D248DDED107A90ED007AD149EE
:101E5000E7EE257AB1EE433AB0EE637AA3EE277A45
:101E6000F0EE477ABEF1000F41F08083BAF1000F27
:101E700043F0CF82BDEEE47AFDEEE77A17EE107AFA
:101E800017EE90CA17EE90EAAC45A8BFAE4667457C
:101E9000C8BFBE4607EE90EAF8EEE77A012AC1ED28
:101EA000007A00F04A8190ED047ADDED117AE7EED8
:101EB000257AB0EE637AA3EE277AFDEEC77A17EEA5
:101EC00090CA17EE90EAAC45A8BFAE46BC45B8BF75
:101ED000BE4607EE90EAF8EEE77A022AC1ED017AF3
:101EE00000F02B8190ED087ADDED127AE7EE257A8D
:101EF000B0EE637AA3EE277AFDEEC77A17EE90CAAA
:101F000017EE90EAAC45A8BFAE46BC45B8BFBE468A
:101F100007EE90EAF8EEE77A032AC1ED027A00F0C4
:101F20000C8190ED0C7ADDED137AE7EE257AB0EEB8
:101F3000637AA3EE277AFDEEC77A17EE90CA17EE02
:101F400090EAAC45A8BFAE46BC45B8BFBE4607EE5A
:101F500090EAF8EEE77A042AC1ED037A00F0ED800A
:101F600090ED107ADDED147AE7EE257AB0EE637A23
:101F7000A3EE277AFDEEC77A17EE90CA17EE90EA25
:101F8000AC45A8BFAE46BC45B8BFBE4607EE90EA1A
:101F9000F8EEE77A052AC1ED047A00F0CE8090EDE4
:101FA000147ADDED157AE7EE257AB0EE637AA3EECA
:101FB000277AFDEEC77A17EE90CA17EE90EAAC4585
:101FC000A8BFAE46BC45B8BFBE4607EE90EAF8EEE5
:101FD000E77A062AC1ED057A00F0AF8090ED187A15
:101FE000DDED167AE7EE257AB0EE637AA3EE277A76
:101FF000FDEEC77A17EE90CA17EE90EAAC45A8BF7F
:10200000AE46BC45B8BFBE4607EE90EAF8EEE77AAA
:10201000072AC1ED067A00F0908090ED1C7ADDED84
:10202000177AE7EE257AB0EE637AA3EE277AFDEE13
:10203000C77A17EE90CA17EE90EAAC45A8BFAE4635
:10204000BC45B8BFBE4607EE90EAF8EEE77A082A2C
:10205000C1ED077A71D090ED207ADDED187AE7EEC8
:10206000257AB0EE637AA3EE277AFDEEC77A17EEF3
:1020700090CA17EE90EAAC45A8BFAE46BC45B8BFC3
:10208000BE4607EE90EAF8EEE77A092AC1ED087A33
:1020900053D090ED247ADDED197AE7EE257AB0EE93
:1020A000637AA3EE277AFDEEC77A17EE90CA17EE91
:1020B00090EAAC45A8BFAE46BC45B8BFBE4607EEE9
:1020C00090EAF8EEE77A0A2AC1ED097A35D090ED68
:1020D000287ADDED1A7AE7EE257AB0EE637AA3EE80
:1020E000277AFDEEC77A17EE90CA17EE90EAAC4554
:1020F000A8BFAE46BC45B8BFBE4607EE90EAF8EEB4
:10210000E77A0B2AC1ED0A7A17D090ED2C7ADDED33
:102110001B7AE7EE257AE3EE273AFDEEE37A17EE37
:10212000900A8542A8BF05468742D8BF2F4607EED2
:10213000907AF8EEE77AC1ED0B7A002B3FF457AEB8
:10214000154B1B68002B7FF45FAE144B1B7893B1CB
:10215000307868B10F4FDFF84C800025E8B2D8F82E
:102160000030B7EC010A9847307801358542F5DB3D
:102170000B4B1B6898479BF80030072B01F01F8121
:10218000012384F800311DB0BDEC0C8BBDE8F08F4D
:10219000F8AC0020988500200C400020F879002041
:1021A0008C750020847500200B9BB2F900E0B3F918
:1021B0000A30C749AEEB0300096880EAE073A3EB7D
:1021C000E0738B42BEF647AEB2F902300B9AB2F919
:1021D0000C209A1A82EAE273A3EBE27399427EF72B
:1021E0003AAE0A99BB4BD1ED017A93ED007AF0EE4D
:1021F000E77AF4EEC77AF1EE10FA7EF52CAED1ED67
:10220000027AF0EEE77AB4EEE77AF1EE10FA7EF7B2
:1022100022AEB14B1A88002384F8D831002A40F04E
:102220006D83AE4AAE4B1178186881F00101F6F764
:1022300089FDFEF710BEAB4BAB4A2B4493ED007A01
:10224000D2ED007AA94B67EE277AF7EE006AF4EE3A
:10225000E67AF1EE10FA93ED007A88BFF0EE667A36
:1022600067EE877A27EE888AFEF74FBE072B02F0CB
:10227000928500279E4B05931B689E4D590501F1E1
:10228000C6809D4B1B78002B40F003819B4B94F83C
:10229000126126B19A4A1288920742F0C68094F8D9
:1022A0001811DA7F002941F0BC809E7F002E00F0DB
:1022B000C785022E02F07280032E01F03E84914801
:1022C00040880232D2B2002902F05B80002802F07E
:1022D00058808D4E3668B0FBF6F006B2A4F848611F
:1022E000002A03F01E8207EE906AF8EEE77AF7EE16
:1022F000006A86EEA77ADFF82092012AD4ED576AA9
:10230000D9ED007A77EEE67A67EE877AC4ED537AF4
:1023100021D0D9ED017AD4ED586A77EEE67A022A17
:1023200067EE877AC4ED547A15D0D9ED027AD4EDF0
:10233000596A77EEE67A032A67EE877AC4ED557A12
:1023400009D0D9ED037AD4ED5A6A77EEE67A67EED2
:10235000877AC4ED567A9BF80000092803F0BA8208
:10236000002E40F3748592B3D4ED577A94ED537AEE
:1023700077EE877A012AC4ED577AC9ED007A21D029
:10238000D4ED587A94ED547A77EE877A022AC4ED28
:10239000587AC9ED017A15D0D4ED597A94ED557A71
:1023A00077EE877A032AC4ED597AC9ED027A09D00B
:1023B000D4ED5A7A94ED567A77EE877AC4ED5A7A4C
:1023C000C9ED037A013A022AB8BF0222D2B200292B
:1023D00018BF022200F03CBD4F023FF563ABFFF790
:1023E00065BB0C98DFF834E10028D8BF404207EE07
:1023F000100A9EF800E0B8EEC77A27EE297ABEF1FF
:10240000000F7EF4CFAFDFF818E19EED006AB4EE66
:10241000EB6AF1EE10FA40F1F487B7EE005A35EEB0
:10242000465ADFED3A6ADFF8FCE036EEC77A25EE71
:102430000C5ADEED006AA5EE076A26EE267AB5EEA6
:10244000C07AF1EE10FA40F22A87CAEE876AB7EE38
:10245000006A35EEC67AF0EE465AE7EE265AF0EEFE
:10246000656AFEF7D1BF01230999C4F8DC11022A7D
:1024700084F8D8317EF477AD174A1288002A43F0E9
:102480005881164A164B11781868F6F75BFCFEF770
:102490006ABD1F4A194BB2F906105A8B91423FF799
:1024A000F6AE1C4A1278012A01F05687192A01F06B
:1024B00053870E2A3FF4EBAE082A3FF4E8AEDFF86C
:1024C00058900022C9F80820C4F80C21DFE600BFAC
:1024D0006C40002070400020187F00201A7F0020F0
:1024E0001C7F0020302500203C4000203840002088
:1024F000747A002024990020D81B0020447A002000
:102500005021002004230020CC850020000034430B
:102510001023002034230020585500204C40002078
:102520005440002048400020002B42F0FF81BEF1C3
:10253000000F41F09982FDEEE47A0DF1400C17EEA8
:1025400090EAFDEEE67A0CEB82030693D848DFF8BA
:10255000649308944FFA8AF317EE907AB1EE433AF7
:102560008AF0010807921C46034693ED007AFCECC2
:10257000017AE7EE257A1030B0EE637AA3EE277A7F
:10258000FDEEC77A17EE903A17EE902AAB42A8BF3D
:102590002A469F42CCBF00210AF00101002914BF46
:1025A000114639469E45CCBF002308F0010307EED3
:1025B000901A002B14BF13467346B8EEE77A07EE65
:1025C000903A069BF8EEE77A002C18BFF0EE477AB7
:1025D0006345E9EC017AC7D1079A089C07E4B4483F
:1025E000DDED107A90ED007AB249E7EE257ABAF186
:1025F000000F42F01182BDEEE47A17EE107AB0EED1
:10260000647AA3EE277AFDEEC77A17EE90CA17EE2A
:1026100090EAAC45A8BFAE466745C8BFBE4607EEC8
:1026200090EAF8EEE77A012AC1ED007A3FF485AD31
:1026300090ED047ADDED117AE7EE257AB0EE647A5A
:10264000A3EE277AFDEEC77A17EE90CA17EE90EA4E
:10265000AC45A8BFAE466745C8BFBE4607EE90EA88
:10266000F8EEE77A022AC1ED017A3FF466AD90ED0B
:10267000087ADDED127AE7EE257AAE46B0EE647A9E
:10268000A3EE277AFDEEC77A17EE90CA6545A8BF7C
:10269000E6466745C8BFBE4607EE90EAF8EEE77A21
:1026A000032AC1ED027A3FF448AD90ED0C7ADDEDDE
:1026B000137AE7EE257AB0EE647AA3EE277AFDEE80
:1026C000C77A17EE90CA17EE90EAAC45A8BFAE469F
:1026D000BC45B8BFBE4607EE90EAF8EEE77A042A9A
:1026E000C1ED037A3FF429AD90ED107ADDED147A57
:1026F000E7EE257AB0EE647AA3EE277AFDEEC77A8C
:1027000017EE90CA17EE90EAAC45A8BFAE46BC459E
:10271000B8BFBE4607EE90EAF8EEE77A052AC1EDAB
:10272000047A3FF40AAD90ED147ADDED157AE7EE08
:10273000257AB0EE647AA3EE277AFDEEC77A17EE1B
:1027400090CA17EE90EAAC45A8BFAE46BC45B8BFEC
:10275000BE4607EE90EAF8EEE77A062AC1ED057A62
:102760003FF4EBAC90ED187ADDED167AE7EE257AC2
:10277000B0EE647AA3EE277AFDEEC77A17EE90CA20
:1027800017EE90EAAC45A8BFAE46BC45B8BFBE4602
:1027900007EE90EAF8EEE77A072AC1ED067A3FF4F1
:1027A000CCAC90ED1C7ADDED177AE7EE257AB0EE31
:1027B000647AA3EE277AFDEEC77A17EE90CA17EE79
:1027C00090EAAC45A8BFAE46BC45B8BFBE4607EED2
:1027D00090EAF8EEE77A082AC1ED077A3FF4ADAC4B
:1027E00090ED207ADDED187AE7EE257AB0EE647A86
:1027F000A3EE277AFDEEC77A17EE90CA17EE90EA9D
:10280000AC45A8BFAE46BC45B8BFBE4607EE90EA91
:10281000F8EEE77A092AC1ED087A3FF48EAC90ED24
:10282000247ADDED197AE7EE257AB0EE647AA3EE2C
:10283000277AFDEEC77A17EE90CA17EE90EAAC45FC
:10284000A8BFAE46BC45B8BFBE4607EE90EAF8EE5C
:10285000E77A0A2AC1ED097A3FF46FAC90ED287A45
:10286000DDED1A7AE7EE257AB0EE647AA3EE277AE8
:10287000FDEEC77A17EE90CA17EE90EAAC45A8BFF6
:10288000AE46BC45B8BFBE4607EE90EAF8EEE77A22
:102890000B2AC1ED0A7A3FF450AC90ED2C7ADDEDB5
:1028A0001B7AE7EE257AE3EE274AFDEEE47A36E47A
:1028B000F8AC00209885002007EE902AF8EEE77A21
:1028C000724EDFF8ECC1D6ED004ADCED003A704EF6
:1028D000C4ED7D3A77EE677A06EE905ABCEEC77A81
:1028E000F8EEE66A17EE102A77EEE67AC4ED7E4A35
:1028F000A4F8F021D6ED006AFEF7E0BD65494A690B
:10290000002A3EF4A8AA0A6813604B74FEF7A3BA23
:1029100007EE103A9BF80030DFF89881C4F8A871F0
:10292000B8EEC77AF7EE006A132B86EE879AB8F9ED
:102930000400B4F8AC6195ED080A01F01484564B1C
:10294000564A93ED001A93ED093A93ED162A93ED4A
:102950001F6AD3ED0B1A93ED144AD3ED015AD3ED50
:102960000A3A93ED0C7A93ED155AD3ED172AD3ED6D
:10297000206AD3ED044AD3ED030A67EE897A69EE43
:10298000288A29EE088AA1EE273A02EB8607002161
:10299000A2EE286AC4F89C11C4F8A011A1EE884ADE
:1029A000E5EEA73AA7EE085A93ED1A7AD3ED0F5A3F
:1029B00093ED021AD3ED0E1A87ED003AE2EEA86A03
:1029C00064EEC34A27EE467A93ED0D2AD3ED192A19
:1029D00087ED204AE0EEC33A65EEC45A93ED183A0B
:1029E000C3ED093AE1EE274AF0EE477AA1EEC45A68
:1029F000E2EE085AE2EEC66AE3EE287AC3ED0A4A2E
:102A000083ED145AC3ED155A87ED406AC3ED1F6A72
:102A1000C3ED207AC4F8A411731C03F01F03A4F8BB
:102A2000AC31A8F80400FEF70DB91D4A1079002852
:102A30003EF4C2AD1B48007800283EF4BDAD1278CC
:102A4000DFED192A07EE902A184AF8EE676A128815
:102A500007EE900A06EE102AF8EEE77AB8EE466A1C
:102A600066EEA77AF7EE006A87EE862AB4EEE22ACF
:102A7000F1EE10FA88BFB0EE622AB4EEE62AF1EE6B
:102A800010FAB8BFB0EE662AFEF798BDB8AD0020C8
:102A9000D0AD0020207F002020A4002084A10020B1
:102AA000701F002057550020713DAA3F145500208B
:102AB0001CB00020605400200000000090ED026A6D
:102AC00090ED012AD0ED037A5FED052A27EE066A24
:102AD000A5EE026AA7EE846A26EE266AB4EEE26AE2
:102AE000F1EE10FAB4BFF0EE627AF0EE467A8DEDB8
:102AF000106A88BFB0EE626A012A3EF461AFD0ED81
:102B0000062AD0ED051A90ED072A67EE222AE5EE97
:102B1000212AE2EE042A62EEA62AF4EEC62AF1EE9B
:102B200010FAF4EEE72A8CBFB0EE462AB0EE622A25
:102B3000F1EE10FA98BFB0EE426AA8BFF0EE627AEA
:102B4000022ACDED112A3EF43BAFD0ED0A2AD0ED9A
:102B5000091A90ED0B2A67EE222AE5EE212AE2EE11
:102B6000042A62EEA62AF4EEC62AF1EE10FAF4EE7A
:102B7000E72A8CBFB0EE462AB0EE622AF1EE10FAD8
:102B800098BFB0EE426AA8BFF0EE627A032ACDED9C
:102B9000122A3EF415AFD0ED0E2AD0ED0D1A90EDAD
:102BA0000F2A67EE222AE5EE212AE2EE042A62EEDF
:102BB000A62AF4EEC62AF1EE10FAF4EEE72A8CBF4C
:102BC000B0EE462AB0EE622AF1EE10FA98BFB0EEEF
:102BD000426AA8BFF0EE627A042ACDED132A3EF4D1
:102BE000EFAED0ED122AD0ED111A90ED132A67EE58
:102BF000222AE5EE212AE2EE042A62EEA62AF4EE6B
:102C0000C62AF1EE10FAF4EEE72A8CBFB0EE462A9F
:102C1000B0EE622AF1EE10FA98BFB0EE426AA8BF99
:102C2000F0EE627A052ACDED142A3EF4C9AED0ED5D
:102C3000162AD0ED151A90ED172A67EE222AE5EE36
:102C4000212AE2EE042A62EEA62AF4EEC62AF1EE6A
:102C500010FAF4EEE72A8CBFB0EE462AB0EE622AF4
:102C6000F1EE10FA98BFB0EE426AA8BFF0EE627AB9
:102C7000062ACDED152A3EF4A3AED0ED1A2AD0EDEA
:102C8000191A90ED1B2A67EE222AE5EE212AE2EEC0
:102C9000042A62EEA62AF4EEC62AF1EE10FAF4EE49
:102CA000E72A8CBFB0EE462AB0EE622AF1EE10FAA7
:102CB00098BFB0EE426AA8BFF0EE627A072ACDED67
:102CC000162A3EF47DAED0ED1E2AD0ED1D1A90EDF1
:102CD0001F2A67EE222AE5EE212AE2EE042A62EE9E
:102CE000A62AF4EEC62AF1EE10FAF4EEE72A8CBF1B
:102CF000B0EE462AB0EE622AF1EE10FA98BFB0EEBE
:102D0000426AA8BFF0EE627A082ACDED172A3EF497
:102D100057AED0ED222AD0ED211A90ED232A67EE8E
:102D2000222AE5EE212AE2EE042A62EEA62AF4EE39
:102D3000C62AF1EE10FAF4EEE72A8CBFB0EE462A6E
:102D4000B0EE622AF1EE10FA98BFB0EE426AA8BF68
:102D5000F0EE627A092ACDED182A3EF431AED0EDBC
:102D6000262AD0ED251A90ED272A67EE222AE5EED5
:102D7000212AE2EE042A62EEA62AF4EEC62AF1EE39
:102D800010FAF4EEE72A8CBFB0EE462AB0EE622AC3
:102D9000F1EE10FACDED192A98BFB0EE426AB8BF35
:102DA000F0EE672A0A2A02F08D84D0ED2A7AD0ED5F
:102DB000291A90ED2B2A67EE277AE5EE217AE2EECA
:102DC000047A67EEA67AF4EEC67AF1EE10FAF4EE23
:102DD000E27A8CBFB0EE462AB0EE672AF1EE10FA26
:102DE000CDED1A7A98BFB0EE426AB8BFF0EE627AC3
:102DF0000B2A3EF4E5ADD0ED2E2AD0ED2D1A90ED44
:102E00002F2A67EE222AE5EE212AE4EE022A62EE5C
:102E1000A62AB4EEE26AF1EE10FAF4EEE27A8CBF82
:102E2000B0EE627AB0EE467AF1EE10FACDED1B2AE2
:102E300058BFB0EE476AB8BFF0EE627AFEF7C0BD89
:102E4000A4F84861002900F07281DFF86C93022237
:102E5000CB49DFEDCC6A08689BF800C0017890F898
:102E600002E007EE901AF8EEE77AB0EE007A67EE2D
:102E7000A67AF4EEC77AF1EE10FA40F3A88237EEA4
:102E8000C77ADFEDC16AB0EE676AA7EE266AB0EED8
:102E9000467A9FEDBE6AD9ED006A66EE866AB0EEAC
:102EA000E66AC4ED5B6A84ED5E6ABEF1000F13D082
:102EB00005EE90EAB8EEE55ADFEDB25A66EEA64AA4
:102EC00025EE255AF7EE005A75EEC55A64EE864A8D
:102ED000E5EE245A66EEA56ADFEDAD5A417927EE9C
:102EE000257A27EE267AC9B1DFEDA66ADFEDA95A69
:102EF00026EE266A06EE901AF8EEE66A66EE866A16
:102F0000F4EEE56AF1EE10FA00F3AA85F7EE005A46
:102F100075EEE66A85EEA66A27EE067ABCF10C0F1E
:102F20009FED9D8ADFED9D6A00F05A85B4EEC87A68
:102F3000F1EE10FA98BFB0EE478AB4EEE68AF1EEF1
:102F400010FAB8BFB0EE668A84ED418A002A00F01C
:102F5000E280B0EE007AF4EEC77AF1EE10FA05DD09
:102F600037EEC77ADFED886AE7EE267A99ED017AC7
:102F7000DFED866A27EE267AB0EEC76A84ED5C7ACA
:102F800084ED5F6ABEF1000F13D006EE90EADFED2C
:102F90007D5AF8EEE66A27EE075A66EEA56AF7EE66
:102FA000005A75EEE65A25EE065AE6EE855A27EEE9
:102FB000257ADFED776A817967EEA67A67EE877A00
:102FC000A9B107EE101AB8EEC77ADFED6E5ADFED41
:102FD000716A27EE067A27EE257AB4EEE67AF1EEEC
:102FE00010FA40F32F85DFED6E6A67EEA67ABCF12A
:102FF0000C0F00F0D484DFED686A9FED687AF4EE80
:10300000E67AF1EE10FA88BFF0EE667AF4EEC77A4F
:10301000F1EE10FAB8BFF0EE477A012AC4ED427A19
:1030200079DD4278DFED576A07EE902AF8EEE77A0D
:10303000B0EE007A67EEA67A427AF4EEC77AF1EE45
:1030400010FA05DD37EEC77ADFED4F6AE7EE267A34
:1030500099ED027ADFED4D6A27EE267AB0EEC76A67
:1030600084ED5D7A84ED606A9AB106EE902ADFED18
:10307000455AF8EEE66A27EE075A66EEA56AF7EEBD
:10308000005A75EEE65A25EE065AE6EE855A27EE08
:10309000257ADFED3F6AC27967EEA67A67EE877A16
:1030A0000AB307EE102AB8EEC77ADFED365ADFED25
:1030B000396A27EE067A27EE257AB4EEE67AF1EE43
:1030C00010FA0CDCB5EEC07AF1EE10FA01F14B818A
:1030D000B7EE006A36EE477AC6EE076A01E0DFED2A
:1030E000306A67EEA67ABCF10C0F00F09684DFED33
:1030F0002A6A9FED2A7AF4EEE67AF1EE10FA88BF9A
:10310000F0EE667AF4EEC77AF1EE10FAB8BFF0EEA0
:10311000477AC4ED437ABCF1090F00F0348493F888
:103120002160002E40F0E783002384F818311D4B06
:103130001B689E0609D51C4B1B8803F0300323B186
:103140001A4B1B78D80701F1FF86194B1B7823B95E
:10315000184EB378002B41F0AA81099821F0FCFDAC
:103160009BF80030072B00F062840022072B84F8C4
:1031700000217DF414ADFDF743F90690FDF711BD74
:10318000582100200AD7233CD7A368416F12033B84
:1031900000004843A4707D3F00C0F94400C0F9C45A
:1031A0000000C8425CA10020502100207E1F0020AA
:1031B00067430020C255002058550020D54A0A9286
:1031C00092460026D44FDFF86C83B146B7EC018AF3
:1031D000D5ED087AB8EEC88A28EE278AB9F1000F33
:1031E00002F023857BBB9BF8001008293BD006F535
:1031F000D260B0EE480A2844D5F88C36984706F5D8
:10320000E360D5F81437284498479BF80030032B27
:10321000B0EE408A22D0D5F8AC30D7F84406B0EEF4
:10322000480A98470AEB890309F10109B9F1030F2C
:1032300006F12C0683ED010A3DF426AD059B1B68C3
:1032400003F00053C2E706F5F460B0EE480A2844E4
:10325000D5F89C379847B0EE408AC4E724F05AF876
:1032600028F81900D7E7B0EE480A24F053F828F8F8
:103270001900BCE7A94BAA4C1A68AA4BDFF8B48224
:1032800094F80001D2691B88A8F80020A8F8023041
:1032900000287EF4EEAF0690A34DFDF782BCDFED73
:1032A000A36AFEF7BFB8DFF8B492D4ED017A94EDCB
:1032B000006AB9F80000D9F8143077EEA77AF0EE7A
:1032C000006AB0EE677AA6EE267A013804EBC002F7
:1032D000D6EE267A083A1033F6EE003A27EE237A35
:1032E00067EEA37A84ED207AC4ED217A8C4CA64651
:1032F00004F1800192ED027A92ED036ADEED036A39
:10330000DEED027A53ED014A13ED025A37EE674AB9
:1033100076EEC65A77EE277AE4EE845A0138A2F1A7
:103320000802E5EE047A0EF1080E03F1080336EE0A
:10333000267A01F10801E4EE877AE5EE475A67EE56
:10334000A37A25EEA37AC1ED007A81ED017AD1D17D
:10335000142F09D1FDF754F8DFF8D881A0EB0A004B
:10336000A8F80200D4F8B0616A4B0A93704A059B32
:10337000DDF828A01B68013682FB06129119F217AE
:10338000C2EBA102C2EBC202B61AC4F8B06103F0EC
:10339000005316E7FDF734F89BF800300D9ADFF87C
:1033A0009481801A012BA8F8020000F0A180072B5D
:1033B0007DF403AEFDF724F80590FDF700BEFDF7A0
:1033C0001FF8059A5B4B801AD880FEF7D9BEB0EE85
:1033D000677A5EE5584D594E594AD5ED004AD6ED0B
:1033E000003A584D1278C4ED7D3AC4ED7E4AD5EDD1
:1033F000006A12B1012284F80022D4ED7F7AFEF730
:103400005DB8DFF85CE19EED007AFFF718B8AB68B5
:10341000002B3EF436AF05F1440128469847FEF7ED
:1034200030BF4948494ED0F8EC00366844F6206E6B
:103430007045A8BF7046B0F57A7FB8BF4FF47A7078
:1034400016F0100F059E80B2A4F81A01366801F03C
:10345000B884F60400F17B833D4ED6F800C0BCF979
:1034600036E0DFF80091DFF80081D4F81C61D9ED77
:10347000037AA8FB00084FEA9818642090FBF8F044
:103480001428BDEEE77A04EB4609A8BF14200136E4
:103490008642C4F81C6117EE10AAA4BF0026C4F827
:1034A0001C6104EB4606A9F820A1B6F9200107EE3D
:1034B000100AB8EEC77A77EEC77AFDEEE77ACDED5F
:1034C000067ABDF9186086EAE670A0EBE6707045F2
:1034D00002F318811F4806464FF07E503060FEF719
:1034E000E4BEFCF78DFF0D90FDF7E8BBDFF84480EC
:1034F000FCF786FF184AD4F8EC3112680590C31A1D
:103500009A1AC4F8EC01A8F80430A8F80620FDF7D0
:1035100056BD00BF48A100205C9900208C8200208D
:10352000B8230020BE3A00202499002000000000AB
:1035300093244992605400208CAE0020BCAD002042
:1035400090750020CCAD0020D8170020FCAF0020E3
:103550005421002094000020CC8500206CA1002084
:103560004840002058550020D34D6210BAF1000F9A
:103570003EF480ACF4EEE47AF1EE10FAB8BFF0EE6F
:10358000667AFDEEE77ABDEEE67A17EE90EA17EE80
:1035900090CAAE4517EE107AA8BFAC467745C8BFB3
:1035A000BC4607EE90CAF8EEE77A012AC1ED007A30
:1035B0003EF4C3AD90ED047ADDED117AE7EE257AA5
:1035C000B0EE637AA3EE277AB4EEE47AF1EE10FA65
:1035D000F0EE477AB8BFF0EE667AFDEEE77A17EEC6
:1035E00090EA17EE90CAAE45A8BFAC46BE45B8BF3C
:1035F000BC4607EE90CAF8EEE77A022AC1ED017ADE
:103600003EF49BAD90ED087ADDED127AE7EE257A77
:10361000B0EE637AA3EE277AB4EEE47AF1EE10FA14
:10362000F0EE477AB8BFF0EE667AFDEEE77A17EE75
:1036300090EA17EE90CAAE45A8BFAC46BE45B8BFEB
:10364000BC4607EE90CAF8EEE77A032AC1ED027A8B
:103650003EF473AD90ED0C7ADDED137AE7EE257A4A
:10366000B0EE637AA3EE277AB4EEE47AF1EE10FAC4
:10367000F0EE477AB8BFF0EE667AFDEEE77A17EE25
:1036800090EA17EE90CAAE45A8BFAC46BE45B8BF9B
:10369000BC4607EE90CAF8EEE77A042AC1ED037A39
:1036A0003EF44BAD90ED107ADDED147AE7EE257A1D
:1036B000B0EE637AA3EE277AB4EEE47AF1EE10FA74
:1036C000F0EE477AB8BFF0EE667AFDEEE77A17EED5
:1036D00090EA17EE90CAAE45A8BFAC46BE45B8BF4B
:1036E000BC4607EE90CAF8EEE77A052AC1ED047AE7
:1036F0003EF423AD90ED147ADDED157AE7EE257AF0
:10370000B0EE637AA3EE277AB4EEE47AF1EE10FA23
:10371000F0EE477AB8BFF0EE667AFDEEE77A17EE84
:1037200090EA17EE90CAAE45A8BFAC46BE45B8BFFA
:10373000BC4607EE90CAF8EEE77A062AC1ED057A94
:103740003EF4FBAC90ED187ADDED167AE7EE257AC3
:10375000B0EE637AA3EE277AB4EEE47AF1EE10FAD3
:10376000F0EE477AB8BFF0EE667AFDEEE77A17EE34
:1037700090EA17EE90CAAE45A8BFAC46BE45B8BFAA
:10378000BC4607EE90CAF8EEE77A072AC1ED067A42
:103790003EF4D3AC90ED1C7ADDED177AE7EE257A96
:1037A000B0EE637AA3EE277AB4EEE47AF1EE10FA83
:1037B000F0EE477AB8BFF0EE667AFDEEE77A17EEE4
:1037C00090EA17EE90CAAE45A8BFAC46BE45B8BF5A
:1037D000BC4607EE90CAF8EEE77A082AC1ED077AF0
:1037E0003EF4ABAC90ED207ADDED187AE7EE257A69
:1037F000B0EE637AA3EE277AB4EEE47AF1EE10FA33
:10380000F0EE477AB8BFF0EE667AFDEEE77A17EE93
:1038100090EA17EE90CAAE45A8BFAC46BE45B8BF09
:10382000BC4607EE90CAF8EEE77A092AC1ED087A9D
:103830003EF483AC90ED247ADDED197AE7EE257A3B
:10384000B0EE637AA3EE277AB4EEE47AF1EE10FAE2
:10385000F0EE477AB8BFF0EE667AFDEEE77A17EE43
:1038600090EA17EE90CAAE45A8BFAC46BE45B8BFB9
:10387000BC4607EE90CAF8EEE77A0A2AC1ED097A4B
:103880003EF45BAC90ED287ADDED1A7AE7EE257A0E
:10389000B0EE637AA3EE277AB4EEE47AF1EE10FA92
:1038A000F0EE477AB8BFF0EE667AFDEEE77A17EEF3
:1038B00090EA17EE90CAAE45A8BFAC46BE45B8BF69
:1038C000BC4607EE90CAF8EEE77A0B2AC1ED0A7AF9
:1038D0003EF433AC90ED2C7ADDED1B7AE7EE257AE1
:1038E000E3EE273AF4EEE34AF1EE10FAC8BFF0EE49
:1038F000663AFEF712BC1E21CD48F6F756FB0028AB
:103900003FF412ACCB4B1B885B063FF50DAC94F833
:103910008431B34241F06A87C74BD4ED627A93EDAC
:10392000017A94ED435ADFEDC55A9FEDC56A67EE03
:10393000C56A68EE277AE8EE076AE5EE077AF4EEE4
:10394000E56AF1EE10FA8CBFB0EE657AB0EE667AF9
:10395000B4EEC67AF1EE10FAF4EEE57AB8BFB0EE46
:10396000467AF1EE10FA88BFF0EE657AF4EEC67A88
:10397000F1EE10FAB8BFF0EE467A84ED417AC4ED6C
:10398000437AFFF7D1BBFDEEC87ADFF8D48217EE99
:10399000902AA8F80460A8F80620FFF7C0BB9FEDA6
:1039A000A77ADFEDA76ADFF8B882F4EEC77AF1EE06
:1039B00010FA98BFB0EE677AFDEEE77AB4EEE67AD9
:1039C000F1EE10FA17EE901AB8BFB0EE667A012A3F
:1039D00084ED427AA8F802103FF723ABFFF79FBBB4
:1039E000B4EEC87AF1EE10FA98BFB0EE478ABDEE99
:1039F000C77AB4EEE68ADFF86882F1EE10FA17EEC5
:103A0000101AB8BFB0EE668A84ED418AA8F800109B
:103A1000002A7FF49EAAFFF782BBBDEEE77ADFF8AB
:103A2000408217EE102AA8F80420FFF760BBFCF7CD
:103A3000E7FCDFF82C829BF80030C01BA8F80400DC
:103A4000FFF793BBB5EEC07AF1EE10FA00F18F8468
:103A5000B7EE006A36EE477AC6EE076AFFF7C5BAD8
:103A60009FED786AFFF758BAFDEEE47A10A817EEDA
:103A700090EAFDEEE67A00EB82030693DFF8E4912C
:103A8000DFF8E4C108944FFA8AF317EE907AB1EEAA
:103A9000433A8AF0010807921C464B4693ED007AA0
:103AA000F0EC017AE7EE257A0AF0010309F110093A
:103AB000B0EE637AA3EE277AF4EEC74AF1EE10FA7D
:103AC000D8BF0023002BF0EE477A18BFB0EE667A1D
:103AD000BDEEC77AFDEEE77A17EE102A17EE901AC0
:103AE000AA4217EE103AA8BF2B469742CCBF00223D
:103AF0000AF00102002A08BF3B46A94217EE902AAD
:103B000007EE103AA8BF2A468E45CCBF002308F026
:103B10000103002B08BF724607EE902AB8EEC77A61
:103B2000F8EEE77A069B002C18BFF0EE477A984231
:103B3000ECEC017AB1D1FEF74FBD93F82000C0EB59
:103B4000401600EB8600C00080B2FEF7BABB3E4EC6
:103B5000D6F800C0BCF836E04FEA5E0E81E43B4B7D
:103B6000D4F8B4810A93B4F8AC91C9F12003D8B267
:103B7000374B09EB481E03EB8E0E830801F0A58638
:103B800001331B013349344A07930EEB030C0EF14A
:103B9000100313ED024A13ED035A13ED016A13EDFE
:103BA000047A51ED024A51ED035A51ED016A51ED8B
:103BB000047A64EE244A65EE255A66EE266A67EEBC
:103BC000277A1033634542ED024A42ED035A42ED33
:103BD000016A42ED047A01F1100102F11002D8D11C
:103BE000079B1E49A3F11002964401EB020C2244EC
:103BF00010F0030309D0BEEC017AFCEC017A67EE09
:103C0000277A013BE2EC017AF5D1B9F1000F41F0DE
:103C10002084142F7FF4AAABFCF7F2FBDFF840807E
:103C2000D4F8B061A0EB0A00A8F80200FFF79EBB31
:103C3000FCAF0020502100209400002000C0F94477
:103C400000C0F9C40000C8425421002048A100204F
:103C500084A1002014A30020C823002004A3002076
:103C600060540020F8AC002098850020D4F8B4916E
:103C7000E74AE84B0A9203EBC903126807929DEDED
:103C8000077A9B88DFEDE47AE44AF8EE478A09EE8A
:103C9000103A643BC82BA8BFC82368EEA78AF8EE89
:103CA000497A782BB8BF782368EEA78A07EE903A56
:103CB0004FF02C08B0EE680A08FB0928B8EEE78A36
:103CC00023F074FBB8EEC99AF0EE409AB0EE680AA1
:103CD00023F0CEFA38EE097A79EE487A28EE098A8E
:103CE00067EE877AB7EE006A88EE277A142FF8EE2F
:103CF000007A77EE076A60EE277A89EEA67A77EE89
:103D0000065A36EE477AC6EE256A67EEA67A27EEA1
:103D1000267AC8ED006A88ED047AC8ED026AC8ED1B
:103D2000017AC8ED037A01F0FB85BD4B9BF800706A
:103D300009F1010983FB0938A8EBE97808EB480889
:103D40000136A9EB0808C4F8B061C4F8B4810AE7E9
:103D5000DFF8EC92B9F80070D9F804E04FEA570C9C
:103D60004FEA8C0204EB8708FF0804EB020300F023
:103D70009F8010320137AB4803EB071742441033E2
:103D80000EF1100608F1100151ED032A51ED043A2D
:103D900010ED043A10ED032A51ED026A11ED016AAB
:103DA00010ED020A10ED018A12ED044A12ED035AD9
:103DB00053ED044A53ED035A13ED027A53ED017AA1
:103DC00052ED020A12ED011A73EE238A72EE221AE4
:103DD00040ED048A40ED031A70EE268A78EE061A4A
:103DE00040ED028A40ED011A74EE848A75EE851A60
:103DF00043ED048A43ED031A77EE208A77EE811AA9
:103E000043ED028A43ED011A73EE633A75EE655A8B
:103E100016ED035A32EE623A74EE644A65EE631AA6
:103E200016ED044A23EE052A64EE652AE3EE041A31
:103E30001033BB4224EE843AA3EE842A00F1100032
:103E400006F11006A5EE853A01F1100102F110020B
:103E5000E4EE852A41ED071A01ED082A02ED073A42
:103E600042ED082A56ED055A16ED065A70EE666ABE
:103E700038EE466A30EEC77A71EE677A26EE253A5A
:103E800065EEE63A25EE674A67EE054AE6EE053A44
:103E9000A6EE853AA7EE254AE7EEA54A01ED063AD9
:103EA00041ED053A02ED064A42ED054A7FF46CAF5A
:103EB0001FFA8CF6724631465B481BF025FB3146F3
:103EC000D9F8042040461BF01FFB9BF80030142B50
:103ED0007FF448AAFFF73EBA544B1A78D4F8B4E1FD
:103EE0004C489FED537A4FEACE0C00EB0C0383ED68
:103EF000007A002A7CD04C49B0EE476AF0EE476A5F
:103F00000023F1EC017A013367EEA77A05EE903ACF
:103F1000B4EEE77AF1EE10FAF8EEE55AB8BFB0EE7B
:103F2000677A934276EEA76AA7EEA56AE9D1F5EE25
:103F3000C06A00EB0C03F1EE10FA83ED007A57DD56
:103F4000C6EE265A3B4B3C4A1288F7EE007A75EED5
:103F5000E75AD3ED007A65EEA77AFDEEE77A17EE21
:103F6000903A812B41F370809342A8BF134607EE2D
:103F7000903AF8EEE77A314B2C2101FB0E3393EDAA
:103F8000097AD3ED003A93ED0A6A93ED014AD3ED35
:103F9000046AD3ED034A93ED025AA3EEA77AA4EE86
:103FA000276A66EEC76AA7EE646ABDEEC77AE5EED9
:103FB000276A17EE101A812983ED096AC3ED0A6A90
:103FC00041F33F808A42A8BF0A4607EE902AF8EEE6
:103FD000E77AFCEEE77ACDED077ABDF81C3000EB0E
:103FE0000C029380BEF1000F02D1132F01F0BE83AB
:103FF000152F7FF4ADA96044DFF84880838828F846
:104000001E30034BD4F8B0610A93FFF7AFB900BF7D
:1040100048A1002084A3002027D4D236C4A00020C9
:1040200056555555C8230020B823002066A100200E
:104030000000000068A1002064A100209CA30020D3
:104040006CA1002060540020DFF88493D748D9F891
:104050000820B9F80C1022F0A1F89BF80070142F7A
:1040600001F08784D4F8B0610136C4F8B061FFF77D
:104070001CB9DFF8609399F800205FEA920801F01C
:10408000E084DFF854C308F1010040010CEB000E9E
:104090000CF12003ACF1700113ED076A53ED056AD2
:1040A00013ED037A53ED017A53ED025A13ED084AEA
:1040B00053ED064A13ED045A26EE066A66EEA66A2A
:1040C00027EE077A67EEA77AA4EE046A20337345D9
:1040D000E4EEA46A01F11001A5EE057AE5EEA57AF9
:1040E000F1EEC65AB1EEE66AF1EEC76AB1EEE77AD2
:1040F00041ED085A01ED076A41ED066A01ED057AC6
:10410000CAD12038844404EB081112F0030318BF0D
:104110000CF1080C0FD05CED017A1CED027A67EE11
:10412000A77A013BE7EE077A0CF1080CB1EEE77ACB
:10413000A1EC017AEFD1142F01F027840136C4F8E5
:10414000B061CBE6FCF75CF99BF80070142F05BF5B
:10415000DFF88882D4F8B061D4F8B061A8F80060C4
:104160008246FCF778BD924FDFF8749297ED004AD3
:1041700097ED097AD7ED014A97ED0A6AD7ED046AFF
:1041800097ED035AD7ED025A67EE897A09EB860359
:10419000A4EE277AA4EEA76A66EEC76AA5EE476A80
:1041A000E5EEA76A27EE000A87ED096AC7ED0A6AFD
:1041B00083ED007A29EE088A23F0ACF869EE288AAC
:1041C000D7ED145AD7ED1F6A97ED0B1AD7ED161AD3
:1041D00097ED155A97ED207A97ED0C2AD7ED172A0F
:1041E00097ED0F6AD7ED1A7A97ED0E3AD7ED0D3AA3
:1041F00097ED194AD7ED184AE1EE085A002209EB6B
:104200008603E8EEA16A00B2C4F89C21A2EE085A27
:10421000C4F8A021C4F8A421A8EEA27A26EE656A0B
:1042200067EEE67AA3EE655AA3EE886AA6EEC47A34
:10423000E8EEA47A87ED145AC3ED205A87ED156A8B
:10424000C3ED406A87ED1F7AC7ED207AFEF7E4BB25
:10425000B5F92430EA6207EE903A0122F8EEE77AE7
:104260002B66EA670023012FC5ED1C7AC5ED1B7A8A
:104270006B6701F06D82B7427CF482AFB5F92630EE
:104280006B6607EE903A00220123F8EEE77A2A6384
:10429000C5F890300023012FC5ED217AC5ED207AB5
:1042A000C5F8883001F04182B7427CF499AFB5F986
:1042B0002830AB6607EE903A00220123F8EEE77A49
:1042C0006A63C5F8A4300023012FC5ED267AC5ED39
:1042D000257AC5F89C307CF4B3AF9FED368AB9F1EE
:1042E000030F48D0BAF1000F09D007EE90AAF8EEFC
:1042F000E77AF4EEC87AF1EE10FA01F1C4832E4A9F
:10430000AB6E126894F8B811A8F8060003EB5603D8
:1043100093FBF6F600236E6393621363D36221B1BD
:10432000264B1B88002B7CF48DAF254B1B6813F4A8
:10433000003304D0234B1B79002B41F036832249F4
:104340001A46C85C012803F10C0301F066800132B3
:10435000152AF6D1FCF776BF1C4A927B002A3EF460
:10436000AEA8FDF794BFF7EE006AFEF7BABEF7EE0F
:10437000006AFEF73ABEB0EE480A22F0CBFF00B268
:10438000B0E7B4F84861013E36B2002EA4F84861A7
:104390007EF758ADDFF84C90FDF7E5BFB4F81A0191
:1043A00000F57A7080B2FDF78CBF00BFB823002003
:1043B00020A40020000000008C8200204E2100205C
:1043C000D03B0020701F002078A0030894740020C8
:1043D0006CA1002066A10020382400206054002039
:1043E00084A1002058550020C448DFEDC57A00683C
:1043F000C4ED727A10F0805000F00285B7EE007ABA
:1044000077EE677AF4EEE57AF1EE10FA88BFF0EE17
:10441000657AF0EE675AC4ED7F7AFDF747BB9EF8E8
:10442000003003F00103FDF788BEB64ADFEDB67A2F
:1044300092ED080AB4EEE70AF1EE10FA41F20580B7
:10444000069322F0FDFFD4ED457A20EE270A22F0F4
:1044500061FFB0F5617F069B01F3678007EE900A6C
:10446000F8EEE76ADFEDA97A66EEA76A07EE906AD2
:10447000B8EEE77AFDEEE67A17EE902A2032402A6F
:1044800041F29B829FEDA20A069322F043FF00B205
:1044900007EE900A069BB8EEE77ADFF89492D9ED22
:1044A000037A77EE877AC9ED037AFDF7F8BEDFF875
:1044B000848298F80020013A0D2A18D8DFE812F01B
:1044C000EA012A02FB01C701AD017A0163019801EB
:1044D0003E010701E600DA00CF000E001F20069320
:1044E00020F05EF9069B10B9012288F80020012B0C
:1044F00001F00580F278002A3EF42FAE059A12688A
:10450000D20441F1B482834A928807EE902AF8EEF1
:10451000E77A814991ED012AD1ED022A91ED033A22
:10452000D1ED043A91ED054AD1ED064A91ED075AD5
:10453000D1ED085A91ED096AD1ED0A6A91ED0B7A35
:10454000B4EE672AF1EE10FAF4EE672A14BF0122E6
:104550000022F1EE10FAB4EE673A18BF42F0010201
:10456000F1EE10FAF4EE673A18BF42F00102F1EEF4
:1045700010FAB4EE674A18BF42F00102F1EE10FAE9
:10458000F4EE674A18BF42F00102F1EE10FAB4EE01
:10459000675A18BF42F00102F1EE10FAF4EE675AC2
:1045A00018BF42F00102F1EE10FAB4EE676A18BFCC
:1045B00042F00102F1EE10FAF4EE676A18BF42F021
:1045C0000102F1EE10FAB4EE677A18BF42F0010270
:1045D000F1EE10FA18BF42F00102002A41F0AE815C
:1045E00091ED007AB4EE677AF1EE10FA41F0A6810F
:1045F0004A4ED4F898113268914201F2A68198F897
:104600000030012B3EF4A9AD94F89421002A3EF429
:10461000A4AD0B2B18D801229A4040F6030112EAF0
:10462000010917D112F4C06F0ED0093B012B0BD832
:10463000452011F0EDFFFF2011F0EAFF384811F09E
:104640005DFF484611F0E4FF364B32685A600B2399
:1046500088F80030002384F89431FEF77EBD012BEA
:1046600001F017820E23132088F8003006F060F85E
:10467000B3783CE7012B01D1F5F7AEFE0D231320F3
:1046800088F8003006F054F8B37830E7254A23491B
:1046900052680968C8328A4205D322F039FBB378E0
:1046A00000283FF424AF032B7FF41EAFDFF888907F
:1046B000D9F8000020F0F2FE1B4B1B780022022BE1
:1046C000C9F8002001D120F09DFCB3780CE7174B0E
:1046D0001B78002B01F0BA811A2020F061F8002825
:1046E00041F0B48194F89431002B41F0AF8109235B
:1046F00088F800301EF01CFFB378F8E6FCAF00200D
:104700000000008080A700208FC2753CD06D393A30
:1047100000000000C0AD0020C8AC0020407F002099
:104720005CC3030820B00020C88500202486002038
:1047300058550020C1550020705600201A2020F046
:104740002FF80028D6D0A64B1B88002BD2D1A54B22
:104750004520D3F8009011F05BFF0E2011F058FFB8
:1047600048461EF0CFFBDDF8249048461EF0CAFBF9
:104770009D4A4FF480510A234846118088F8003042
:104780001EF0D2FBB6E711F095FE984B00210520F4
:104790008DE80300A3F10802029153201FF096FB5D
:1047A00000287FF465AF924AB3781060082288F839
:1047B00000209CE611F07EFE8E4A0292A2F10C03CC
:1047C0004FF007090193CDF80090A2F108030021F2
:1047D000143A47201FF07AFB00287FF449AF844B3E
:1047E00088F800904FF0FF3283E80500B3787EE64A
:1047F00011F060FE1EF0B6FE00283FF439AF22F043
:1048000087FA00283FF434AF774AB3784FF48051E9
:1048100011800A2288F8002069E611F04BFE764BE1
:10482000002102208DE80300A3F108020291482034
:104830001FF04CFB00287FF41BAF6D4AB37810606B
:104840004FF0FF315160062288F800204FE611F04A
:1048500031FE6A4A0292A2F10C03252101930091D4
:10486000A2F10A035021163A49201FF02FFB00281D
:104870007FF4FEAE059B1B6813F0800201F0C0813F
:104880005B4AB37810604FF0FF315160052288F821
:1048900000202CE6DFF87CE19EF80030D90701F11A
:1048A000BA811F201FF07CFF00283FF4E1AE0C23EB
:1048B00088F80030DCE6DFF8389111F0FBFD504A53
:1048C000D9F80430126864339342BFF4D1AE40206B
:1048D00011F0C8FD00287FF4CBAED9F8003049496B
:1048E0004FF0400A0FE0069111F092FE0699D9F8B8
:1048F00000300A680133013ABAF1010A0A60C9F8C6
:10490000003001F03281404AD35C1846002BEAD1D6
:1049100001F030B93A4A364912684A6039480022F3
:104920000A600321026088F80010E0E5069B002B76
:1049300000F01586FDEEE47A10A901EB820217EE75
:1049400090CAFDEEE67A91462346524674462F48B9
:104950002F4F17EE908AB1EE433A9E46CA4613E0B7
:10496000FDEEC77A17EE903A634503DBAB42A8BF72
:104970002B46994607EE909AF8EEE77A5145E7EC18
:10498000017A00F1100027D090ED007AF1EC017A65
:10499000E7EE257AE146B0EE637AA3EE277AF0EEF1
:1049A000477A002ADCD0434634B1B4EE647AF1EEA3
:1049B00010FA48BFF0EE667AFDEEE77A17EE909AAD
:1049C000C14504DBA94517EE903AA8BF2B4607EE78
:1049D000903AF8EEE77AD1E77446FDF7B1BB00BF35
:1049E00070AE002080AE00201AB000206C9C03083E
:1049F00020B00020249C0308089C03085A9A03084E
:104A0000407F00206C560020E4990308F8AC002099
:104A100098850020CD7F0020BDEEE67A17EE107A53
:104A2000B0EE647AA3EE277AF0EE477ABEF1000F7B
:104A300040F02C83FDEEC77A17EE90CA17EE90EA8D
:104A4000AC45A8BFAE466745C8BFBE4607EE90EA74
:104A5000F8EEE77A012AC1ED007A3DF46EAB90EDF5
:104A6000047ADDED117AE7EE257AB0EE647AA3EEF2
:104A7000277AFDEEC77A17EE90CA17EE90EAAC459A
:104A8000A8BFAE46BC45B8BFBE4607EE90EAF8EEFA
:104A9000E77A022AC1ED017A3DF44FAB90ED087A36
:104AA000DDED127AE7EE257AB0EE647AA3EE277A8E
:104AB000FDEEC77A17EE90CA17EE90EAAC45A8BF94
:104AC000AE46BC45B8BFBE4607EE90EAF8EEE77AC0
:104AD000032AC1ED027A3DF430AB90ED0C7ADDEDA6
:104AE000137AE7EE257AB0EE647AA3EE277AFDEE2C
:104AF000C77A17EE90CA17EE90EAAC45A8BFAE464B
:104B0000BC45B8BFBE4607EE90EAF8EEE77A042A45
:104B1000C1ED037A3DF411AB90ED107ADDED147A1E
:104B2000E7EE257AB0EE647AA3EE277AFDEEC77A37
:104B300017EE90CA17EE90EAAC45A8BFAE46BC454A
:104B4000B8BFBE4607EE90EAF8EEE77A052AC1ED57
:104B5000047A3DF4F2AA90ED147ADDED157AE7EED1
:104B6000257AB0EE647AA3EE277AFDEEC77A17EEC7
:104B700090CA17EE90EAAC45A8BFAE46BC45B8BF98
:104B8000BE4607EE90EAF8EEE77A062AC1ED057A0E
:104B90003DF4D3AA90ED187ADDED167AE7EE257A8A
:104BA000B0EE647AA3EE277AFDEEC77A17EE90CACC
:104BB00017EE90EAAC45A8BFAE46BC45B8BFBE46AE
:104BC00007EE90EAF8EEE77A072AC1ED067A3DF49F
:104BD000B4AA90ED1C7ADDED177AE7EE257AB0EEF7
:104BE000647AA3EE277AFDEEC77A17EE90CA17EE25
:104BF00090EAAC45A8BFAE46BC45B8BFBE4607EE7E
:104C000090EAF8EEE77A082AC1ED077A3DF495AA12
:104C100090ED207ADDED187AE7EE257AB0EE647A31
:104C2000A3EE277AFDEEC77A17EE90CA17EE90EA48
:104C3000AC45A8BFAE46BC45B8BFBE4607EE90EA3D
:104C4000F8EEE77A092AC1ED087A3DF476AA90EDEC
:104C5000247ADDED197AE7EE257AB0EE647AA3EED8
:104C6000277AFDEEC77A17EE90CA17EE90EAAC45A8
:104C7000A8BFAE46BC45B8BFBE4607EE90EAF8EE08
:104C8000E77A0A2AC1ED097A3DF457AA90ED287A0D
:104C9000DDED1A7AE7EE257AB0EE647AA3EE277A94
:104CA000FDEEC77A17EE90CA17EE90EAAC45A8BFA2
:104CB000AE46BC45B8BFBE4607EE90EAF8EEE77ACE
:104CC0000B2AC1ED0A7A3DF438AA90ED2C7ADDED7D
:104CD0001B7AE7EE257AE3EE274AFDEEE47A17EE3B
:104CE000900A8542A8BF0546B842A8BF2F4607EEE6
:104CF000907AF8EEE77AC1ED0B7AFDF71EBA069BC3
:104D0000002B00F08784FDEEE67A10A901EB820209
:104D100017EE908AFDEEE47A914623465246744699
:104D2000CB48CC4F17EE90CA9E46CA4614E0FDEE23
:104D3000C77A17EE909ACC4503DCA9454B46A8BF2D
:104D40002B4607EE903AF8EEE77A5145E7EC017A08
:104D500000F110003FF440AE90ED007AF1EC017AE2
:104D6000E7EE257A6346B0EE647AA7EE837AF0EE3A
:104D7000477A002ADBD034B1F4EE474AF1EE10FA5C
:104D8000C8BFF0EE667AFDEEE77A434617EE909ADA
:104D9000C845D2DDD5E7FBF733FB0746FDF76ABA16
:104DA000AD48006810F080502AD0B6EE007A67EE69
:104DB000877AF4EEE75AF1EE10FA3FF52AABFFF7E7
:104DC0001DBB16F0805F7EF444ABFDF76EBAA34DB9
:104DD000A34EA44AD5ED004AD6ED003AA24D127872
:104DE000C4ED7F7AC4ED7D3AC4ED7E4AD5ED006A0C
:104DF000002A3CF463AB012284F80022FCF75EBB7E
:104E000011F4800001D00020CFE7B6EE007AF4EE76
:104E1000C75AF1EE10FAC8DCFCF748BEFDEEE67AA0
:104E2000284610AB8A49DFF82CC217EE907A7546F7
:104E300003EB82088646D1ED007AB3EC017AA7EE47
:104E4000A57A1031B0EE646AA3EE076A07EE907A95
:104E5000B0EE467A35B1F4EE464AF1EE10FAC8BF2C
:104E6000B0EE667ABDEEC77A17EE100A874204DC10
:104E70007045A8BF704607EE900AF8EEE77A434502
:104E8000ECEC017AD7D1FCF7B2BF012A40F3608481
:104E900007EE101AB8EEC77AC7EE876AB1EEE68A57
:104EA000B9F1030F14D0BAF1000F09D007EE90AAA0
:104EB000F8EEE77AF4EEC87AF1EE10FA00F1E38545
:104EC0002B6E03EB560393FBF6F3EB62FFF7D3B9BC
:104ED000B0EE480A22F01EFA00B2E4E7012A7FF79A
:104EE000FCA907EE101AB8EEC77AC7EE876AB1EED2
:104EF000E68AFFF7F4B9012A40F3178407EE101A87
:104F0000B8EEC77AC7EE876AB1EEE68AB9F1030F49
:104F100014D0BAF1000F09D007EE90AAF8EEE77AA4
:104F2000B4EEE78AF1EE10FA00F3AD856B6E03EB99
:104F3000560393FBF6F32B63FFF7B6B9B0EE480ABE
:104F400022F0E8F900B2E4E7484B494AB3F90430EB
:104F5000DFED487A82FB0312DB17C3EBA2031BB21F
:104F600008EE103AB8EEC88A28EE278AB0EE480A52
:104F7000F4F744FFF0EE408AB0EE480AF4F7C4FEBE
:104F80003D4BD878002800F0A1833C4AB4F98E113B
:104F9000B2F9023044F250665B1AB34200F3E28386
:104FA000374EB342BCBF03F50C43A03346429E428A
:104FB00000F3D6838342A8BF0346B2F90020B4F9B8
:104FC0008CE10B4419B2A2EB0E0344F250629342FF
:104FD000A4F88E1100F3C083294A9342BCBF03F5A5
:104FE0000C43A0339E4203DC9842A8BF18460646F5
:104FF0000EEB06031BB207EE903A07EE101AF8EE1E
:10500000E77AF8EEC76A27EEE87A60EE277AA0EE34
:10501000267AA4F88C31E8EEA67ADFED1A6A27EE3C
:10502000267A67EEA67ABDEEC77AFDEEE77A17EE2E
:10503000102A17EE903AA4F89021A4F89231FEF7C6
:1050400084B88223FEF7CBBFDFED0F7AFEF793BF64
:10505000F8AC002098850020FCAF00208CAE00202A
:10506000BCAD002090750020CCAD0020681F002052
:105070006766666635FA8E3C004400205C4400207A
:10508000B0B9FFFFCDCCCC3D00000243B4EEE47AD2
:10509000F1EE10FAB8BFF0EE667AFDEEE77A17EEA1
:1050A00090EA17EE90CAAE45A8BFAC467745C8BF98
:1050B000BC4607EE90CAF8EEE77A012AC1ED007A05
:1050C0003DF43BA890ED047ADDED117AE7EE257A08
:1050D000B0EE647AA3EE277AB4EEE47AF1EE10FA39
:1050E000F0EE477AB8BFF0EE667AFDEEE77A17EE9B
:1050F00090EA17EE90CAAE45A8BFAC46BE45B8BF11
:10510000BC4607EE90CAF8EEE77A022AC1ED017AB2
:105110003DF413A890ED087ADDED127AE7EE257ADA
:10512000B0EE647AA3EE277AB4EEE47AF1EE10FAE8
:10513000F0EE477AB8BFF0EE667AFDEEE77A17EE4A
:1051400090EA17EE90CAAE45A8BFAC46BE45B8BFC0
:10515000BC4607EE90CAF8EEE77A032AC1ED027A60
:105160003CF4EBAF90ED0C7ADDED137AE7EE257AA7
:10517000B0EE647AA3EE277AB4EEE47AF1EE10FA98
:10518000F0EE477AB8BFF0EE667AFDEEE77A17EEFA
:1051900090EA17EE90CAAE45A8BFAC46BE45B8BF70
:1051A000BC4607EE90CAF8EEE77A042AC1ED037A0E
:1051B0003CF4C3AF90ED107ADDED147AE7EE257A7A
:1051C000B0EE647AA3EE277AB4EEE47AF1EE10FA48
:1051D000F0EE477AB8BFF0EE667AFDEEE77A17EEAA
:1051E00090EA17EE90CAAE45A8BFAC46BE45B8BF20
:1051F000BC4607EE90CAF8EEE77A052AC1ED047ABC
:105200003CF49BAF90ED147ADDED157AE7EE257A4C
:10521000B0EE647AA3EE277AB4EEE47AF1EE10FAF7
:10522000F0EE477AB8BFF0EE667AFDEEE77A17EE59
:1052300090EA17EE90CAAE45A8BFAC46BE45B8BFCF
:10524000BC4607EE90CAF8EEE77A062AC1ED057A69
:105250003CF473AF90ED187ADDED167AE7EE257A1F
:10526000B0EE647AA3EE277AB4EEE47AF1EE10FAA7
:10527000F0EE477AB8BFF0EE667AFDEEE77A17EE09
:1052800090EA17EE90CAAE45A8BFAC46BE45B8BF7F
:10529000BC4607EE90CAF8EEE77A072AC1ED067A17
:1052A0003CF44BAF90ED1C7ADDED177AE7EE257AF2
:1052B000B0EE647AA3EE277AB4EEE47AF1EE10FA57
:1052C000F0EE477AB8BFF0EE667AFDEEE77A17EEB9
:1052D00090EA17EE90CAAE45A8BFAC46BE45B8BF2F
:1052E000BC4607EE90CAF8EEE77A082AC1ED077AC5
:1052F0003CF423AF90ED207ADDED187AE7EE257AC5
:10530000B0EE647AA3EE277AB4EEE47AF1EE10FA06
:10531000F0EE477AB8BFF0EE667AFDEEE77A17EE68
:1053200090EA17EE90CAAE45A8BFAC46BE45B8BFDE
:10533000BC4607EE90CAF8EEE77A092AC1ED087A72
:105340003CF4FBAE90ED247ADDED197AE7EE257A98
:10535000B0EE647AA3EE277AB4EEE47AF1EE10FAB6
:10536000F0EE477AB8BFF0EE667AFDEEE77A17EE18
:1053700090EA17EE90CAAE45A8BFAC46BE45B8BF8E
:10538000BC4607EE90CAF8EEE77A0A2AC1ED097A20
:105390003CF4D3AE90ED287ADDED1A7AE7EE257A6B
:1053A000B0EE647AA3EE277AB4EEE47AF1EE10FA66
:1053B000F0EE477AB8BFF0EE667AFDEEE77A17EEC8
:1053C00090EA17EE90CAAE45A8BFAC46BE45B8BF3E
:1053D000BC4607EE90CAF8EEE77A0B2AC1ED0A7ACE
:1053E0003CF4ABAE90ED2C7ADDED1B7AE7EE257A3E
:1053F000B0EE647AA3EE277AF4EEC74AF0EE477A6D
:10540000F1EE10FAC8BFF0EE667AFDEEE77AFCF72F
:1054100086BEBDEEE67AFCF72FBDD4F8BC61530022
:105420003EB1981801EB800076784078B042BBF42A
:1054300009AF134401EB83010023C4F8BC11A4F8A5
:105440000A32C4F80C32FBF7FDBE9FEDD07AFFF7AD
:1054500024B8830001EB030E04EB030CCC4B03EBED
:10546000C8185FEA990300F07C8301331B0107939E
:1054700008EB03000EF1100108F110030CF110020B
:1054800013ED024A13ED035A13ED016A13ED047A8A
:1054900051ED024A51ED035A51ED016A51ED047A82
:1054A00064EE244A65EE255A66EE266A67EE277A90
:1054B0001033834242ED024A42ED035A42ED016A43
:1054C00042ED047A01F1100102F11002D8D1079BDC
:1054D000103B08EB03020EEB0301634419F00309D0
:1054E0003EF497ABB2EC017AF1EC017A67EE277AE1
:1054F000B9F10109E3EC017AF4D1FEF78ABBA549C1
:10550000A54AC968126891423EF6F4AF98F80020A7
:105510000C3A022A7DF621AE94F8942188F80030E6
:10552000002A3DF41AAEFFF795B807EE906ADFED5A
:105530009B6AB8EEE77A66EEA65A9FED995A9FED00
:10554000996ADFED997AA5EE856A26EEA55AE5EE11
:10555000867AE5EE276A26EE870AFEF795BFFDEE0E
:10556000E67A10ABCDED087AFDEEE47A0B948F4F1E
:10557000DFF86082CDF82490544617EE90CADDF82B
:1055800020A00A91B1EE433A03EB8202CDF818E075
:1055900097ED007AF3EC017AE7EE257AB0EE637AC4
:1055A000A3EE277AF0EE477ADCB9FDEEC77AE6463D
:1055B00017EE909ACC4504DCA94517EE90EAA8BFF7
:1055C000AE4607EE90EAF8EEE77A002800F0438254
:1055D0009342E8EC017A07F11007D9D10B9CFCF754
:1055E000AFBD069931B1F4EE474AF1EE10FAC8BFEB
:1055F000F0EE667AFDEEE77A17EE90EAF24507EEF6
:1056000090AA04DCAE45A8BFAE4607EE90EAF8EEDD
:10561000E77ADAE7FDEEE47A10AB17EE90CAFDEE1A
:10562000E67A0B94614FDFF8AC81CDED087A5446F1
:1056300003EB8202CDF824900A91CDF818E017EE22
:1056400090AA05E09A42E8EC017A07F11007C5D06C
:1056500097ED007AF3EC017AE7EE257AB0EE647A02
:10566000A3EE277AF0EE477ADCB9FDEEC77AE6467C
:1056700017EE909ACC4503DCA945CE46A8BFAE46AE
:1056800007EE90EAF8EEE77A0028DBD10A990029C4
:10569000D8D109998E4607998E45B8BFF0EE667A43
:1056A000D0E7069931B1F4EE474AF1EE10FAC8BFDF
:1056B000F0EE667AFDEEE77AD64617EE909ACA4586
:1056C000DEDCD9E7F0EE627AFCF77AB9384B9FED71
:1056D000396AB3F90020B3F9023007EE902A06EEDA
:1056E000903AF8EEE77AF8EEE66A27EEE87A60EEAE
:1056F000277AA0EE267AE8EEA67A27EE067A67EEFB
:10570000867A90E4BCF838009FED2B7A07EE900A79
:10571000F8EEE77A294867EE877AC0ED007AFCF761
:10572000C4BDDFF8B490FCF716BE9FED188AFFF7F2
:10573000EDBB234A516900293BF415AC2149088887
:10574000214991FBF0F1106801605374FBF70BBC29
:105750009FED0E8AFFF7A4BBA3F50C43A03B41E4E9
:1057600033462AE4A3F50C43A03B1FE49FED170A40
:10577000174B0A9325EE800A21F0CCFDDFF85C8000
:10578000D4F8B061A8F80600FDF7F0BD00000000F5
:1057900084A1002070010020D085002084F9223FE0
:1057A00092E741B99730083C15A82ABEF8AC002012
:1057B0005C440020CDCCCC3D6F12833A9400002095
:1057C000207F0020387F002020A107000000C84271
:1057D00048A10020988500205855002060540020E2
:1057E00035FA8E3CDB0FC93F0000000007EE906ADF
:1057F000B8EEE76A5FED067A1FED067A84F88461F9
:1058000026EE276A76EE077AFDEEE76A16EE903A04
:105810002033402B40F247811FED0D7ADC4BFDEE2B
:10582000C67A83ED017A17EE903A2033402B00F2CE
:105830003781DFEDD87AB4EEE76AF1EE10FA40F383
:105840002082DFEDD55ADFEDD57A01E0B0EE666A51
:10585000B4EEE76AF1EE10FA76EE656AF6DCDFED9B
:10586000E17AF4EEE76AF1EE10FA40F10782DFED3B
:10587000CA5A9FEDCB6A01E0F0EE676AF4EEC66AA1
:10588000F1EE10FA76EEA57AF6D4DFEDC66AF4EE04
:10589000E67AF1EE10FA40F35081DFEDBE6A76EE63
:1058A000E77A67EEA75A9FEDC05A9FEDC06ADFED19
:1058B000C06AA5EE856A27EEA55AE5EE866AE5EE92
:1058C000267AC4ED627AFEF72CB8BA49BA4A8C46F9
:1058D000FEF78EB999ED000A08930791069221F020
:1058E00019FDDFF8F0E2DFF8F082DEF8ECE0DFF837
:1058F000ECC2A8F800008CFB0E3C4FEAEE70C0EB47
:10590000AC1007EE900AF8EEE77A069A0799089B22
:10591000FDEEE77A17EE900AA8F80200FCF720BD2A
:10592000FAF76EFDDFF8B082D4F8B491D4F8B06124
:10593000A0EB0A00A8F80200FEF7F7B99F4A126828
:1059400002F59C520832C4F8982198F80020012AE8
:105950007DF403AC94F89421002A7DF4FEAB032B74
:1059600000F0928121F0E6F9012384F89431FDF7EB
:10597000F4BBFAF745FDDFF860829BF80070A0EBFE
:105980000A00A8F80200FEF76DBBFAF739FDDFF850
:10599000488299F80020D4F8B0619BF80070A0EB21
:1059A0000A00A8F80400FEF7C9BB854B1B78002B42
:1059B00000F0CF800023FEF7C2BCDFED767AF4EE74
:1059C000E76AF1EE10FA40F35681DFED735A9FED6E
:1059D000736A01E0F0EE676AF4EEC66AF1EE10FA5F
:1059E00076EEE57AF6DCDFED7F6AF4EEE67AF1EE4C
:1059F00010FA40F13D81DFED685A9FED696A01E0E0
:105A0000F0EE667AF4EEC67AF1EE10FA77EEA56A59
:105A1000F6D4DFED647AF4EEE76AF1EE10FA04DD15
:105A2000DFED5C7A77EEE66A85E5DFED6D7AF4EE20
:105A3000E76AF1EE10FA44BFDFED6A7A77EEE66AC4
:105A400079E55D4901F1800CFEF75FBB09981DF017
:105A50006BFAFEF74FBE0A9900297FF4B9AD099998
:105A60008E4607998E45B8BFF0EE667AB0E5554A86
:105A70001278002A71D1544A128B07EE902AF8EE60
:105A8000E77AFEF746BDA8F80600A5F8A860FBF780
:105A9000E0BBF4F747FB00283EF4EAADFEF7E2BDB9
:105AA000DFED4A7A0DE7B4EEC76AF1EE10FA0FDDCA
:105AB000B0EE677ADFED385ADFED386A01E0B0EE1C
:105AC000677AB4EEE67AF1EE10FA77EEE57AF6DC74
:105AD0009FED447AF4EEC77AF1EE10FA0FD5B0EEEE
:105AE000677ADFED2D5ADFED2E6A01E0B0EE677ABE
:105AF000B4EEE67AF1EE10FA77EEA57AF6D49FEDE1
:105B0000297AF4EEC77AF1EE10FA6DDD9FED217A75
:105B100077EE677A67EEA75A9FED235ADFED236A87
:105B20009FED237AE5EE856A27EEA55AA5EEA67AC3
:105B3000E5EE077AB0EE677A70E6DFED296AF4EEFB
:105B4000E67AF1EE10FA44BFDFED266A76EEE77AE8
:105B5000A7E604F0D1FDFBF775BBDFED1C7AFEF77D
:105B6000D8BC634671464246B8E4194AD35C002B60
:105B70007EF47EAD00234FF0FF32C9F800300423DD
:105B800088F80030C9F80420B378FEF7B0BC00BF35
:105B900094000020DB0F4940DB0FC940E4CB1641E5
:105BA000E4CB16C1DB0FC93F92E741B99730083CFF
:105BB00015A82ABE04A30020B8230020407F00209F
:105BC00057550020907500206875002000000000E7
:105BD000E4990308D817002060540020D34D6210C8
:105BE000DB0FC9BFDB0F49C01FED037AF4EEC77AA4
:105BF000F1EE10FA44BF1FED057A77EE677A89E778
:105C00003E49B3780A604FF0FF324A60072288F8B5
:105C10000020FEF76CBC802011F00EF808B11FF0D8
:105C200067FC21F087F8FEF73CBE9BF800101329B3
:105C300013D0002B43D113297DF4D7AAB0EE480A24
:105C400021F068FBA8F80200FDF7D1BA94F8E8311A
:105C5000002B7BF4AAA9FBF793B9B0EE480A08938E
:105C6000079121F057FB0799A8F80000089BE0E78F
:105C7000F0EE676ACDE6F0EE667AB4E6F0EE667AAC
:105C800003E6F0EE466AEAE5802010F0D5FF002832
:105C90007DF463AA66E694F8D831EBB10A9BD3EDA4
:105CA00003DA174B93ED020A164B38EE6DDA29EE44
:105CB000000A20EE0D0A83ED020AFBF70ABB06F587
:105CC000F460B0EE480A2844D5F89C3798479BF812
:105CD0000010B0EE408AAEE7094B2B4493ED000A6A
:105CE000059BD3ED01DA29EE000A38EE6DDA20EEDD
:105CF0000D0A88ED000AFBF7ECBA00BF20B00020C7
:105D0000144000206485002003680A7A591C016051
:105D10001A70704738B50B4C23688BB15A68821AD9
:105D2000002A054604DA0CE05A68AA1A002A07DBA2
:105D30009A68226018461A6890472368002BF3D1AE
:105D400038BD38BD2485002070B54E680546304604
:105D500020F084FA314604460246286821F066F9AC
:105D60002A68131901333B212B60115570BD00BF08
:105D700008B51BF023FCF4F7FDFC00BF024A034BFF
:105D8000127819780DF0DCBDA8230020A92300208B
:105D9000F0B5474B1A6883B00123500200935CBFF3
:105DA00003F180530093D100424909685CBF43F07E
:105DB000100300938F0748BF43F0C6033E4948BF16
:105DC0000093160648BF43F44063097848BF009328
:105DD000D40548BF43F0006301F0EF0048BF0093D3
:105DE00008286D465BD00E2959D0D0033348009B5C
:105DF00000784CBF43F4204343F40053D7044CBF16
:105E000043F0644343F0444300280CBF07200F20B5
:105E1000960648BF43F48073540748BF43F40033E9
:105E200043F400245205009403D5254A1279002A30
:105E300039D1182908BF009B019004BF43F060735B
:105E400000930027012639462846FCB2F4F7ADF846
:105E500060B11C4B002203F5D87103E08B420FD0D8
:105E600013F80C2C944203F10C03F7D10137242FC3
:105E7000E9D195E80300144B83E8030003B0F0BDBB
:105E80007A0904F01F0455F8223006FA04F40137A9
:105E900023EA0404242F45F82240D4D1E9E743F44F
:105EA00080530093A1E743F4C0130093C1E700BF00
:105EB000747A00205CA1002034230020907500201B
:105EC000F4540020A0970308A02300202DE9F84FE8
:105ED0004E014FF0000B174D8146904606F120070A
:105EE0005C46594628465FFA8BFAF4F75EF8C0B173
:105EF000A64215D8A74213D900200F4A014604E054
:105F00000131242914D012F80C0C504502F10C0276
:105F1000F6D10A4B01EB410103EB81014846C04732
:105F200001340BF1010BBBF1240FDAD1BDE8F88F7E
:105F30000021F3E7A0230020A0970308949703080B
:105F400000210A4A0B4604E00133242B0BD012F83F
:105F50000C1C884202F10C02F6D1054803EB430306
:105F600000EB830070470020704700BFA89703082C
:105F70009497030800210A4A0B4604E00133242BBE
:105F80000BD012F80C1C884202F10C02F6D1054825
:105F900003EB430300EB830070470020704700BF12
:105FA000A0970308949703081C4C08B50121022010
:105FB000FAF712FD237803F00502052A29D003F031
:105FC0000903092B08D000210120FAF705FD002163
:105FD0000846FAF701FDFEE7114A124B11681A68EC
:105FE0000B68114C23F001030B601388206823F029
:105FF00001031B041B0C138018B12922002382719A
:10600000C37109224A21F9F779FC2068F2F77CFE76
:10601000D9E71BF083FB2378D1E700BFE0390020EC
:10602000C4B00020C8B00020D8B00020022828BF8B
:10603000022010B4084C094B207000EBC00200EBAA
:10604000820207495DF8044B013003EB4203C0B202
:106050000B6004F081BC00BF99550020B4440020BF
:106060005421002008B5F9F7D7F919F035FAF3F7FC
:10607000ADF9BDE8084019F017BA00BF08B519F02E
:106080002BFAF3F7A3F9BDE8084019F00DBA00BFE9
:106090002DE9F047A84FA94E19F01EFABE421ED2B4
:1060A000DFF82483DFF824934446258862197DB104
:1060B0004A450DD2052D0BD933886188C3F30B03F4
:1060C000994200F0D880144625886219002DEFD13E
:1060D000716830461436F3F7FDF8BE42E4D3984AAF
:1060E0005378022B40F2EC800023964953701378CA
:1060F0009548022B016000F2DF8003EBC301934A55
:1061000003EB810302EB4303914C184623600BF031
:1061100099F8904A1378A3F1170102290FD98E49F3
:1061200011F83300002840F0D180D80001444978AC
:1061300029B18A4911F83330002B00F0F580884BE3
:106140009A78042A00F0E78032B91A88B2F5F07F15
:1061500084BF4FF4F0721A80824D834A2B681A4034
:10616000002A00F0E480DE0700F1D080580400F13E
:10617000C880190700F1C0809A0100F1B7809B0424
:1061800000F1AD8023689A8CD98C914224BF002203
:106190009A84F9F7C1F812F0DDF910B9734803F0E9
:1061A000B1F91EF075FB00213022714823F0BDF9D2
:1061B000704B256803F1500102E00433994279D015
:1061C0001A78002AF9D19C78D8788442F5D26A49A5
:1061D0006A4B0A7028461D600CF00AFF684B694A3A
:1061E0001E78694969486A4B1160C825642212FB10
:1061F0000652684C006B31F8041C5A600022218062
:106200009A60DA601A615A619A61DA6183F8202033
:1062100083F8212008B119F09BF85F4B9FED5F5A7E
:106220001B885F4A9FED5F6A55795F4C5F49604804
:10623000086006EE903AF8EEE66A1388C5EE265A34
:1062400007EE103A53881279C4ED005A07EE903ADF
:10625000B8EEC77A574BF8EEE77A1D725A7227EEFE
:10626000067A67EE867ABDE8F04783ED017AC3EDE2
:10627000007A19F019B963799B077FF424AF71682C
:1062800094F804A03046F3F725F83388BAEB133FAF
:106290000BD173887068AA1FC3F30B039A4204F1F1
:1062A0000601A8BF1A4620F0C1FE1436BE42FFF414
:1062B000FBAE14E701228AE700231370234B23E788
:1062C000204903EB430301EB830110E7D8000D18CD
:1062D0006D68002D7FF42AAF1725157026E7364824
:1062E000F3F72EF84020F3F72BF84BE746F20900BE
:1062F000F3F726F82B6842E73048F3F721F82B68CC
:106300003AE72F48F3F71CF82B6832E72D48F3F7EC
:1063100017F82B682AE71A8BB2F57A7FBFF41CAF07
:106320004FF47A721A8317E71823137007E743F0C4
:1063300008032B6017E700BFAC05000888010008C0
:1063400099550020B045002058210020B444002079
:10635000542100203423002028A60308B8A20308F3
:10636000687500204046002009600002DC9800208B
:106370008C260020D4850020D81B0020C0260020B9
:10638000D4AD002030B100203CB00020241F0020FC
:106390006821002084840020C8240020C0C9FB4854
:1063A000CC25002017B7D138CC240020CCA7002062
:1063B0003661023DA8A700200940000201600002EA
:1063C0000920000208600002074000080080000861
:1063D0002DE9F0430B684A680B388BB00C46D51A90
:1063E000EF2800F27881DFE810F07C017601760179
:1063F00076017601760176017601760176017601E5
:1064000076017601760176017601760176017601D4
:1064100076017601760176017601EA0176018A023B
:1064200076017B02760176017601740276012602FE
:106430007601D2017601C1017601BA01760194019B
:106440007601520176017601760176014D017601E1
:106450007705760176016A05760176017601760187
:1064600076017601650576017601760146057601AD
:10647000C105760176018405760176017601760103
:10648000760176017601F0007601D0047601E80508
:1064900076010605760134057601760176017601EE
:1064A0007601760176017601760176017601760134
:1064B0007601760176017601760176017601760124
:1064C0007601760176017601760176017601760114
:1064D0007601760176017601760176017601760104
:1064E00076017601760176017601760176017601F4
:1064F00076017601760176017601760176017601E4
:1065000076017601760176017601760176017601D3
:1065100076017601760176017601760176017601C3
:1065200076017601760176017601760176017601B3
:1065300076017601760176017601760176017601A3
:106540007601760176017601760176017601760193
:106550007601760176017601760176017601760183
:1065600076017601A4047D04640476012704F30314
:10657000E7037601DC03AE039C0397036D0376010A
:106580005A03760176014B0336032E031C030C03DA
:10659000FD02E90276017601760176017601760147
:1065A0007601760176017601760176017601760133
:1065B0007601DE0276017601B3027601760176017C
:1065C00076017601760176011B020846F3F70DF994
:1065D00005460DF0A9F9FF2854D0B5F57A7F80F073
:1065E0002F850AAF002307F8243DEE0839460DF148
:1065F00003008DF8033001360CF080FD9DF8033068
:10660000F6B205F00705B34205F1010503D19DF887
:106610000430AB4203D0294630460DF071F994E8BE
:106620000C009B1A012B2DDD531C0AA823600023AC
:10663000157800F8253D0CF055FD9DF80330AB4270
:106640000AD0B44B1B683BB19A79AA4204D31B68A9
:106650001B690BB12846984723685A1C22603846AC
:1066600000221C788DF804200CF030FD9DF80430D9
:10667000A34207D0A74B1B6823B11B685B690BB112
:1066800020469847012318460BB0BDE8F083A24985
:10669000A1FB05216A1A01EB52018908C1EBC10275
:1066A000B5EB020817D1C9B24E1EF6B20029E9D0E7
:1066B000DFF8689201365A1C226093F90010974B5C
:1066C000002593F902208A4203F1080300F0938425
:1066D0000135062DF5D14FF0FF3318460BB0BDE85C
:1066E000F0838F49102D4FF0000328BF10250B6059
:1066F0004B608B60CB600B74002DC3D023685A199C
:106700000133236013F8010C01F8010B9A42F7D111
:10671000B8E75A1C0A601A780E2ADCD8991C216046
:1067200058780328D7D87F4D02EB42025200A918AF
:10673000DE1C487126609878A8541A1D2260DA7809
:106740004A705A1D22601A798A709A1D22605A79FD
:10675000CA70DA1D22609B790B71012393E75A1CE2
:106760000A60714A1B78537501238CE75A1C0A6032
:106770001E781F2EAFD8052DADD10846F3F71EF8B1
:106780006A4B43F826000BF03DFD01237BE7674D84
:1067900005F140062046F3F728F82368A5F88000A5
:1067A000591C1A46216012F8021B85F882102260DB
:1067B0005B7885F883300435AE42EBD162E75A1C32
:1067C0000A601E78132E86D89A1C0A6000205D7815
:1067D0005749024605E00132242A3FF47CAF11F804
:1067E0000C0C854201F10C01F5D15248524902EBE3
:1067F000420210F8222001F82620D81C206001EB6C
:10680000860299785170191D2160D8789070581DB2
:1068100020604A491B790868D3701DF0C7FF31E733
:10682000474B1B78DB073FF556AFFFF727FCFFF719
:106830002FFC012327E75A1C0A603B4E1B7833725A
:106840000846F2F7D2FFB0832046F2F7CEFF30833E
:106850002046F2F7CAFF236870835A1C22601B7817
:10686000F374082D7FF60EAF2046F2F7BEFFF084DA
:106870002046F2F7BAFF0C2D30857FF603AF236870
:106880001A46591C216012F8021BB17722605B780E
:1068900086F820302046F2F7A8FF102DB0847FF64E
:1068A000F1AE23685A1C22601B78F3722046F2F77F
:1068B00085FF2368F0605A1C22601A783274162D06
:1068C0007FF6E0AE9A1C22605B7886F821300123C7
:1068D000D9E65A1C0A601B4A1B7813700123D2E6C2
:1068E0000846F2F782FF184D28602046F2F77DFF38
:1068F00068602046F2F779FF0123A860C3E6134DD4
:1069000000232B600846F2F759FF2B6818432860D4
:106910000123B8E68044002025499224DC98002019
:106920009E550020D83B0020447A0020088000209B
:10693000A897030894970308D485002054210020C9
:10694000CD7F002034230020083A0020404600205C
:106950005A1C0A601A780F2A3FF6BDAE991C2160B6
:10696000C2EBC202A04958788854D81C20600A445F
:1069700099785170191D2160D9789170591D216045
:106980001979D170991D216059791171D91D216032
:106990009979517103F108012160DB7993710AF053
:1069A000BDFB01236FE60846F2F71FFF8F4DA8815C
:1069B0002046F2F71AFF0123688164E619465A1C43
:1069C00022608B4A11F8020B1070216059785170C7
:1069D000D91C216099789170191D2160DB78D370E2
:1069E000012350E60846F2F700FF824DA8822046B8
:1069F000F2F7FBFEE8822046F2F7F7FE0123288338
:106A000041E61A46591C216012F8020B2260DA1C7A
:106A1000597822609A7817F039F800287FF432AE5E
:106A200059E61A46591C2160734912F8020B087086
:106A300022606E495A788A70DA1C22606F4A9B780D
:106A4000937001231FE66E4B6E4918684A2220F0AE
:106A5000EDFA012317E619465A1C22606A4A11F81A
:106A6000020B1070216059785170D91C21609B78FD
:106A700093702046F2F7B9FE644A0123D08002E603
:106A80000846F2F7B2FE614D28802046F2F7ADFECF
:106A900068802046F2F7A9FE0123A880F3E55C4F49
:106AA0003B78002B3FF4EEAD5A4E00252046F2F71E
:106AB0009CFE1AF04DFD3B78A6EC010A0135AB4275
:106AC000F4DCDFE50F2D7FF406AE5A1C0A601D785A
:106AD000072D3FF600AE08464F4F05EB4505F2F790
:106AE00084FEAD007E19B0802046F2F77EFEF08075
:106AF0002046F2F77AFE236830811A46591C21603D
:106B000012F8021BB17222605B78F3722046F2F732
:106B100055FE01237851B6E50846F2F766FE0123DB
:106B2000B1E55A1C0A601878050600F1EB823B4B70
:106B30001B78DC073FF5A6AD032828BF0020FFF730
:106B400075FA01239FE55A1C0A6008461D78F2F782
:106B500035FE80462046F2F731FE07462046F2F722
:106B60002DFE06462046F2F740FE2046F2F73DFE97
:106B7000236801332360002D00F0B082102D7FF4D4
:106B800081AD274BC3F800805F600EB1254B1E60BE
:106B90002549264B0222081F1A700CF0D9F901234F
:106BA00071E51E4B1B78D8073FF56CADFFF75AFA1D
:106BB000FFF76EFA012366E5184B1B78DA073FF5FD
:106BC00061AD1B4A137843F00403137001235AE5A7
:106BD000124B1B78D9073FF555AD164B4FF4C872D1
:106BE0001A8001234FE500BF9C3F002038B00020F1
:106BF00060410020687500201099002050B00020EE
:106C0000542100208CB0030830B00020C0AD00201B
:106C10004D540020C8AC0020A83E0020CD7F0020AD
:106C2000C4260020AC230020C8260020704300208A
:106C30007E1F0020B0B00020092D7FF64CADB84F6C
:106C40001A46591C3E68216012F8021B31702260FE
:106C50005A78B270DA1C22609A78642A03F104012F
:106C6000A8BF642272712160DA78642A03F10501F9
:106C7000A8BF6422B27121601A79F2719A1D226054
:106C80005A79642A28BF6422D91D327221609A7908
:106C9000F27003F108022260DB7933712046F2F7CB
:106CA000A4FD0A2D708140F037821DF0F1FD012313
:106CB000E9E49C4A1068DA1C01462133951E2560E0
:106CC00012F8035C0D70551E256012F8025C4D70C1
:106CD000226012F8015C8D7003329A4201F10301C7
:106CE000ECD1B2E05A1C0A601A788F49002A00F0F1
:106CF000A3810A7842F00202981C0A708B4D206032
:106D00005B782B702046F2F759FD68602046F2F759
:106D100055FDA8602046F2F768FDA8812046F2F7ED
:106D200064FD834A6882137843F0020313700123E1
:106D3000A9E4C5F34705122D3FF6CDACBDB10AABB2
:106D40000DF1020703EB45083E46A8F12608204650
:106D5000F2F74BFD26F8020FB045F8D1754B37F826
:106D6000022F23F8022FBE42F9D1112D09D8724A01
:106D70006B00023B13440021223223F8021F93428E
:106D8000FBD16E4A012313707DE41A46591C216021
:106D90006B4E12F8021BB17022606A495A780A7071
:106DA000DA1C2260684D9A782A711A1D2260DB78FD
:106DB000092BA8BF09232046AB70F2F716FD236804
:106DC00062682880D11A012905DD2046F2F70DFD01
:106DD000626823686882934240F05781F8F79CFA12
:106DE000236862689A423FF44DAC5A1C22601B78BB
:106DF000EB70012347E40846F2F7F7FC2046F2F770
:106E0000F4FC2046F2F7F1FC2368464F9A1C3E68DA
:106E100022605A7886F82F20DA1C22609A7886F849
:106E20003A201A1D2260DA7886F83B200733236067
:106E30002046F2F7DAFCF08720463E68F2F7D5FCF0
:106E4000112DB08700F2138138680AF041FB01234D
:106E500019E41A46591C21603C4912F8020BC8700B
:106E600022603B495A780A70DA1C2260394A9B78C2
:106E7000D370012307E41A46591C2160364D12F8DD
:106E8000021B297022605B786B702046F2F7ADFC24
:106E9000236868805A1C22601B782B712046F2F709
:106EA000A4FC2368E8805A1C22601B782B72012303
:106EB000FFF7E9BBF3F790FA0123FFF7E4BB274A9A
:106EC00003F108000133236013F8011C02F8011FCD
:106ED0009842F7D1FFF7D6BB591C1A4621602049CA
:106EE00012F8020B887022605B784B700123FFF769
:106EF000CABB1C4A1278012A3FF6C4AB19465A1C79
:106F00002260194A11F8020B9070216059781170B3
:106F1000D91C21609B7853700123FFF7B4BB00BFDD
:106F200058210020542100207E1F0020801F0020B7
:106F30006E430020D67A0020D87A0020FC7A002008
:106F4000109900202CB000206875002038B0002077
:106F500048B0002050B00020D4AD0020437A00207B
:106F60005CB00020C1550020C25500205A1C0A60A8
:106F70001E78112E3FF6AFAB9A1C0A606D4D5B7800
:106F800005F816300846F2F730FC40F6CA0398427E
:106F9000A8BF184640F2EE239842B8BF1846664B89
:106FA000A0F2EE2083FB002305EB4605C017C0EBE3
:106FB000E3036B700123FFF766BB5A1C0A605F4F47
:106FC000DFF88C811B783E6888F805300846F2F7B8
:106FD0000CFC308420463E68F2F707FC052D7084D7
:106FE0005BD8F8F799F918F029FF38681AF0E8F833
:106FF0000123FFF748BB09EBC5072046B970F2F73C
:10700000F4FB216829F835000B464A1C226013F86E
:10701000022BFA7023604B783B71CB1C23608B787A
:10702000BB710B1D236008F10108CA787A714645CF
:107030007FF441ABFFF726BB0A7802F0FD025BE666
:1070400001AF38460CF036F8BDF80430AB423FF4DF
:10705000E6AA3B4B1B68002B3FF4E1AA1B689B6927
:10706000002B3FF4DCAA28469847FFF7D8BA2368DC
:107070003868591C1A46216012F8021B80F831103A
:1070800022605B7880F83230DFE65A1C22601B7881
:10709000003318BF0123F371A0E62046F2F7A5FBE9
:1070A000A8F80A002046F2F7A0FBA8F80C0020463A
:1070B0003E68F2F79AFBB08420463E68F2F795FBF3
:1070C0000D2DF0848DD92046F2F78FFBA8F80E0025
:1070D0002046F2F78AFBA8F8100082E7194B10202F
:1070E000C3F800805F6003F04FFC174A137843F049
:1070F00001031370002E3FF4C5AA144A0123166041
:10710000FFF7C1BA00F07F00032828BF002005F078
:10711000CDFB0123FFF7B7BA23683A68591C2160F9
:10712000197851720B2D1FBF991C21605B78537029
:10713000BBE500BF987C00201F85EB515421002047
:1071400080440020902100207E1F0020AC230020DE
:107150001099002008B518F0BFF9F2F737F918F0C8
:10716000A3F9FEF795FF0120BDE8084003F0F4BB4A
:107170002DE9F04F2DED028B994A9A49137895B07D
:1071800000F59C4808F120080990C1F80080002B08
:1071900000F0AC8694490968884240F29480934993
:1071A0000591D1F800B092489249934C0290013B6E
:1071B00013700BF4805303910893002B40F09280DE
:1071C000039B5B7D002B40F0FD841BF4004F41F0DE
:1071D00054801BF4807F0BD0099A884BDFF850A2B3
:1071E0009A429AF8022001F22682002A41F0278270
:1071F000834B844D06931BF4805940F05F86039BBC
:10720000B4F906605B8B9E42B4BF00260126DFF80E
:107210001882D8F8003013F0805370D0069A127894
:1072200012F0010272D003987749808C91ED037AB5
:10723000049107EE900AF8EEE77AB4EEE77AF1EE01
:1072400010FA81F2F580002E68D1029991F8A4100D
:10725000002963D16D486E49006890F8300000271E
:107260000F604F608F606B49002858D10870002A6A
:1072700059D01BF0100F56D0674A1278D20652D45C
:10728000B9F1000F4FD1002B4DD11BF4800F4AD123
:107290002F78002F02F09980604B9B78002E42F0EF
:1072A000DA803BB15E4A5F4B12681B689B1A002B69
:1072B000C2F2B780102003F03BFA029A2F78012324
:1072C00082F8A53030E0494B0593D3F800B0494B24
:1072D000474A03930BF480530292474C0893002BC8
:1072E0003FF46EAF00215048F2F75FFE00287FF4B4
:1072F00067AF04F067F9059BD3F800B060E71BF4B3
:10730000800F8BD1069A127802F0010202980021B8
:1073100080F8A4103C490491002E9BD03D490120E7
:107320000870002AA5D12F78039AB4F900C0518BB8
:10733000928BB4F902008C45CCBF4FF0800E4FF019
:10734000000E4EF040039445A8BF73469B0843F0DF
:10735000800E8842C8BF734643F0400E9042B8BFCB
:1073600073469B08B4F904E0B4F9060043F0800CBE
:107370008E45C8BF634643F0400C9645B8BF634690
:107380009B0843F0800E8842C8BF7346029943F0C1
:10739000400E91F8A6C09042B8BF73469C4500F0DD
:1073A0007D864FF0000C81F8A63081F8A7C0002F31
:1073B00000F0E987059B1B6803F00403002B40F0F5
:1073C00057850DF1480B194D0023CBF8043005F11A
:1073D0005009129340F6330A192740F283362CE005
:1073E0005C8600208084002058860020747A00206B
:1073F000DC250020447A002010230020404B4C0064
:10740000CD7F0020D81B002058550020542100209B
:1074100070850020A02500207E1F00205CB0002089
:10742000407F0020DC2B0020FCAF0020D485002012
:107430006821002004354D4520D0AA78EB789A4287
:1074400017FB0261F6D26A78043217FB036334F942
:1074500012205245A8BF5246B2F5617FB8BF4FF423
:1074600061729142E6DA9A42E4DC29782329E1D874
:1074700058460435F2F78AFD4D45DED15F4B9BE857
:1074800003001E7888E80300002E00F077845C4B30
:1074900007935C480121F2F788FD002840F09782AD
:1074A000059B1B68D80500F18D82574F574D2B88DF
:1074B0001EB226F001061FFA86F94B45A5F800908A
:1074C00000F05A86524E4FF002080F204FF0140B76
:1074D0004FF0FF0A86F8008086F801B086F802A017
:1074E00003F026F941464748B5F80090F2F75DFDF4
:1074F000002841F02D8229F002039BB24B452B80DE
:107500000BD0434B1421FF2202260F201E7059700E
:107510009A7003F00DF9B5F800903E4BDFF800A12A
:107520001978DAF80400089319F0030F08BF81F006
:107530000201C1F34001F1F705FC3B6813F00A0FAB
:107540001CD005212F48F2F730FD002800F00687F7
:107550002E88720741F174812A480621F2F725FD31
:10756000002800F0E886730641F162810721254872
:10757000F2F71BFD002840F046833B68980600F1B7
:1075800051832E881F480C21F2F70FFD002800F0D0
:107590003D8246F48073B3422B8009D01C4B0226F7
:1075A0001421FF220F201E7059709A7003F0C0F84A
:1075B000194B1B78082B00F035820E2B00F032821D
:1075C000059B1B6858055CD5144B1B79002B00F0FC
:1075D000178114210B48F2F7E8FC002840F01581D0
:1075E00015F006FF012002F0F5FF002849D0DFF872
:1075F000349000264FF0CC0B19E000BF6743002009
:1076000058210020FCAF00205CA100205021002068
:10761000F03C0020087F002034230020F454002098
:107620000C7F0020D46F0020DEB2022E29D80BFB85
:1076300006F8731C59F80870002FF5D1C378CB4AAF
:1076400090F9020052F823300197032200920121A1
:107650003A4601F099FF034606EB460000EB0010A6
:10766000029353B1394609EB8000CC2221F05DFF33
:10767000029B49F808300136F6B218F085FB002865
:10768000D3D1069B1E7816F0010600F0F881B84BA6
:1076900001221A70079BB4F906101B68B5485A8975
:1076A00001279142077080F2D081B34B4FF07E5298
:1076B0001A60B24A039BB4F900C01F8B92F90430E0
:1076C00092F801E01078002BACEB070314BF012205
:1076D0004FF0FF32002B40F35D82B3F5FA7FC0F22A
:1076E0005F824FF4FA731B1A07EE903AF8EEE77ACE
:1076F000049B6745C3ED007A03DDF1EE677AC3EDC5
:10770000007AB4F902C0ACEB0703002B40F34E82C1
:10771000B3F5FA7FC0F250824FF4FA731B1A07EEEA
:10772000903AF8EEE77A049B6745C3ED017A03DDF2
:10773000F1EE677AC3ED017AB4F90400C31B002BA4
:10774000D8BF3B1AB3F5FA7F80F20A827345D8BFDF
:107750004FF0000E00F3068202FB0EF207EE902AB5
:10776000049A059BF8EEE77AB842C2ED027ABCBFF4
:10777000F1EE677AC2ED027A1A6812F4805200F0D4
:10778000F481B1F5FA6FA8BF4FF4FA61B1F57A7FD1
:10779000B8BF4FF47A71A1F57A71794C794884FBBE
:1077A000013ECB17C3EB6E1303F1010E6FF0630CB8
:1077B00030F91EE030F913000CFB0313AEEB0001AF
:1077C00003FB01F384FB0314DB17C3EB64130344D3
:1077D0001BB207EE903A049BB8EEE78A83ED038A6A
:1077E000002A40F057822B885A0624D4002E40F0FD
